:10C00000F46D0020E5400200F74002000D410200FF
:10C010000F4102000F4102000F410200000000002A
:10C020000000000000000000000000000F410200BE
:10C030000F410200000000000F4102003306010022
:10C040000F4102000F4102000F4102000F410200A8
:10C050000F410200030C0200A50902000F4102007B
:10C06000C59801000F4102000F4102000F4102007C
:10C070000F4102000F410200011A0100DDC500005E
:10C080000F410200CBAF01002B0601000F4102005F
:10C090000F4102000F4102000F410200691A010026
:10C0A0000F4102000F4102000F4102000F41020048
:10C0B0000F4102000F4102000F4102000F41020038
:10C0C0000F4102000F4102000F4102000F41020028
:10C0D0000F4102000F4102000F410200B73202007F
:10C0E0000F4102000F410200000000000F4102005A
:10C0F0000F4102000F4102000F4102000F410200F8
:10C100000F4102000F410200CDC700000F410200A5
:10C1100000000000000000000F4102000F4102007B
:10C120000F4102000F4102000F4102000F410200C7
:10C130000F410200FB1101000F4102000F410200FC
:10C1400000000000000000000000000000000000EF
:10C150000F4102000F41020003B001000F41020035
:10C1600000000000000000000000000000000000CF
:10C1700000000000000000000000000000000000BF
:10C1800000000000000000000000000000000000AF
:10C19000000000000000000000000000000000009F
:10C1A000000000000000000000000000000000008F
:10C1B0000F4102000F4102000F4102000F41020037
:10C1C00053C300000F4102000F4102000F41020063
:10C1D0000F4102000F410200C14B0100014C010060
:10C1E0000F4102000F4102000F4102000000000059
:10C1F000000000000F4102000F4102000F41020049
:10C200000F4102000F41020000000000000000008A
:10C210000F4102000F4102000F4102000F410200D6
:10C220000F4102000F4102000F4102000F410200C6
:10C230000F4102000F4102000F4102000F410200B6
:10C240000F4102000F4102000F4102000F410200A6
:10C250000F4102000F4102000F4102000F41020096
:10C260000F4102000F4102000F41020010B502F021
:10C27000C3FC0421DFF8F80703F08CFE0020DFF890
:10C28000F41708600821DFF8F00703F083FE0020B0
:10C29000DFF8E81708600020DFF8E41708700A20CC
:10C2A000DFF8E01708700120DFF8DC17086002F003
:10C2B0002FFE02F070FE002003F02AFF30280FD17D
:10C2C000012003F025FF30280AD140F2D920DFF801
:10C2D000281908604FF42D70DFF82019086009E074
:10C2E00040F2F320DFF81019086040F2FD20DFF87B
:10C2F0000C190860DFF80849206830F01000206051
:10C3000002F0AAFE022002F0D9FB0020DFF8F418A8
:10C3100008700020DFF8F01808700020DFF8EC1833
:10C3200008600020DFF8E81A086004F065FB0028C8
:10C3300004D1206830F48070206003E0206850F45D
:10C340008070206003F04CFB206850F001002060FA
:10C3500010BD80B51521DFF8B80804F072FD04F0B7
:10C360004EFEDFF89C080068C00703D4042005F0E7
:10C370002CF93CE0032005F0BDFADFF898180860BE
:10C38000DFF894180868012810D1DFF89028107899
:10C39000002805D01078052802D01078042805D18F
:10C3A00000200860DFF8780805F0D5F803F05FF8A2
:10C3B000DFF8D0060178112906DADFF8581A00787C
:10C3C00051F82000804704E0042005F0FEF801F059
:10C3D000E3FD01F01EFE01F067FE01F0A5FE02F094
:10C3E0009DF802F0F3FA02F0C3FB04F0AAFE01BDCF
:10C3F00010B4DFF88C4620700400E4B2012C02D0A7
:10C40000C0B2022809D1DFF81C080160DFF8180863
:10C410000270DFF8040A03700BE00020DFF8041854
:10C4200008600020DFF8001808700020DFF8E81925
:10C43000087010BC7047DFF8E40900687047DFF847
:10C44000E009006870470120DFF8CC1708607047EA
:10C45000DFF8D8070068012801D1062002E0DFF8E4
:10C46000BC0700787047DFF8BC0900687047DFF848
:10C47000A00900687047DFF8940700687047DFF88C
:10C48000A8090068DFF878271168C1F34011002976
:10C4900011D11168C1F3C011002906D08821484389
:10C4A0004FF4FA6190FBF1F005E0942148434FF41A
:10C4B000FA6190FBF1F0704780B504F085FA02BD97
:10C4C000DFF83C170868C0F34010002818D108684E
:10C4D000C0F3C010002809D0DFF850090168882097
:10C4E00041434FF4167091FBF0F00CE0DFF83C098B
:10C4F0000168942041434FF4167091FBF0F002E084
:10C50000DFF828090068704710B50100DFF8F00671
:10C510000068C0F3401000280CD0DFF89C0B0468C2
:10C52000C9B2012003F0B0FA844201DB002009E027
:10C53000012007E0DFF8800B0068142801DB0020F1
:10C5400000E0012010BDDFF8B8060068C0F300204D
:10C55000002803D1DFF8D808006803E0DFF8D0082E
:10C5600000684042DFF8C416096801290CD1DFF8E1
:10C57000C4080068002803D4DFF8400B006803E01B
:10C58000DFF8380B006840427047DFF8E8040068C5
:10C59000002801D0012000E00020704780B5DFF8BE
:10C5A0009808006806F0E0F9DFF854160968C1F34E
:10C5B0004011002907D14043DFF8041B09684900F6
:10C5C00090FBF1F009E040430A214843DFF8F01AFC
:10C5D0000A6806214A4390FBF2F002BD70B50220C2
:10C5E000DFF858180860DFF818462068C00740F1E7
:10C5F000E880DFF84C0806680568DFF84818096825
:10C60000890709D4DFF840180968890704D4DFF8DE
:10C610003C180968C9051BD4DFF83448216831F09B
:10C620000201216000E00168DFF820180968C905EF
:10C63000F9D5DFF81C580121280006F0F7FA01218E
:10C64000280006F0F9FA206850F002002060BCE0F3
:10C65000DFF834040068012851D1DFF8A815087804
:10C66000002814D1DFF8EC170A680F2000FB0266DF
:10C67000102096FBF0F00860DFF8DC170A680F2046
:10C6800000FB0255102095FBF0F0086026E00878CA
:10C69000042823D103F038FDDFF8C0170968401AD9
:10C6A000B0F57A7F1AD3DFF88407006806F05CF9EA
:10C6B000002813D1DFF89C170A680F2000FB0266E0
:10C6C000102096FBF0F00860DFF88C170A680F2046
:10C6D00000FB0255102095FBF0F008600020DFF809
:10C6E000801708600020DFF8DC1908600020DFF800
:10C6F000D81908600020DFF86C1708602FE0DFF819
:10C70000602711680F2000FB0166102096FBF0F1F6
:10C710001160DFF840070068091ADFF8DC040068E0
:10C720004143642091FBF0F0DFF89C190860DFF8CA
:10C73000942911680F2000FB0155102095FBF0F1A2
:10C740001160DFF814070068091ADFF8B004006808
:10C750004143642091FBF0F0DFF808170860DFF830
:10C76000D0060068002812D42068C0F300200028FA
:10C7700006D1DFF854090068DFF8E41A086018E011
:10C78000DFF8E0060068DFF8D81A086011E02068DA
:10C79000C0F30020002806D1DFF8C8060068DFF8E3
:10C7A000C01A086005E0DFF820090068DFF8B01A59
:10C7B0000860DFF8AC0A0168002906D50021016095
:10C7C00003E00020DFF8981A086070BDDFF8FC086D
:10C7D000002101605FF48021DFF8F4281160FF225E
:10C7E000DFF8F0381A6001600F20A64908700120B8
:10C7F000DFF8701A0860704710B50420DFF80814DD
:10C80000087003F0BFF80400DFF82C06006806F09B
:10C81000ABF8844204DA03F077FCDFF8BC18086058
:10C8200040F29114DFF8A0080168A14204DBDFF8B0
:10C8300034160968002907D4DFF828160968A142D0
:10C8400007DB0068002804D503F05EFCDFF88818D9
:10C85000086003F059FCDFF880180968401AA0420C
:10C8600009D3022002F02AF90A208649087005201F
:10C87000DFF8A813087082480078002801D001F082
:10C88000BBF910BD38B55020DFF890150860DFF80F
:10C890007843002020707C4D01202860022002F0A7
:10C8A0000DF97748007800280BD00C2075490870E6
:10C8B00003F02AFCDFF82018086004202070002014
:10C8C000286031BD10B50420DFF83C13087001204A
:10C8D00002F0F4F803F056F80400DFF85C05006895
:10C8E00006F042F8844204DA03F00EFCDFF8E817A1
:10C8F000086003F009FCDFF8E0170968401A40F20D
:10C90000E931884201D301F077F910BD80B5552097
:10C91000DFF8081508600420BB49087058490878FA
:10C92000032802D00020584A10600878002802D15D
:10C9300001F04EF91CE00878012802D101F0EEF96F
:10C9400016E00878042802D101F06BF910E00878AD
:10C95000022802D101F09CF90AE00878052802D1EA
:10C9600001F008FB04E00878062801D101F090F9F5
:10C9700001BD80B55620DFF8A41408600020A2494C
:10C980000870DFF8D00B0078042801D001F034F9EA
:10C9900001BD38B504209C490870DFF8CC482068F8
:10C9A000012809DB4FF4805007F083FA002803D1F7
:10C9B0002068401F206034E05120DFF860140860D8
:10C9C000DFF84C44206800282BD1904D28680128BE
:10C9D0001ED18B490868C0F34010002804D1DFF84D
:10C9E000D80600680B280DDA0868C0F3401000284C
:10C9F0000ED01421012003F047F8DFF8BC160968B7
:10CA0000884205DA5FF4802004F0EFFD0020286002
:10CA10000020DFF8A4160860002008F0C5F8012007
:10CA20002060DFF8301B0878012802D101F076F988
:10CA30001CE00878002802D101F0CAF816E0087856
:10CA4000032802D101F0D8F810E00878042802D1B8
:10CA500001F0E7F80AE00878062802D101F0B0FA00
:10CA600004E00878052801D101F084FA31BD000006
:10CA7000007000401070004000400640204006401A
:10CA8000E62D0020E72D00202C2C0020F8B50420F6
:10CA90005D490870DFF8D0070168012903DB0168F0
:10CAA000491F016082E05320DFF870130860574C83
:10CAB000206800287AD103F087FFDFF854532868F4
:10CAC000012826D14E4E3068C0F34010002807D10F
:10CAD000DFF8E405076803F077FF3238874211DB9F
:10CAE0003068C0F3401000285ED0DFF8CC0506683F
:10CAF00003F06AFF07003221002002F0C5FF3F1A51
:10CB0000BE4251DA5FF4802004F06FFD00202860FF
:10CB10004AE0DFF8A45503F057FF28603849086859
:10CB2000C0F3002000281DD10868C0F34010002881
:10CB300016D10868C0F3C010002808D029684FF447
:10CB4000FA6041438731882091FBF0F02AE02968A0
:10CB50004FF4FA6041439331942091FBF0F021E0CF
:10CB600028681FE00868C0F34010002818D1086842
:10CB7000C0F3C010002809D0296849424FF4FA6078
:10CB800041438739882091FBF0F00BE02968494246
:10CB90004FF4FA6041439339942091FBF0F001E0A7
:10CBA0002868404208F000F801202060DFF8A4194E
:10CBB0000878002802D101F00BF81CE0087803285F
:10CBC00002D101F019F816E00878042802D101F02A
:10CBD00028F810E00878022802D101F059F80AE09C
:10CBE0000878062802D101F053F804E008780528F7
:10CBF00001D101F0BFF9F1BDDC2C0020E02C0020B8
:10CC0000202C0020EC2D0020EB2D0020382C0020C3
:10CC100000700340642C0020302C0020ED2D0020FB
:10CC2000400004028C2C0020EE2D0020342C00202B
:10CC300070B55420794908600220DFF81C1908708B
:10CC4000012003F043F8DFF814190860DFF8040945
:10CC50000178022903D00178062940F0D4800078B9
:10CC6000022813D1DFF8F8080068C0F3401000284C
:10CC70000CD1DFF8F00800686430DFF83C14096874
:10CC8000884203DA5FF0007004F0AFFC604800688F
:10CC9000002847D1012002F0A9FFDFF82014086026
:10CCA00002F0CAFF040003F02FFADFF8BC1809688D
:10CCB000401A844202D200F0C0FFA7E002F062FEF8
:10CCC0000500DFF89C683068C0F34010002805D1EB
:10CCD0005948006805F048FE85420ADA3068C0F31A
:10CCE0004010002818D05148006805F03DFE8542EC
:10CCF00012DB03F009FADFF8AC190968401AA04208
:10CD000078D348480068652803DA402004F06DFCB9
:10CD100070E000F092FF6DE003F0F6F9DFF884199F
:10CD2000086067E0012002F003FFDFF8901308605D
:10CD3000DFF830050068012802D1402004F055FCDE
:10CD4000DFF864090168012002F09EFE0400FFF78D
:10CD500025FC0419DFF860030068844202DB01F05F
:10CD6000DDF847E0DFF844090078012810D1DFF84A
:10CD70004009006810F1640F0ADADFF8E407006880
:10CD8000C0F34010002803D1012001F07AF831E00F
:10CD900002F07CFF040003F0B7F9DFF8CC17096854
:10CDA000401A844207D2DFF80C090068002802D13B
:10CDB00001201B49086002F0E5FD1F490968C142D6
:10CDC00013DB03F0A1F9DFF8DC180968401A84428C
:10CDD00010D214480068652803DA402004F005FCEE
:10CDE00008E001200E49086004E003F08DF9DFF847
:10CDF000B4180860DFF8C00804F010FC002805D063
:10CE000001F0CAF802E0012001F03BF870BD00001B
:10CE10003C2C002030400200EF2D00201C2C002074
:10CE2000282C0020CC2C0020502C0020582C002036
:10CE3000682C0020982C0020A02C00200C8003409F
:10CE40006880034010800340188003406C800340DA
:10CE500000800340D02C0020D42C0020002D002086
:10CE6000082D0020C42C002070B55220DFF8FC13E0
:10CE700008600220DFF8E0160870002002F026FFAC
:10CE8000DFF8D8160860DFF8CC060078012840F0FB
:10CE90000F81DFF8CC462068C0F3401000280BD18A
:10CEA00085480068DFF8BC1609686439884203DAEF
:10CEB0005FF0007004F099FBDFF8000800680028BC
:10CEC00048D1002002F092FE7C49086002F0B4FED6
:10CED000050003F019F9DFF890160968401AA84216
:10CEE00002D300F0BBFEE6E002F04CFD0600206835
:10CEF000C0F34010002806D1DFF8C407006805F031
:10CF000033FD86420BDA2068C0F3401000281BD0A6
:10CF1000DFF8B007006805F027FD864214DB03F058
:10CF2000F3F8DFF880170968401AA842C0F0B7800C
:10CF3000DFF894070068652803DA402004F055FB09
:10CF4000ADE000F08BFEB6E003F0DEF8DFF854173A
:10CF50000860A4E0002002F0EBFD58490860C148D9
:10CF60000068012802D1402004F03FFBDFF83807B9
:10CF70000168DFF8580700684118002002F084FDBE
:10CF800005004D480668FFF709FBDFF844170968FC
:10CF90004D1B2D1AAE4202DB00F0D6FF7FE0206869
:10CFA000C0F3401000280DD1DFF8000700780128F9
:10CFB00008D1DFF8FC060068652803DB012000F0DB
:10CFC00085FF6CE02068C0F3401000280DD0DFF82A
:10CFD000DC060078012808D1DFF8D4060068AB2809
:10CFE00003DB002000F072FF59E02068C0F340101E
:10CFF00000280CD1DFF8B4060078022807D1DFF84A
:10D00000B0060068642802DA00F0F4FE47E0206809
:10D01000C0F3401000280CD0DFF8900600780228FA
:10D0200007D1DFF88C060068AA2802DA00F0E2FED9
:10D0300035E002F02BFE040003F066F8DFF8281557
:10D040000968401A844208D2DFF8680600680028A0
:10D0500003D10120DFF87C16086002F093FCDFF8B2
:10D0600060160968884215DB03F04EF8DFF83416C5
:10D070000968401A844212D2DFF84C06006865281D
:10D0800003DA402004F0B1FA09E00120DFF8441689
:10D09000086004E003F038F8DFF808160860DFF8ED
:10D0A000180604F0BBFA002805D000F075FF02E076
:10D0B000012000F00BFF70BDAC2C0020D82C00200C
:10D0C000702C00200C2D0020C02C00200890034064
:10D0D0000C90034034900340F02C002070B5542095
:10D0E00062490860DFF86C040178022903D00078F7
:10D0F000062840F0B0800A21012002F0C5FC5C4CFB
:10D100002168884258DB012002F070FDDFF85C14D2
:10D110000860DFF8C415086800280BD101200860FA
:10D1200002F0F2FFDFF87C15086002F0EDFFDFF897
:10D13000381408602068002802D500F07EFD8DE0DC
:10D1400002F07AFD040002F0DFFFDFF81C1409682A
:10D15000401AA04202D300F070FD7FE002F012FC02
:10D160000500DFF8FC633068C0F34010002806D1EA
:10D17000DFF84C05006805F0F7FB85420BDA3068F4
:10D18000C0F34010002811D0DFF83805006805F022
:10D19000EBFB85420ADB02F0B7FFDFF808150968F0
:10D1A000401AA04247D300F048FD44E002F0ACFF33
:10D1B000DFF8F01408603EE00020DFF81C1508607E
:10D1C000012002F0B5FCDFF8A413086002F09CFF18
:10D1D000DFF8204A2268DFF890130968401A82427B
:10D1E00003D20120DFF8EC14086002F0CBFB05004D
:10D1F000DFF8CC04006805F0B7FB854216DB02F0CF
:10D2000083FF2268DFF89C140968401A824212D218
:10D21000DFF8B4040068652803DA402004F0E5F97B
:10D2200009E00120DFF8AC14086004E002F06CFFB4
:10D23000DFF8701408600B480068012802D1402014
:10D2400004F0D3F9DFF8700404F0E8F9002805D001
:10D2500000F0A2FE02E0012000F013FE70BD00000D
:10D26000C82C0020242C0020E42C00201C2C0020A2
:10D27000AC2C00202DE9F0415220DFF80C1A086098
:10D28000B4480078012840F0CA80DFF8006A3468AA
:10D29000DFF83C54DFF83474D5F80080396800209A
:10D2A00002F0F2FBB8EB0008444508DB5FF48010A5
:10D2B00007F01BFE002802D100F0D0FCB2E0396874
:10D2C0003231A74C2068C0F34010002806D13268E4
:10D2D0002B6838681B1A323B9A420CDA2068C0F37C
:10D2E0004010002855D036682D68002002F0CCFB95
:10D2F0002D1AAE424DDB002002F078FC9B490860FD
:10D30000DFF8141A086800280AD10120086002F02A
:10D31000FBFEDFF89013086002F0F6FE9249086009
:10D3200002F08AFC050002F0EFFE8F490968401AFE
:10D33000A84202D300F092FC74E002F023FB060046
:10D340002068C0F34010002806D1DFF8740300689D
:10D3500005F00AFB86420BDA2068C0F34010002873
:10D3600011D0DFF86003006805F0FEFA86420ADBA0
:10D3700002F0CAFEDFF82C130968401AA8423FD316
:10D3800000F06CFC3CE002F0BFFEDFF81813086010
:10D3900036E0002002F0CCFB744908600020DFF882
:10D3A0007819086002F0B0FEDFF8484822686E493C
:10D3B0000968401A824202D20120C649086002F080
:10D3C000E1FA0500BE48006805F0CEFA854213DB9D
:10D3D00002F09AFE2268B3490968401A82420FD2CD
:10D3E000B9480068652803DA402004F0FEF807E039
:10D3F0000120B849086003E002F086FEA9490860F0
:10D40000B6480068012802D1402004F0EEF8AA488E
:10D4100004F004F9002805D000F0BEFD02E0012070
:10D4200000F054FDBDE8F08170B55420DFF85818C5
:10D4300008604B480068C0F34010002801D11E2549
:10D4400000E0642502F09EFA04009D4E306805F06D
:10D450008BFAA0420EDADFF898090168491D0160D5
:10D460000068652803D23B480078012812D100F0FB
:10D47000C3FB0FE0306805F077FAA84206DA3548BA
:10D480000078012802D100F0B7FB03E00020DFF8AC
:10D490006019086091480068012802D1402004F01A
:10D4A000A4F8854804F0BAF8002801D000F074FD13
:10D4B00070BD80B55220DFF8D017086002F062FA24
:10D4C0007F49096881420ADADFF824090168491DA9
:10D4D00001600068652806D300F08EFB03E00020A1
:10D4E000DFF80C1908607D480068012802D140204F
:10D4F00004F07BF8DFF8000C04F090F8002801D06D
:10D5000000F04AFD01BD80B5DFF8BC0901680129C2
:10D510000CDB5721DFF87027116001680A390160C0
:10D520000168002914D50021016011E0016800297B
:10D530000CD55721DFF85027116001680A310160CE
:10D540000168012904DB0021016001E000F040FBDB
:10D5500001BD0000E62D0020EB2D0020442C002012
:10D56000202C0020B02C0020E82C0020D82C0020FB
:10D5700038B55120DFF810170860DFF8C8090078C7
:10D58000062840F08C80DFF8E8492068C0F340109E
:10D59000002804D1DFF8F4060068102809DB2068B1
:10D5A000C0F3401000281BD0DFF8E0060068032815
:10D5B00016DADFF8DC4901F083FF2060DFF8D409D8
:10D5C00021680268914202DB2168016002E0016883
:10D5D0001439016002F098FDDFF8DC19086046E0BC
:10D5E00002F092FDDFF8D0592968401ADFF8CC1913
:10D5F000884205D301F064FFDFF89419086028E041
:10D6000002F082FD2968401A4EF66121884210D34B
:10D610002068C0F3C010002805D040F2DC50DFF8CD
:10D620007019086015E040F6C410DFF8641908604E
:10D630000FE02068C0F3C010002805D040F6C410E9
:10D64000DFF84C19086004E04FF47A60DFF8401905
:10D650000860DFF84019DFF838090A6803689A4261
:10D6600002DB0068086002E00868143008601648B1
:10D67000006865280DDA02F047FDDFF8801A0968B6
:10D68000401A40F2E93188420BD3402003F0ADFF4D
:10D6900007E002F039FDDFF8641A086001E000F0ED
:10D6A000ABFA31BDF82C00207C2C0020EE2D0020A0
:10D6B000942C0020402C002040000402382C002034
:10D6C000A02C0020582C0020CC2C0020802C0020E6
:10D6D000B82C0020282C00204C2C0020242C0020CA
:10D6E00070B5DFF8A40564210160DFF8B049216856
:10D6F000491D2160DFF84C180978052916D0DFF89C
:10D70000A0090168012903DB012000F0DFFB08E02C
:10D710000068002803D5012000F0B3FB01E000F011
:10D720006BFA0020DFF87C1908703FE2DFF87459CB
:10D73000297800290ED001293ED0022900F0BE80B0
:10D74000032900F0E280052900F00D82072900F08E
:10D75000858128E201202870DFF8A4090168491CAE
:10D76000016003F049F9002806D1DFF804080168D8
:10D7700031F48071016005E0DFF8F407016851F4CD
:10D780008071016002F02CF90020DFF87819087030
:10D790000020DFF8F8140860002007F005FA0120E7
:10D7A00001F02EFE0120DFF86019086002F0ACFCE9
:10D7B000DFF848190860F9E165210160DFF8446984
:10D7C00002203070012002F011FADFF8C81708605B
:10D7D000012002F07BFADFF8301908600020206099
:10D7E00002F02AFA040002F08FFCDFF82019096821
:10D7F000401A844206D20420307001F0BFFE02209D
:10D80000287052E0DFF868572868C0F340100028FD
:10D8100004D1DFF878040068652809DA2868C0F3C5
:10D820004010002808D0DFF864040068652803DB96
:10D830005FF0007003F0D9FEDFF8D408006801281B
:10D8400002D1402003F0D1FE02F09CF806002868C7
:10D85000C0F34010002806D1DFF8B808006805F0D2
:10D8600083F886420BDA2868C0F34010002817D0EE
:10D87000DFF8A408006805F077F8864210DB02F0B4
:10D8800043FCDFF878180968401AA0420DD3DFF88E
:10D890008C080068652808DA402003F0A6FE04E042
:10D8A00002F032FCDFF854180860DFF84C0803F08F
:10D8B000B5FE002801D000F06FFB77E1206840F250
:10D8C000D17188421CDB0020DFF83818087020680E
:10D8D00040F6B931884217DB03202870002007F09A
:10D8E00063F901F04BFE002001F08AFD0120DFF812
:10D8F0001818086002F008FCDFF80018086003E060
:10D900000420DFF80018087050E166210160022051
:10D91000DFF8F0170870002002F068F9DFF87416DD
:10D92000086000202060002002F0D0F9DFF8D8174E
:10D93000086002F081F9040002F0E6FBDFF8CC1782
:10D940000968401A84422DD2DFF824060068C0F32B
:10D95000401000280DD0CD48016840F6AD529142EC
:10D9600003DB402003F041FE19E0006803F03AF8C1
:10D9700015E0C6480168B1F5967F04DA5FF48020AF
:10D9800003F033FE0BE0016840F6A172914203DB25
:10D99000402003F02AFE02E0006803F023F807208D
:10D9A000287052E0DFF8C8552868C0F340100028FE
:10D9B00004D1B648006810F1640F09DB2868C0F391
:10D9C0004010002808D0B148006810F1640F03DA55
:10D9D0005FF0007003F009FEDFF8340700680128EB
:10D9E00002D1402003F001FE01F0CCFF06002868C0
:10D9F000C0F34010002806D1DFF81807006804F0D3
:10DA0000B3FF86420BDA2868C0F34010002817D015
:10DA1000DFF80407006804F0A7FF864210DB02F07D
:10DA200073FBDFF8D8160968401AA0420DD3DFF85F
:10DA3000EC060068652808DA402003F0D6FD04E013
:10DA400002F062FBDFF8B4160860DFF8AC0603F002
:10DA5000E5FD002801D000F09FFAA7E0DFF8686438
:10DA60004FF49670306001F08DFFDFF8A81609685A
:10DA7000884202DA002020606CE0206840F2D17118
:10DA800088424EDBDFF898060168306841434FF466
:10DA9000FA60B1FBF0F1DFF884261068012806DB9C
:10DAA0004FF47A704143106891FBF0F000E00020E1
:10DAB000DFF8702610601068002803D1402003F0C2
:10DAC00094FD25E0DFF8A8140868C0F3C010002812
:10DAD0000CD01068B0F5FA6F08DADFF82406006899
:10DAE000032803D2402003F080FD11E00868C0F352
:10DAF000C01000280CD1106840F69901884207DB5D
:10DB0000DFF8FC050068032802D2402003F06DFD19
:10DB10000520287001F032FD0420DFF8E8150870B8
:10DB200018E0DFF8FC050168306841434FF4FA6003
:10DB3000B1FBF0F1DFF8DC291068012806DB4FF4B7
:10DB40007A704143106891FBF0F000E00020DFF8AC
:10DB5000D4150860DFF8A00503F060FD002801D0AF
:10DB600000F01AFA22E0206840F2D171884215DBF9
:10DB70000020DFF890150870206840F6B93188421F
:10DB800010DB0120DFF8901908600120DFF8F4199C
:10DB900008600E20DFF8F019087003E00420DFF8B9
:10DBA0006415087002E0042003F00FFD70BD80B51D
:10DBB0005FF0FF30344908600420DFF84815087032
:10DBC000DFF880030078052801D000F015F801BDCA
:10DBD00080B501F0D3FC0B20DFF8AC19087002F01F
:10DBE00093FADFF8A81908600420DFF81815087008
:10DBF00001BD0000882C002080B50420DFF804154A
:10DC000008700820DFF8801908700120DFF88019FB
:10DC1000086002F079FADFF8201C086001F0AEFC21
:10DC200001BD80B50020DFF8DC1408700920DFF8A2
:10DC30005819087001F0A2FC01BD80B50420DFF87E
:10DC4000C41408700020DFF84019087001F096FC39
:10DC50004FF4C870DFF8E41B086001BD80B50420F4
:10DC6000DFF8A01408700320DFF81C19087001F019
:10DC700085FC0020DFF8281408604FF4C870DFF836
:10DC8000BC1B086001BD00001C2C0020AC2C002037
:10DC900080B501F073FC0120DFF86C1408600120EE
:10DCA00001F01CFADFF870080068002803D1012099
:10DCB00001F0A6FB1CE0DFF8DC080078012811D198
:10DCC000AB480068C0F34010002805D07FF0A900E1
:10DCD000DFF8CC1308600BE07FF06300DFF8C013BF
:10DCE000086005E0DFF8B0080068DFF8B4130860EA
:10DCF0000220DFF8101408700420DFF88C18087078
:10DD0000DFF898080068DFF89818086002F0FCF95E
:10DD1000DFF8E813086001BD482C002038B501F099
:10DD20002DFC0120DFF8E0130860002001F0D6F997
:10DD3000DFF870482068642804D0DFF848080068DD
:10DD4000002807D102F040FEDFF85C18086064206C
:10DD5000206009E002F038FE21684843642190FB0E
:10DD6000F1F0DFF844180860DFF818582868002838
:10DD700003D1002001F044FB17E0DFF81808007819
:10DD800001280DD17A480068C0F34010002803D064
:10DD9000A920C349086008E06320C149086004E085
:10DDA000DFF8F4070068BE490860206864280DD0D9
:10DDB000DFF8E8070068DFF8F0170968884205DB3C
:10DDC0002868012802D1FFF749FF06E00220CD496B
:10DDD00008700120DFF8B0170870DFF8C00700688E
:10DDE000DFF8BC17086002F08FF9C449086031BD44
:10DDF000EC2C002010B50120C3490860162006F065
:10DE000091F80B2801DB0A2002E0012800DA01204A
:10DE100057490968C1F34011002903D164214FF427
:10DE2000167202E0AA2140F2EE22DFF86C37521A95
:10DE3000092492FBF4F2401E00FB021018601868DF
:10DE400097490860DFF85C07006864280ED0DFF8A7
:10DE50004C070068DFF850170968884206DBDFF8D6
:10DE600024070068012801D1FFF7F8FEDFF82C072E
:10DE70000068DFF82C17086002F046F99F49086037
:10DE800010BD38B5C0B2012804D101F0BFFCDFF8E5
:10DE9000B0190860DFF804070568DFF8A849FEF745
:10DEA0007DFB2D1A256020680A2801DA0A202060EF
:10DEB0000720DFF8D416087002209249087000206D
:10DEC000DFF8EC1B086031BD682C002038B5C0B20B
:10DED000012804D101F09AFCDFF864190860DFF82A
:10DEE000BC060568DFF85C49FEF758FB451925605C
:10DEF000DFF8B40601680A392268914202DA006844
:10DF00000A3820600620DFF88016087002207D495C
:10DF100008700020DFF8981B086031BD80B505202F
:10DF2000DFF864160870DFF874060068DFF8701612
:10DF3000086002F0E9F8714908600020DFF81C1C55
:10DF4000086001BDE62D002080B50220DFF83816FC
:10DF50000870DFF848060068DFF84416086002F031
:10DF6000D3F8664908600020DFF8F41B086001BDA3
:10DF7000202C002080B50420624908700D20DFF8B5
:10DF80000816087000204749087001F0F7FA01BD33
:10DF9000102D0020D82C002080B55A480178022985
:10DFA00002D0FFF715FE05E0022101700F20DFF817
:10DFB000D815087001BD0000FC2C0020A1860100CE
:10DFC00080B502204F49087001F0D8FA01F078FAC4
:10DFD000DFF8E01A0860DFF8E00A0068C0F34010DC
:10DFE000002804D17FF063002D49086003E0DFF8CA
:10DFF000740B2B49086002F087F8DFF86C1B08608F
:10E0000002F082F83D4908601020DFF87C150870A6
:10E0100001BD10B5DFF8544B2078012801D100F084
:10E0200025FF38490878227890422FD0DFF8880AF7
:10E03000026852F0020202600878042802D100F05F
:10E04000DFFE29E00878002802D100F06FFE23E00F
:10E05000087803280BD12078042802D020780028E3
:10E0600002D100F0ABFE17E000F000FF14E00878EA
:10E07000022811D12078042802D02078002802D16B
:10E0800000F09CFE08E000F077FE05E0DFF8280ACB
:10E09000016831F00201016010BD0000F42C002085
:10E0A000942C0020E82D002080B5DFF80C0A0068D1
:10E0B000C0F34000002814D0DFF8B00A007804282C
:10E0C00007D1002300220121DFF8A40C04F043FD56
:10E0D00011E0032306220121DFF8940C04F03BFD3C
:10E0E00009E0DFF8880A0078042804D10121DFF86C
:10E0F000800C04F0BAFD01BD40000402F82C0020A1
:10E10000042D0020EB2D0020442C0020E82C0020C2
:10E11000242C0020A02C0020582C0020CC2C0020E7
:10E12000642C0020602C002038B5DFF85C040178F6
:10E1300005293AD101F00AFADFF8B40A0168012092
:10E1400001F0A2FCDFF854140A68904219DA096859
:10E15000081ADFF8EC16096800FB01F0400007F030
:10E16000B9FC5FF0FF314843DFF8881A0A68824241
:10E1700000DA0868DFF820140A68904204DA0868B8
:10E1800002E0DFF8700A0068DFF82C190968C1F3B3
:10E190004011002905D101F035FADFF8D81B0860DD
:10E1A000B6E1DFF8D01B0860B2E1017802293BD16B
:10E1B00001F0CCF9DFF8700B0168DFF8340A006871
:10E1C0004118002001F060FCDFF8DC23DFF8CC13FD
:10E1D0000B681468241AA34212DA1268101A09682C
:10E1E000401ADFF85C16096800FB01F0400007F0F8
:10E1F00071FCDFF8A4130A68824204DA086802E0BE
:10E20000DFF8F0090068DFF8B0180968C1F34011C1
:10E21000002905D101F0F6F9DFF8581B086077E115
:10E22000DFF8501B086073E10178072928D101F05D
:10E230008DF9DFF868030168DFF808060068081A3E
:10E2400001280BDBDFF8F815096800FB01F040003E
:10E2500007F040FC5FF0FF31484300E00020DFF8AA
:10E2600058180968C1F34011002905D101F0CAF915
:10E27000DFF8001B08604BE1DFF8F81A086047E19F
:10E280000178062924D101F061F9DFF8B8050168A9
:10E29000C2480068081A012808DBDFF8A4150968DD
:10E2A00000FB01F0400007F015FC00E00020DFF863
:10E2B00008180968C1F34011002905D101F0A2F93D
:10E2C000DFF8B01A086023E1DFF8A81A08601FE140
:10E2D0000178012910D001780D2904D1DFF8DC1B69
:10E2E0000978032908D001780D2940F07F80DFF8F4
:10E2F000CC1B0978072979D1DFF8C40B0068012805
:10E3000010D1DFF8B4070068C0F34010002804D033
:10E31000AA20DFF8B01B08600AE06420DFF8A41B25
:10E32000086005E0DFF8A00B0068DFF8981B0860C4
:10E33000DFF884070068C0F34010002805D1DFF83B
:10E34000844B206801F05EF92060002001F08CF918
:10E35000DFF8703BDFF81C2A11681C68A1421CDA48
:10E36000DFF8A84B2568052101FB005020602068DC
:10E370004FF47A7190FBF1F01060106819688842D0
:10E3800006DB1868106019684FF47A704143216009
:10E390000120DFF8C01C0860BAE019681468A142C7
:10E3A00018DADFF8683B1C68052101FB1040186093
:10E3B00018684FF47A7190FBF1F010601068012832
:10E3C00003DA00201060002018600020DFF8841CB1
:10E3D00008609DE019684FF47A704143DFF82C0B18
:10E3E00001600020DFF86C1C086091E001780429CE
:10E3F0000AD001780D2904D1DFF8C01A0978012963
:10E4000002D0017810297BD1DFF8B40A0068012816
:10E4100012D1DFF8A4060068C0F34010002805D030
:10E420007FF0A900DFF89C1A08600BE07FF0630022
:10E43000DFF8901A086005E0DFF88C0A0068DFF862
:10E44000841A0860DFF870060068C0F340100028E6
:10E4500005D1DFF8704A206801F0D4F8206001206F
:10E4600001F002F9DFF85C3ADFF80829196814684E
:10E47000A1421CDADFF8944A2568052101FB1050FF
:10E48000206020684FF47A7190FBF1F010601868FA
:10E490001168884206DB1868106019684FF47A70BA
:10E4A000414321600120DFF8AC1B086030E01168B7
:10E4B0001C68A14218DADFF8543A1C68052101FBF8
:10E4C0000040186018684FF47A7190FBF1F010600A
:10E4D0001068002803D4002010600020186000207D
:10E4E000DFF8701B086013E019684FF47A7041433D
:10E4F000DFF8180A01600020DFF8581B086007E009
:10E5000000780F2802D101F021F801E001F036F87F
:10E5100031BD0000C82C00203C2C002080B51A48DA
:10E5200001780F292DD001780D2904D1DFF88C193D
:10E530000978072925D00178012914D00178042908
:10E5400011D0017805290ED0017802290BD001786D
:10E55000072908D00178062905D00178102902D0B2
:10E5600000780D2809D100F0B1FC012802D100F09B
:10E570006BF906E000F01AF803E00020DFF83C1B1E
:10E58000086001BD382C0020E72D0020F02C002071
:10E590002C2C0020EE2D0020782C0020AC2C00200C
:10E5A000B02C00208C2C0020B82C00202DE9F84342
:10E5B000DFF8C067306840F6E731884203DB40F699
:10E5C000E630306005E0DFF8F80A3168814200DAB1
:10E5D0003060DFF8F04A31684FF4FA60414340F6AA
:10E5E000E63091FBF0F02060DFF8DC7A3168DFF88C
:10E5F000DC0A0068091A3960DFF8D45A2878012843
:10E6000014D02878042811D0287805280ED028782E
:10E6100002280BD02878072808D02878062805D0AB
:10E620002878102802D028780D282FD1DFF88814F8
:10E630000868C0F3C00000280BD10868C0F3800050
:10E64000002806D1DFF88C1A0A68386882180A6038
:10E650001CE00868C0F38000002809D03868002852
:10E6600006D5DFF8701A0A68386882180A600DE06B
:10E670000868C0F3C000002808D03868012805DB0E
:10E68000DFF8501A0A68386882180A602878052866
:10E6900008D02878022805D02878072802D02878C2
:10E6A000062815D1386804F058F98146DFF8248A25
:10E6B000D8F8000004F051F9814509D0D8F80010CD
:10E6C000D8F80000042290FBF2F0091AC8F80010F4
:10E6D000DFF8E81922683B684FF4967043434FF423
:10E6E0007A7093FBF0F08218DFF8E80903680520E0
:10E6F00043434FF47A7093FBF0F082180A6030685D
:10E70000002801D1002008602878022829D1DFF8EC
:10E71000A8231068C0F3401000280BD1DFF8B80917
:10E720000068642806DA2068022390FBF3F00B6887
:10E73000834210DB1068C0F34010002842D0DFF89D
:10E7400098090068AA283DDA2068022290FBF2F0BE
:10E750000A68824236DA2068022290FBF2F00860F2
:10E7600030E0287805282DD1DFF84C231068C0F35D
:10E77000401000280DD1DFF86009006810F1630F28
:10E7800007DB20687FF0010390FBF3F00B689842F1
:10E7900012DB1068C0F34010002813D0DFF83809EE
:10E7A000006810F1A90F0DDB20687FF0010290FBDB
:10E7B000F2F00A68904205DA20687FF0010290FBCF
:10E7C000F2F00860DFF88C080068012812D10868B0
:10E7D000322805DA2878012802D13220086009E0C1
:10E7E000086810F1310F05DB2878042802D17FF08A
:10E7F00031000860B048026832F00402026002682A
:10E8000032F008020260DFF8F02B0B68934205DA61
:10E810000A60016851F0080101600BE00A6840F2EB
:10E820006D739A4206DB40F26C720A60016851F027
:10E8300004010160BDE8F183002D0020E42C0020DC
:10E84000702C0020B42C0020F8B59A4EDFF8244D2F
:10E8500030682168884229DADFF8A00B0068216857
:10E86000884223D020683168411A4FF47A704143BE
:10E87000206891FBF0F1DFF84428106841434FF421
:10E880007A7091FBF0F01168081A1060106840F27D
:10E890006D71884203DB40F26C70106067E0DFF856
:10E8A000580B1168814262DA106060E020683168BC
:10E8B000B1F5C871884209DB20683168884256DAB0
:10E8C000DFF8380B00682168884250D1DFF8FC0778
:10E8D000006804F049F80700DFF89854286804F04D
:10E8E00043F8092148430A2190FBF1F0874208DAF6
:10E8F0003168072041430A2091FBF0F021688142F2
:10E9000004DA0020DFF8B41B08601FE030682168DB
:10E91000411A4FF47A704143206891FBF0F1DFF81F
:10E920009C67306841434FF47A7091FBF0F004F03B
:10E930001BF80A2800DA0A202968002903D4316864
:10E940004018306002E03168081A3060DFF86C0768
:10E95000016840F26D72914203DB40F26C7101601C
:10E9600005E0DFF8941A02688A4200DA0160206844
:10E97000DFF8881A0860DFF8440B0068002824D10B
:10E9800001F0C2FBDFF8A81C0860DFF8E82311687B
:10E990004FF4FA60414340F6E63091FBF0F1106825
:10E9A000DFF828271268821ADFF810070068411A7A
:10E9B0004FF47A7041434FF4967000FB121105201A
:10E9C00091FBF0F0DFF80C170860F1BD70B56748F7
:10E9D000007802286AD1384C2068C0F30020002853
:10E9E00008D1DFF8D806006810F5FA60DFF8881B58
:10E9F000086007E0DFF8C4060068D0F5FA60DFF8C9
:10EA0000781B0860DFF8F85BDFF86C6B3268402138
:10EA1000280007F09CF832688221280007F097F858
:10EA2000DFF89806006800281ED42068C0F3002094
:10EA300000280CD14FF480724021280007F0D3F851
:10EA40004FF400724021280007F0C7F82AE04FF485
:10EA500000724021280007F0C6F84FF48072402170
:10EA6000280007F0BAF81DE02068C0F30020002855
:10EA70000CD14FF400724021280007F0B4F84FF495
:10EA800080724021280007F0A8F80BE04FF4807254
:10EA90004021280007F0A7F84FF400724021280019
:10EAA00007F09BF8032128000160C04670BD0000FC
:10EAB000EC2C0020D82C0020202C002010B50128A0
:10EAC00033D1052002F016FF47F23051884215D2AB
:10EAD0004FF47F41DFF85C0B02F040F90221DFF8D0
:10EAE000580B01F057FA0220DFF8501B0860DFF8DE
:10EAF000EC0C016831F0100101602DE0DFF8DC4C16
:10EB00002068C0F30010002826D100F0A5FA0221E9
:10EB1000DFF8240B01F078FADFF8240B01F08CFA0F
:10EB2000206850F01000206016E0022814D14FF445
:10EB30007F41DFF8000B02F011F90221DFF8F80A3B
:10EB400001F028FA0020DFF8F41A0860DFF88C0CD6
:10EB5000016831F01001016010BD00004C2C002054
:10EB6000482C002070FEFFFFFC2C0020EC2D002024
:10EB700080B5DFF85C0501780F290ED1DFF83C0580
:10EB80000068002804D00420DFF8D41C08602EE0C0
:10EB90000020DFF8CC1C086029E00178052908D0A6
:10EBA0000178022905D00178072902D000780628CB
:10EBB00019D1DFF8900A01684AF21142914206D356
:10EBC00004220421DFF8700A01F0B8F90FE00068B0
:10EBD0004AF2280188420AD200220421DFF8580AAA
:10EBE00001F0ACF903E00020DFF8741C086001BDFF
:10EBF0007C2C0020742C002038B5DFF84C0A07F07C
:10EC00001BF8DFF8480A01F017FADFF8440A01F0B0
:10EC100013FADFF8400A01F00FFADFF83C0A01F0BE
:10EC20000BFADFF8384A0121200001F0D5F9022162
:10EC3000200001F0D1F9DFF8284A1021200001F06E
:10EC4000CBF92021200001F0C7F9DFF8B449DFF843
:10EC5000145A2A004021200006F056FF2A00802185
:10EC6000200006F051FFE020DFF8741B0860B020A0
:10EC7000DFF8701B0860AA20DFF86C1B08604FF4F7
:10EC80007A624021200006F055FF4FF47A6280211D
:10EC9000200006F04FFF4021200006F055FF8021A4
:10ECA000200006F051FF0321200006F06FFF5FF403
:10ECB0007020DFF8B01B086000220F21200006F052
:10ECC0007AFF01220F21200006F07EFF00220F2193
:10ECD000200006F05EFF00220F21200006F062FFF8
:10ECE0004FF4FA624021200006F031FF4FF4FA623F
:10ECF0008221200006F02BFF0E230E22402120004F
:10ED000006F037FF0E230E228021200006F031FF8F
:10ED1000032120000160C0464FF400724021200012
:10ED200006F05BFF31BD0000802C002010B5DFF83D
:10ED3000D04800220321200006F02BFF00220C21E6
:10ED4000200006F026FFFFF757FF0020DFF8181B12
:10ED50000870DF4800780A2804D10520DFF8741C09
:10ED6000087003E00020DFF86C1C087010BD000084
:10ED700000800340982C002010B5DFF88448002262
:10ED80000321200006F005FF00220C21200006F0E0
:10ED900000FFFFF731FF01220321200006F0F9FEFA
:10EDA00001220C21200006F0F4FE0220DFF8B81A40
:10EDB00008700220DFF81C1C087010BD10B5DFF8C9
:10EDC000404800220321200006F0E3FE00220C212F
:10EDD000200006F0DEFEFFF70FFF012202212000D7
:10EDE00006F0D7FE01220821200006F0D2FE012005
:10EDF000DFF8741A08700120DFF8D81B087010BD06
:10EE000038B5DFF8FC4700220321200006F0C1FEE0
:10EE100000220C21200006F0BCFEDFF84048032150
:10EE2000200001F0B7F8DFF838583021280001F051
:10EE3000B1F800220121200001F080F80222022115
:10EE4000200001F07BF800221021280001F076F864
:10EE500020222021280001F071F80420DFF8081A90
:10EE600008700420DFF86C1B087031BD10B5FFF787
:10EE7000C3FEDFF88C474FF4FA624021200006F011
:10EE800066FE4FF4FA628221200006F060FE032144
:10EE900020000160C04601220321200006F079FE17
:10EEA00001220C21200006F074FE0320DFF8B819BF
:10EEB00008700320DFF81C1B087010BDE82D00202F
:10EEC000442C0020902C0020942C002010B5DFF85A
:10EED000EC452068002815D101F016F9DFF850172D
:10EEE0000860DFF8940B0168012909DB0068DFF88E
:10EEF00084160968884203DA01202060012004E0BA
:10EF0000002002E001202060012010BD9C2C002088
:10EF100010B5DFF8C40A0068002802D1042002F00E
:10EF200054FBDFF8B84A0821200001F00BF8042157
:10EF3000200001F007F8DFF8E84B0121200003F082
:10EF4000EFFD0121200003F0FEFD03230622012135
:10EF5000200003F000FE002300220121200003F026
:10EF600024FE612301220121200003F01EFE012165
:10EF7000200003F0E3FD00211F2007F012F801211B
:10EF8000200003F0D0FD1F2007F01CF80121200015
:10EF900003F06BFE10BD38B5DFF8E00A06F04CFE5A
:10EFA000422007F03BF8DFF8D84A0221200003F0A6
:10EFB000B7FD0221200003F0C6FD0021200003F070
:10EFC0008CFE0720DFF8BC1A08600221200003F045
:10EFD00070FE40F674654FF47A632A000021200029
:10EFE00003F05FFE4FF47A632A000121200003F052
:10EFF00058FE41F61D552A000021200003F04BFE6B
:10F000002A000121200003F046FE2021200003F009
:10F010003AFE03230F220221200003F09CFD5FF43F
:10F02000002300220221200003F0BFFDDFF8FC3B9B
:10F0300001220221200003F0B8FD0221200003F08C
:10F040007DFD422006F0BEFF0221200003F036FEC7
:10F0500031BD0000402C002010B5DFF8C80A06F0D2
:10F06000EBFDDFF8D0454FF47F41200001F076FE44
:10F07000DFF8B41A200001F07AFEDFF8B40B016863
:10F0800031F4007101604FF496524FF47F4120003B
:10F0900001F0B6FE00224FF47F41200001F0A4FEF3
:10F0A0004FF4C8624FF47F41200001F0BAFE4FF4E4
:10F0B0007F41200001F04CFE10BD0000682C0020B4
:10F0C0001AF4FFFF142D0020A82C0020582C00203B
:10F0D000E72D0020A42C0020A02C0020F8B504006F
:10F0E0002000C0B2002803D1042004F01BFF02E07E
:10F0F000082004F017FF012801DA012002E00B28A4
:10F1000000DB0A20DFF8D4562968C1F3401100293A
:10F1100019D12968C1F3C011002909D02100C9B251
:10F12000002902D14FF402720BE04FF4967208E00E
:10F130002100C9B2002902D14FF4167201E04FF448
:10F140001672C8210AE02100C9B2002902D142F298
:10F15000107201E040F6B8324FF44871521A401E66
:10F160004243092092FBF0F04118DFF87C0A01606D
:10F170002000C0B2002803D1062004F0D3FE02E034
:10F180000A2004F0CFFE012801DA012002E00B285A
:10F1900000DB0A202968C1F3401100290BD129683E
:10F1A000C1F3C011002902D04FF4967201E04FF470
:10F1B000C872C82103E04FF4487140F6B832521AC1
:10F1C000401E4243092092FBF0F04118DFF8640A28
:10F1D00001602000C0B2002803D1162004F0A2FE76
:10F1E00002E0182004F09EFE012801DA012002E06E
:10F1F0000B2800DB0A202968C1F3401100290BD13C
:10F200002100C9B2002903D14FF4167264210EE027
:10F210004FF4167264210AE02100C9B2002903D11B
:10F2200040F2EE22AA2102E04FF4C872AA21DFF8D0
:10F23000583A521A092692FBF6F2401E00FB0211C0
:10F2400019602000C0B2012802D11868404218603D
:10F250002000C0B2002804D1102004F063FE401C3E
:10F2600003E0122004F05EFE401C002800D50020C0
:10F270002968C1F34011002900D00A300A267043E2
:10F28000DFF8401A08605C2004F04CFE0B2800DB1D
:10F290000A20DFF8347A70433860162007F001F84E
:10F2A000012801D1002038602000C0B2002803D11D
:10F2B000002004F037FE02E0022004F033FE0428B0
:10F2C00001DB032002E0012800DA01202100C9B29D
:10F2D00000292AD12968C1F34011002912D103283D
:10F2E00004D13220DFF8441A08604EE0022804D12D
:10F2F0002820DFF8381A086047E01E20DFF82C1AB3
:10F30000086042E0032804D1AA20DFF8201A086030
:10F310003BE0022804D19620DFF8101A086034E0A0
:10F320008220DFF8081A08602FE02968C1F3401135
:10F33000002915D1032805D17FF03100DFF8EC1941
:10F34000086022E0022805D17FF02700DFF8DC19F1
:10F3500008601AE07FF01D00DFF8D019086014E0A3
:10F36000032805D17FF0A900DFF8C01908600CE080
:10F37000022805D17FF09500DFF8B019086004E09D
:10F380007FF08100DFF8A41908602000C0B20028D7
:10F3900007D10E2004F0C6FD4FF4FA6141F2883225
:10F3A00006E00C2004F0BEFD4FF4FA6141F2883211
:10F3B0000B2801DB0A2002E0012800DA0120521AA2
:10F3C000401E4243092092FBF0F04118DFF860092B
:10F3D0000160E4B2002C03D11C2004F0A3FD02E084
:10F3E0001A2004F09FFD1F2800DB1E2064214843E3
:10F3F000DFF840190860F1BD94F8FFFF182D0020D8
:10F40000C0B2012812D1DFF8D4030068C0F3401065
:10F41000002805D07FF08100DFF81C1908601FE08C
:10F420007FF04500DFF81019086019E0DFF8AC1331
:10F430000868C0F34010002804D08220DFF8F818D4
:10F4400008600DE00868C0F38010002804D0642034
:10F45000DFF8E418086003E04620DFF8DC180860F5
:10F46000DFF8D8080068DFF8D8180860704780B562
:10F4700000F0A4FADFF8CC18086000F0F7F9DFF824
:10F48000C8180860FDF71CF8DFF8C0180860FCF722
:10F49000F6FFDFF8A818086000F004F8DFF8B018ED
:10F4A000086001BD33480168DFF8A408026809203C
:10F4B00000FB02110A2091FBF0F07047342C002071
:10F4C00010B5042004F0F5FC00280BD05D2004F0FA
:10F4D00029FD0400012C01DA01240CE00B2C0ADBCD
:10F4E0000A2408E04FF4805004F0E3FC002801D027
:10F4F0000A2400E001244FF4007004F0DAFC002834
:10F500001AD1DFF850080068C0F3C010002809D0F5
:10F51000641E4FF416704443092094FBF0F010F57C
:10F52000167012E0641E40F24C404443092094FBE4
:10F53000F0F010F52F7008E0641E4FF4FA704443A9
:10F54000092094FBF0F010F5FA7010BD0020DFF8F0
:10F55000081808600020DFF8E0170860DFF8FC07F3
:10F560000068DFF8FC1708600020DFF8F817086073
:10F5700070470000C82C00201C2D002080B5002002
:10F58000DFF8D41708600020DFF8AC17086000200F
:10F59000DFF8C81708600020DFF8C41708600020F3
:10F5A000DFF8C01708600020DFF8BC17086000F023
:10F5B000ABFD1F4908600020DFF8BC140860002084
:10F5C000DFF8A81708600020DFF8A4170860002003
:10F5D000DFF8A017086000208B4908600020DFF8E2
:10F5E000701708600020DFF89017086000F08CFDAD
:10F5F000DFF8881708600020DFF88417086001BD75
:10F6000000800240DFF84C170968C1F3C0110029DF
:10F6100006D04FF47A714843E32190FBF1F005E006
:10F620004FF47A714843F62190FBF1F070470000E7
:10F63000E82C002000C0044000700040087000402A
:10F6400007040300642C0020004000F001000D00BE
:10F6500001040D00041001000414010000500640D4
:10F6600000500040BAAA050070B50400DFF8780524
:10F6700005685A4E3068C0F3401000286FD14FF42F
:10F680008040002101F0DDFF002901D1002805D0D4
:10F6900040F2E930854201DB4FF47A753068C0F3FF
:10F6A000C01000281AD0DFF894060168972903DA01
:10F6B0002100C9B201290AD0DFF8C81609689639B5
:10F6C0000068814225DA2000C0B2002821D140F232
:10F6D0002D1085421DDB4FF496751AE040F22D1176
:10F6E000DFF8580602688A4203DA2200D2B2012A01
:10F6F0000BD0DFF890261268B2F59672006882424D
:10F7000007DA2000C0B2002803D18D4201DB4FF49C
:10F7100096752000C0B2002804D1DFF86C0600689E
:10F72000002807D0E4B2012C14D1DFF8600600688D
:10F7300000280FD13068C0F3C010002801D0C825C0
:10F7400008E03068C0F38010002801D0642501E093
:10F750004FF496752800FFF755FF05003CE04FF485
:10F760008040002101F06DFF002901D1002805D063
:10F7700040F22D10854201DB4FF4967509212000DF
:10F78000C0B200F081F9DFF8B4150A68904203DBDB
:10F790002200D2B2012A06D00968814209DB20008A
:10F7A000C0B2002805D140F22D10854201DB4FF494
:10F7B00096752000C0B2002804D1DFF8CC0500689F
:10F7C000002807D0E4B2012C06D1DFF8C00500689C
:10F7D000002801D140F26C75280070BD202C00205B
:10F7E00060800240A080024028800240DFF8A0052F
:10F7F0000178042902D00078052802D140F66A2059
:10F8000001E040F66A207047682C002080B5542043
:10F8100004F088FB0100062901DB052102E0012933
:10F8200000DA0121C1480068C0F34010002804D16B
:10F830004FF496704FF4487202E0C8204FF4FA6219
:10F84000121A491E01FB02F1042291FBF2F1081881
:10F85000DFF8E0130A68904200DA086802BD000091
:10F86000107000401C800240EC2D002010B5DFF825
:10F87000244505F073F92060206844F62061884231
:10F8800008D30020DFF8101508600020DFF80C1501
:10F8900008702DE0DFF80805DFF8A81402680B688F
:10F8A0009A4208DA0020DFF8F01408600120DFF83F
:10F8B000EC1408701CE009680068814208DA002036
:10F8C000DFF8D41408600220DFF8D01408700FE0CD
:10F8D000DFF8C4040168491C016041F288312268E4
:10F8E00003684B439A4203D2006801FB00F1216098
:10F8F0002068002805D0DFF8AC042168B0FBF1F0E7
:10F9000001E040F6E630DFF894241178002905D0B4
:10F910001178DFF894341B78994201D0002008E078
:10F920001178012905D01178022901D1404200E067
:10F93000002001280BDBDFF874341968002913D08C
:10F940001968283181420FDA186828300CE0002845
:10F950000AD5DFF858341968002905D01968283904
:10F96000884201DA18682838DFF840140860DFF8A8
:10F97000D4130968DFF8283419601178DFF82824D7
:10F98000117010BDDFF8CC030068C0F340100028F0
:10F9900001D10A2000E03220704764490868C0F3B2
:10F9A0004010002801D0412007E00868C0F3801013
:10F9B000002801D0322000E02320704780B505F0F8
:10F9C000EBF8DFF890130968C1F30021002900D09B
:10F9D000404202BDED2D002000C7FC4300C00540A1
:10F9E00010B500F0EDFF040001F002F8401EDFF852
:10F9F000C0130860092C0ED1DFF85803016831F0FC
:10FA000020010160016831F040010160016851F09E
:10FA1000800101602FE0072C0ED1DFF83803016868
:10FA200051F020010160016831F04001016001687E
:10FA300031F0800101601EE0082C0ED1DFF81403C4
:10FA4000016831F020010160016851F0400101605E
:10FA5000016831F0800101600DE0DFF8F802016813
:10FA600031F020010160016831F04001016001685E
:10FA700031F08001016010BDD82C0020013800F069
:10FA800000900340C49F034010B4020008002749BF
:10FA90000968C1F34011002940D00A2190FBF1F11F
:10FAA000152924DBD2B2002A11D1DFF80423DFF8B4
:10FAB000043314685420444303EB0400036DBE4830
:10FAC000126850F82200163901FB003026E0B84ACF
:10FAD000BA4B14685420444303EB0400036DB6484A
:10FAE000126850F82200163901FB003016E0D2B23D
:10FAF000002A09D1AF4AAE4803685420434302EBC1
:10FB0000030050F8210009E0AC4AA94803685420DA
:10FB1000434302EB030050F82100FFE710BC70479D
:10FB200000800340025C00F0220A0004202C002028
:10FB300038B50400A24805F0D8F900280ED04FF4DB
:10FB40008040002101F07DFD002904D1002802D170
:10FB500041F2707504E07648056801E07448056874
:10FB600081480068002823D15FF4801005F0BDF9BA
:10FB7000002802D041F2707534E02000C0B20028A5
:10FB800009D14FF4007005F0B0F9002803D0FFF759
:10FB90002DFE050026E0E4B2012C23D14FF4807045
:10FBA00005F0A3F900281DD0FFF720FE050019E09D
:10FBB00068480068C0F38010002808D0E4B2002C28
:10FBC00002D14FF4FA550DE041F270750AE04FF49E
:10FBD0008040002101F035FD002903D1002801D12A
:10FBE00041F27075280032BD6C2C0020594909681B
:10FBF000C1F38011002915D05B490968012908D19A
:10FC0000C0B2002802D14FF4FA500DE041F27070FA
:10FC10000AE0C0B2002802D140F6B83004E041F258
:10FC2000883001E040F6B83070470000210009003C
:10FC300004C00440702C00204B48006801280BD100
:10FC400044480068C0F38010002802D041F65830C4
:10FC500018E040F6B83015E03E490868C0F380105F
:10FC6000002802D040F6B83001E040F6B830484AEB
:10FC70001278052A06D10968C1F38011002901D143
:10FC80004FF47A7070470000782C002080B5364819
:10FC9000006801280BD12F480068C0F380100028AD
:10FCA00002D041F658300CE040F6B83009E0444844
:10FCB00005F01BF9002802D040F6B83001E01D48DD
:10FCC000006802BD7C2C0020802C002070B5040050
:10FCD00025480068002801D1002025E02000C0B29E
:10FCE000002805D11548006815490D68451B04E03A
:10FCF0001348006811490D68451BFFF74EFE0600CA
:10FD00001248006802F030FE86420CDA11480068A2
:10FD1000C0F38010002804D0E4B2012C01D0652D7E
:10FD200001DB002000E0012070BD0000742C0020E9
:10FD3000842C0020882C0020942C0020AC2C002047
:10FD4000B02C0020502C0020582C0020A02C00208B
:10FD5000CC2C0020202C0020902C0020982C00205F
:10FD60009C2C0020402C0020442C0020342C00200F
:10FD7000A42C0020A82C0020242C0020F82C0020EB
:10FD8000282C0020B82C0020382C00203C2C0020EF
:10FD9000E72D0020202D0020242D0020E92D00201B
:10FDA000542C0020C0270900EA2D00205C2C0020E4
:10FDB000BC2C0020883C020048420200843D020026
:10FDC000C00050E030B5CB4300F58064D50725680E
:10FDD0004CBF0D431D40256000F58460920747BF6E
:10FDE0000268114301681940016030BD30B5CB4352
:10FDF00000F58164D50725684CBF0D431D40256083
:10FE000000F20444950725684CBF0D431D40256052
:10FE100000F20C44550747BF236819432168194075
:10FE2000216000F5A760D10301684EBF41F00101D8
:10FE300049084900016030BDF0B5002400F6C475E2
:10FE40000126A640314211D066002F684FF0030C06
:10FE50000CFA06FC27EA0C072F60C2F34117D5F80D
:10FE600000C007FA06F646EA0C062E60641C082C51
:10FE7000E6DBCC4300F5A065D6072E684CBF0E43E9
:10FE800026402E6000F2045596072E684CBF0E43A4
:10FE900026402E6000F5A16556072E684CBF0E4324
:10FEA00026402E6000F5A36516072E684CBF0E4352
:10FEB00026402E6000F23C55D2062A684CBF0A4309
:10FEC00022402A60DD0700F20C5215684CBF0D433A
:10FED0002540156000F5A2629D0715684CBF0D43D3
:10FEE0002540156000F214525D0715684CBF0D43A4
:10FEF0002540156000F21C521D0715684CBF0D43CC
:10FF00002540156000F244529D0515684CBF0D4315
:10FF10002540156000F5A86213F4407F156814BFF2
:10FF20000D432540156000F5A560002B07BF026852
:10FF300041EA020401680C400460F0BD00EB81005E
:10FF40000260704738B501E038B50CE004460D4654
:10FF50000022FFF737FF2946204601B0BDE83040B8
:10FF60000023012268E704460D460222FFF72AFF1C
:10FF70002946204601B0BDE83040082366225BE7F1
:10FF800038B500F055F82946204601B0BDE83040AC
:10FF90000823E6E738B504460D460823FFE70122AB
:10FFA000FFF74AFF29462046BDE83840012209E70D
:10FFB00038B500F01BF82946204601B0BDE83040B6
:10FFC0000923CEE738B500F011F82946204601B0E4
:10FFD000BDE830400823C4E738B500F007F82946EB
:10FFE000204601B0BDE830400823BAE704460D467C
:10FFF0000222E7E638B5FFF7F9FF2946204601B0AF
:020000040001F9
:10000000BDE830400A23ACE738B5FFF7EFFF2946DB
:10001000204601B0BDE830400823A2E738B5FFF71D
:10002000E5FF2946204601B0BDE83040082398E7A7
:1000300004460D460022C5E610B50E4B0FF23802FD
:100040001C68C0F30741CC40E40746BF02EBC10186
:10005000496852F8311001F22C51020A0B680F2442
:10006000944000F00F00A34390401843086010BD77
:10007000000000006CE00F400040004000800540A0
:1000800000500040009005400060004000A0054086
:100090000070004000B005400040024000C0054034
:1000A0000050024000D005400060024000E00540E2
:1000B0000070024000F0054000D003400000064000
:1000C00000100640001006400020064000200640B8
:1000D0000030064000300640004006400040064028
:1000E0000050064000500640006006400060064098
:1000F0000070064000700640008006400080064008
:100100000090064000900640DFF830050068704718
:10011000DFF82C15085C704710B5DFF8284520780B
:10012000002802D16078002810D006F0C4FC10F03E
:10013000210F0BD100F022F8012807D188210020DF
:1001400006F0A0FC002020700020607010BD80B57B
:10015000DFF8F4140868C0F34000002807D10868ED
:1001600050F00200086000F013F801F00AF801BD39
:10017000DFF8D4040068C0F340007047DFF8C8041B
:10018000007810F001007047DFF8C0040068704785
:1001900010B5DFF8B8440020206006F08CFC10F0A9
:1001A000210F07D1FFF7EAFF012803D18021206842
:1001B00006F068FC10BD10B5DFF890442068401CC4
:1001C000206006F078FC10F0210F07D1FFF7D6FF72
:1001D000012803D18021206806F054FCDFF8680470
:1001E000016851F00201016000F0CBFF10BDF8B5CD
:1001F00005F0D0FE4FF44040DFF85414086006F0DC
:100200006DFC06F071FCDFF84C0405F059FD01208F
:1002100005F052FDDFF8400405F00EFDDFF83C0468
:1002200005F00AFDDFF8380405F006FDDFF83404B8
:1002300005F002FDDFF83044200005F0FDFCDFF89A
:100240002C0405F0F9FCDFF8280405F0F5FCDFF8D4
:100250002454280005F0F0FCDFF81C0405F0ECFC49
:10026000DFF8180405F0E8FCDFF8140405F0E4FCFE
:10027000DFF8100405F0E0FCDFF80C0405F0DCFC0E
:10028000DFF8080405F0D8FCDFF8040405F0D4FC1E
:10029000DFF8000405F0D0FCDFF8FC0305F0CCFC2F
:1002A000DFF8F863300005F0C7FCDFF8F40305F071
:1002B000C3FC06F069FB002806D0DFF88C03016858
:1002C00049084900016005E0DFF87C03016851F04E
:1002D0000101016005F0E0FC800704D50020DFF893
:1002E0006C13086012E0DFF8647304228021380088
:1002F00006F067FB386840F2E931884206D30020F7
:10030000386004228021380006F070FB280005F0D8
:10031000CBFD200005F0C8FD300005F08DFC1E204F
:1003200005F07CFE1F2005F079FE202005F076FE0A
:10033000212005F073FE0021DFF8680302F0CDFCF8
:100340000720DFF86413086005F02AFD4FF47A7186
:10035000B0FBF1F006F0D8FB06F0D0FB00210F2037
:1003600005F01FFE0F2005F02DFEB64C042288215B
:10037000200006F026FB2078332802D1607835284B
:100380000AD033202070352060700422882120009C
:1003900006F02CFB0028F8D1DFF81043200005F010
:1003A0004BFC200005F062FC06F0B6FBC04806F0EE
:1003B000C8FB5FF0704005F03FFC5FF0804006F046
:1003C00069FC012803D15FF0804006F05BFCB9496D
:1003D0005FF080400160C0465FF0804006F061FC45
:1003E0005FF0804006F043FC5FF0804006F060FC68
:1003F0005FF0804006F03AFC5FF0804006F03DFC84
:1004000005F0C4FDF1BD70B590B0AB4805F014FC2B
:10041000AA4DAB49280000F0AAFC4FF6FF74012258
:100420002100280000F0E0FCA64E3200FF21280049
:1004300000F0E6FC32004FF47F41280000F0E0FCC1
:100440006021702005F0ADFD0121280000F0F4FCD2
:10045000702005F0B7FD2100280000F079FC402253
:100460001021684606F0ADFA0098452802D00098A1
:1004700041283CD10198312839D1694688685328F0
:1004800005D08868342802D0886878282FD1C868B9
:100490004C2802D0C868302829D10869002802D029
:1004A0000869302823D14869002802D048694128CA
:1004B0001DD18869002802D08869492817D1C869E8
:1004C000002802D0C869522811D1089800280ED1FE
:1004D000099800280BD10A98002808D10B98002809
:1004E00005D1086B002802D1486B002804D05FF4C6
:1004F000003001F07AF803E05FF4003001F02BF8EF
:100500004F480E9901700F994170200005F0C8FB0B
:1005100010B070BD80B55FF0804006F0BBFB0128D5
:1005200003D15FF0804006F0ADFB67495FF080408B
:100530000160C0465FF0804006F09FFB5FF0004026
:1005400001F06CF8002823D03F480068C0F3400059
:1005500000281DD106F04EFC002819D108F0D1FA70
:10056000002815D100F022FA002811D108F02EFC45
:1005700000280DD108F00AFE002809D103F0E4FCA0
:10058000002805D109F09AF9002801D1FFF7DFFD15
:100590002D480068C0F34000002841D0FBF74BFF16
:1005A000502820D108F012FC00281CD109F065FD6C
:1005B000002818D10AF0ABFC022814D006F07BFA10
:1005C00010F0210F03D0FFF7D9FD00280BD100F068
:1005D000EBFD002807D109F071F9002803D100F0E4
:1005E000E5F9002808D0FFF78FFD38490968401A5F
:1005F00041F28931884217D305F0CCFC5FF080408E
:1006000006F048FB012803D15FF0804006F03AFB7A
:100610005FF0704005F010FB2D482E490860FBE7A5
:10062000FFF772FD2949086001BD29482949086082
:10063000FBE702480168491C01607047982D0020C3
:100640009C2D0020A02D0020A42D0020AC2D0020EA
:1006500008ED00E0800300C1000800F0010800F090
:10066000020800F0030800F0040800F0050800F09C
:10067000060800F0070800F0080800F0090800F07C
:100680000A0800F00B0800F00C0800F00D0800F05C
:100690000E0800F00F0800F0100800F0003800F01D
:1006A000005800F000800340C48F0340000C00F0AD
:1006B000001800200008AF2F015C00F0007003401C
:1006C00022220004801A060000350C00A82D00200C
:1006D0000400FA050CED00E038B5DFF85846206854
:1006E000400840002060DFF8505620236022694611
:1006F000280009F054F80028F5D009F0DFF80128A7
:1007000002D108F0F1FFF8E72021280001F0B0FE47
:1007100001280AD1002002E000212954401C202891
:10072000FAD3206850F0020020602021280001F058
:1007300079FE002803D14FF4804000F056FF287E58
:1007400009280FD0287E0A280CD0287E042809D03A
:10075000287E082806D0287E072803D04FF4804042
:1007600000F043FF0020DFF8D4150860206850F047
:100770000100206031BD38B5DFF8B8452078C007EA
:1007800040F1F1800BF0A7F80A2880F2B1804FF415
:10079000804000F0E0FEDFF8A0552021280001F0A5
:1007A00041FE002804D14FF4804000F01EFF4FE0CE
:1007B000287E092810D0287E04280DD0287E0828FD
:1007C0000AD0287E0A2807D0287E072804D04FF4B4
:1007D000804000F00AFF3BE01E2003F0A3FB297ECF
:1007E000884204D04FF4804000F0FFFE30E02868DB
:1007F000002804D14FF4804000F0F7FE28E028687C
:100800006968C943884204D04FF4804000F0EDFE8F
:100810001EE0287F032804DB4FF4804000F0E5FE53
:1008200016E0687F022804DB4FF4804000F0DDFE14
:100830000EE0E87E022804DB4FF4804000F0D5FE95
:1008400006E0A87F032803DB4FF4804000F0CDFED4
:100850004FF4804000F0E2FE002841D14FF4805078
:1008600000F079FE5FF0004003F023FB002802D186
:10087000E87E002808D15FF0004003F01AFB002852
:1008800007D0E87E002804D14FF4805000F0ADFE80
:1008900032E04FF4007003F00CFB002802D1687FB7
:1008A000002808D14FF4007003F003FB002807D0A4
:1008B000687F002804D14FF4805000F096FE1BE0C2
:1008C0005E2003F02FFBA97F884215D01E2003F085
:1008D00029FB072810D14FF4805000F086FE0BE072
:1008E0004FF4805000F037FE202000F034FE03E08B
:1008F0004FF4805000F02FFE2068C0F34000002825
:100900000BD020226021DFF8300408F089FF012895
:1009100003D1206830F0020020600AF0DCFFC0B292
:100920000A281ED1FFF724FC012805D1202000F061
:100930005CFE0AF0F1FF16E0DFF8001408680028FA
:1009400002D100F070F80EE00868012802D100F032
:1009500044F908E05FF4003000F037FE0AF0DCFFF5
:1009600001E000F0D9F931BDDFF8D00300680028BC
:1009700005D1DFF8C003016851F004010160704740
:10098000DFF8B0030068C0F380007047002004E087
:100990000021DFF8A4231154401C2028F8D3DFF8ED
:1009A0009403016851F0020101607047DFF884038D
:1009B000007810F00A0F01D0012000E000207047FD
:1009C000DFF87403007E704780B54FF4804000F07C
:1009D00025FE002803D1DFF86003006801E05FF026
:1009E000FF3002BDDFF850130860C0434860704715
:1009F000DFF84403807F7047DFF83C03C07E0028A7
:100A000001D1002000E00120704780B500200BF0EC
:100A100033F9FFF779FBDFF8281308600020DFF8CF
:100A20001C13086001BD70B580200BF0B3FC0AF008
:100A300055FF04005FF40000002100F0A7FD002333
:100A4000002200210020FBF7D3FC01200AF057FA16
:100A5000B84D2868C0F38000002813D1FFF754FB7D
:100A6000B7490860E4B2022C01D10AF055FF4FF4F7
:100A7000804000F0D3FD002800F0AE80202000F080
:100A80006AFDA9E0FFF740FBAD4E3168401A41F224
:100A90008931884243D22000C0B203283FD0E4B25B
:100AA000022C3CD0A74804F020FA002837D15FF090
:100AB000015004F01AFA002831D1A34804F015FAC5
:100AC00000282CD15FF4801004F00FFA002826D102
:100AD000102000F0A3FD002821D11E2003F022FAEF
:100AE000092813D01E2003F01DFA04280ED01E2062
:100AF00003F018FA0A2809D01E2003F013FA082878
:100B000004D01E2003F00EFA072808D14FF48040CD
:100B1000002100F096FD002901D1002807D02868A7
:100B200030F004002860202000F05FFD54E0FBF767
:100B300082FC502850D1286830F0040028605FF013
:100B4000FF3000F008FD286850F002002860002007
:100B500003E00021784A1154401C2028F9D3764C38
:100B60001E2003F0DFF920765E2003F0DBF9A0778A
:100B70005FF0004003F09DF9002805D0207E062894
:100B800002D00120E07601E00020E0764FF4007012
:100B900003F08FF9002805D0207E062802D001201E
:100BA000607701E000206077022003F082F90028DE
:100BB00002D10220207701E00120207700220021CD
:100BC000092007F0BEFEFFF79FFA306001200AF00F
:100BD00096F901205949086070BD10B50AF07EFEF3
:100BE00004005FF40000002100F01CFDFBF723FC73
:100BF000652803D181200BF0CDFB06E0FBF71BFC41
:100C0000662802D182200BF0C5FB0AF080F9022889
:100C10000ED00AF07CF9012803D15FF4000000F047
:100C2000E4FC0023002200210520FBF7E1FB05E0A6
:100C30000023002200210020FBF7DAFB2000C0B2D5
:100C4000022805D1202000F0D0FC0AF065FE62E009
:100C5000E4B2032C24D03B4804F047F900281FD10C
:100C60005FF4801004F041F9002819D15FF00150C1
:100C700004F03BF9002813D1334804F036F900287A
:100C80000ED14FF48040002100F0DBFC002907D199
:100C9000002805D1274C2068C0F38000002805D02B
:100CA000202000F0A2FC00F037F834E0274800F0E4
:100CB000B5FC002802D000F02FF82CE0FBF7BBFBBE
:100CC00010F1010F27D1022003F0F3F8002803D11F
:100CD00002201949087702E00120174908774FF4EC
:100CE000007003F0E6F8002803D00120124948778D
:100CF00002E000201049487720210F4801F0A8FBAE
:100D0000206850F0020020605FF40000002100F035
:100D10003DFC0AF001FE10BD80B5FFF7F5F908496A
:100D200008600020054908600248016831F00401AC
:100D3000016001BD8C2D00208C280020902D00200A
:100D4000942D002040000080800000405881A66A59
:100D500050F80C3F40F20112114042E050F80C3FB5
:100D600040F20112114023EA010101607047F0B521
:100D700000F10C03164A1C68124D144F14401C60FD
:100D80000A0E026000F108032E680F4A001D16408B
:100D9000BE4201F0FF040BD10D0905F470452C4350
:100DA00044F4007404604FF2FF0000EA112004E0F4
:100DB00044F400740460C1F3072040F4007018602C
:100DC000F0BD000000E00F400000FF7000000A10BE
:100DD000FEFEFFFF40F60C43194050F80C3F8B43DA
:100DE000114019430160704740F2022319400C3052
:100DF000002A026814BF114322EA01010160704712
:100E00000B061CBF00F128031A6011F47F4F18BFB6
:100E100040F82C2F7047FF290CBF28302C30006879
:100E200070470B061CBF00F130031A6011F47F4FAE
:100E300018BF40F8342F704750F8182F1143016045
:100E4000704740F8241F704738B5DFF82C45002064
:100E50002060DFF82805DFF828150860FF20DFF89C
:100E600024150860DFF8205501212800FFF792F8CB
:100E70000823012201212800FEF7DEFF0020DFF811
:100E80000C15086010215FF04020FFF783F8002068
:100E9000DFF8FC140860DFF8FC54280004F0CCFEF6
:100EA000280004F0E3FEDFF8F004FFF7C5F8DFF8F0
:100EB000EC04FFF7C1F80C21DFF8E404FFF7AEF80B
:100EC00004F06EFF0100DFF8DC5460235FF4E132D0
:100ED00028000DF0B5FE1022022128000DF0ACFE16
:100EE000DFF8C404016831F010010160102128000E
:100EF0000DF0F9FE28000DF0D2FE032128000DF0C0
:100F000000FFDFF8A80405F08DFEDFF8A40405F06B
:100F100089FEA0214D2005F044F84D2005F052F83F
:100F20000F21062005F010FEDFF88814062005F0DA
:100F30001EFE00F07FF90F21072005F005FEDFF807
:100F40007814072005F013FEDFF87004002101700B
:100F50000021417000218170DFF86404016851F4C0
:100F600000210160016851F4803101600020DFF848
:100F7000541408600020DFF8501408600020DFF8E7
:100F80004C1408600120206031BD80B5DFF8E80313
:100F90000068002832D0DFF824040078002806D04A
:100FA000DFF81C040068C00101D5FFF7B5F84FF465
:100FB000007002F07EFF002812D1DFF804040168FF
:100FC000090C090401600020DFF80014086000200B
:100FD000DFF8F41308605FF0006000F0BCFA0DE089
:100FE000DFF8DC030068002804D05FF0006000F048
:100FF000FCFA03E05FF0006000F0ADFA01BD80B5DF
:10100000A0B080234FF480726946DFF8C40306F075
:1010100001F8012840F083806946487800281AD0FA
:10102000DFF89803002101700021417000218170D8
:10103000DFF88C03016851F400210160016851F46C
:10104000803101600020DFF8801308600020DFF8A5
:101050008413086062E08878C0283DD10020DFF862
:1010600074231060DFF85803026832F480320260A3
:101070009DF80320872A1CD1DFF8402387231370B3
:10108000036833F400230360497951709DF806101A
:1010900091705178332907D19178352904D10168AD
:1010A00031F08071016039E0016851F080710160B8
:1010B00034E0016851F400210160016831F0807171
:1010C0000160BE4800210170002141700021817043
:1010D0000020BD49086021E08878C2281AD100208C
:1010E000BC4A1060B64A106830F480301060106856
:1010F000000C00041060B548006800280ED1136889
:101100009DF80400034313601068497950EA0120F8
:10111000106003E0AF480168491C016003E0AD487E
:101120000168491C0160AB4800680B2807D3A4483C
:10113000016851F4807101600020A349086021B06A
:1011400000BD80B58C480068012815D14FF40070AF
:1011500002F0AFFE002809D099480168090305D4C0
:101160000168C90302D40068C00102D500F08EF8FE
:1011700006E000F0A9F803E04FF4804000F025FA03
:1011800001BD80B58D480078002809D04FF400706B
:1011900002F08FFE002803D001208B49086002E096
:1011A00000208949086001BD80B54FF4007002F04D
:1011B00080FE002802D08448006800E0002002BDC4
:1011C00001208249086070477C49C0B2085C7047C2
:1011D00010B504004FF4007002F06BFE002801D13E
:1011E000002402E0764800680440200010BD80B56D
:1011F0007348006801F065F902BD10B5694C012122
:1012000020000DF075FD010020000DF077FD6D4808
:101210000068002807D1062005F0F0FC002808D15E
:1012200000F008F805E06C480068800601D500F081
:1012300001F810BD80B5002062490860062005F065
:1012400078FC002003E00021614A1154401CB0F5F5
:10125000807FF8D34FF4807000905D4B514A01219C
:10126000062005F090FC062005F05BFC01BD80B572
:101270000121544A116000904A4B584A012107202D
:1012800005F081FC072005F04CFC01BD80B5A0B045
:1012900005208DF8000000208DF80100C0208DF899
:1012A000020068460421C170C178C943017133212D
:1012B000417135208DF806004849684605F024FF45
:1012C000FFF7D5FF21B000BD70B5A0B008208DF8A4
:1012D00000006C4600206070C120A070FBF7B8F8D9
:1012E0008DF80300FBF72FF920710100090A8DF832
:1012F00005100100090C8DF80610000E8DF807008E
:101300000025FBF742F9012801D155F001052E4EC9
:101310003068012807D1FBF78EF8502803D155F02B
:10132000020500203060294E3068012817D1FBF7F4
:1013300082F8522813D0FBF77EF854280FD0FBF721
:101340007AF857280BD0FBF776F8652807D0FBF71B
:1013500072F8662803D055F004050020306025722D
:1013600000208DF809001D49684605F0CDFEFFF705
:101370007EFF20B070BD00004C2A00204B434F4C34
:1013800020550240245502400050024004500240C3
:1013900040400040051800F001080800010C08005A
:1013A00000D00340001001402C1001400600020054
:1013B000070002000080000C008000C0542A0020BA
:1013C000582A0020502A0020482A0020442A0020C1
:1013D000801900205C2A00203C100140801A002067
:1013E0000020A749086000200021A64AC2E90001A8
:1013F0000020A54908600020A44908600020A449F5
:1014000008600020A349086070472DE9F0419C4C1A
:101410002068002804D0012100200DF0D4FD13E045
:101420009848D0E900019C4A102310401940002937
:1014300001D1002804D0022100200DF0C4FD03E0FA
:10144000002100200DF0BFFD0EF01DF901280FD086
:101450000EF0B2FA01280BD00EF048FD012807D09B
:101460000EF081FF012803D008F005FD012804D10A
:101470000020102100F0D6F803E00020102100F039
:1014800085F8FEF775FE002863D1002521E020686D
:1014900030421DD17C4F3868304219D0300000F006
:1014A000D6F801000022052007F04BFA01280FD1E1
:1014B000386830EA06063E600AE000200200414635
:1014C000042007F03EFA012802D1386806433E6046
:1014D0006D1C202D24D20126AE4020683042D6D08B
:1014E000694F38683042D2D1300000F0B0F8804601
:1014F000B8F11D0F02D1FFF77AFEDFE7B8F1010F57
:1015000005D16348006800F0DCFF401CD6E7B8F165
:10151000050FD2D15F48006800F0D3FF401CCDE733
:10152000584AD2E9000180030FD5584C2068800347
:101530000BD400223C210C2007F003FA012808D12B
:10154000206850F40030206003E0D2E900014F49E8
:101550000860BDE8F08138B50400504D254004F026
:1015600019FD4748016831EA0505056004F00EFDE4
:1015700014F1010F09D1FFF723FEFAF764FF0020F1
:101580004349086000204349086031BD38B5040074
:101590000D0004F0FFFC3B48D0E90023A243AB431D
:1015A000C0E9002304F0F2FC31BD10B5040004F0E2
:1015B000F1FC3348016851F01001016034480168C2
:1015C0000C43046004F0E2FC10BD10B5040004F00C
:1015D000E1FC2B48016851F0080101602D480168C9
:1015E0000C43046004F0D2FC10BD10B5040004F0FC
:1015F000D1FC234801680C43046004F0C7FC10BD13
:1016000080B52348006800F05CFF401C02BD80B537
:101610002048006800F055FF401C02BD18490968C9
:101620000840704738B504000D0004F0B3FC1548BD
:10163000D0E9002322432B43C0E9002304F0A6FC99
:1016400031BD104AD2E9002310401940704780B5DF
:1016500000F037FF202802D21149085C00E000208A
:1016600002BD80B5074AD2E900231040194000F0BE
:10167000AAFF402802D20B49085C00E0002002BD0E
:10168000142B0020F0290020182B00201C2B0020F8
:10169000202B0020242B0020009E4B24B7FFF9FDB7
:1016A000FC4102007440020038B5DFF8284B80216D
:1016B0002000FEF76FFC8020DFF81C1B086004216F
:1016C0002000FEF767FC0020DFF8101B0860DFF841
:1016D000104B10212000FEF75DFC20212000FEF7BA
:1016E00059FC0020DFF8FC1A08602020DFF8F81A07
:1016F0000860DFF8F84A10212000FEF74BFC1020AC
:10170000DFF8EC1A0860DFF8EC5A40212800FEF7F9
:1017100041FC0020DFF8001C086010212800FEF7C3
:1017200039FC0020DFF8D01A086020212800FEF7DD
:1017300031FC0020DFF8C41A0860DFF8C40A04F0A6
:101740007BFADFF8C05A22212800FFF710FB0122A4
:10175000FF212800FFF748FB8021272004F021FC0F
:10176000DFF8A42AFF212800FFF74AFB0121280007
:10177000FFF762FB01212800FFF763FB272004F03D
:1017800021FCFF212800FFF7E3FA0620DFF87C1A8E
:1017900008607121DFF8780AFEF7D4FB03212000EE
:1017A000FEF7D0FB0121DFF86C0AFEF7CBFBDFF878
:1017B000684A012300220021200001F0CCF9052312
:1017C00000220021200001F0F0F90623012200216F
:1017D000200001F0EAF9072302220021200001F095
:1017E000E4F9032303220021200001F0DEF90223A3
:1017F00004220021200001F0D8F96F2305220021E6
:10180000200001F0D2F90021200001F097F9002119
:10181000200001F08FF90021200001F084F9E0217F
:101820001E2004F0BEFB1E2004F0CCFBDFF8EC0A07
:1018300000680028FAD0DFF8C04B206830F01000B4
:101840002060FEF761FCDFF8781B0860FEF75CFCA7
:10185000DFF8701B0860FEF757FCDFF86C1B0860B0
:10186000FEF752FCDFF8941B0860022000F058FDE0
:1018700046F66051884213D24E2002F053FBC00757
:101880000BD41E2002F04EFB082803D04FF48070CA
:10189000FFF7ABFE00F010FA0DE000F0C8F90AE027
:1018A00000F00AFA4E2002F03DFBC00703D5206885
:1018B00050F00800206031BD10B5DFF8600A006804
:1018C000012816D1DFF8304B2078C00702D500F090
:1018D000D7F801E000F042FA00F0A0FC00F0DBFBDA
:1018E0002068C0F30020002803D04FF40070FFF7F9
:1018F0005CFE10BD80B50100C9B2042903D0C0B29E
:1019000000F00EFD02E0DFF8F80A006802BD80B5C5
:101910004FF480400021FFF794FE002901D10028F8
:1019200018D00E2002F01AFB002813D14FF40060EB
:1019300002F0BFFA00280DD009F0D0FF022803D032
:1019400009F0CCFF032805D1DFF8AC0A016851F09B
:101950001001016001BDDFF8A00A016831F010013B
:1019600001607047DFF8900A0068C0F3C0000028EB
:1019700004D1DFF88C0A407D002801D0012000E06E
:101980000020704780B54FF480400021FFF759FEDA
:10199000002906D1002804D18020DFF83C18086017
:1019A00003E00020DFF83018086001BD10B5DFF853
:1019B00028482068002808D14FF480400021FFF714
:1019C00040FE002901D100280BD0206800280AD051
:1019D0004FF480400021FFF734FE002901D1002898
:1019E00001D0002000E0012010BDDFF80C0A0068E3
:1019F000C0F34000002801D1012000E00020704722
:101A000010B586B0DFF810480021200001F092F8F0
:101A10006A460021200001F015F9DFF8F017086888
:101A2000401C08600868062806D10120DFF8EC2871
:101A300010600020086004E00868062801D3002038
:101A4000086000220CE0DFF8BC390C681820444321
:101A500003EB04006B4653F8223040F82230521C4E
:101A6000062AF0D306B010BD80B50121DFF8940737
:101A7000FFF7E7F90021DFF8A00701F0F6F801BD54
:101A800070B54FF480400021FFF780FDDFF8685902
:101A9000286830F010002860FEF736FBDFF8681980
:101AA0000860286830F400702860DFF8544902208C
:101AB00000F036FC606046F660566068B0420FD2B7
:101AC000FEF722FBDFF8F8180968401A652807D3EB
:101AD0004E2002F027FAC00702D500F0A8F8A5E0D2
:101AE0006068B0421AD25FF08040FFF734FDFEF725
:101AF0000BFBDFF8CC180968401A65281BD34E2071
:101B000002F010FAC00716D41E2002F00BFA0828C3
:101B100011D04FF48070FFF768FD0CE0FEF7F4FA87
:101B2000DFF89C1808605FF08040FFF714FD4FF469
:101B30008070FFF710FD00F0B5F900F004FA052001
:101B400000F0EEFBA0606168A068081A41F27171B4
:101B500088420EDBFEF7D8FADFF86C180968401AE5
:101B600040F2D17188420DD3286850F4807028600B
:101B700008E0FEF7C9FADFF850180860286830F46A
:101B8000807028604E2002F0CDF9C0070DD44FF4CC
:101B90000070FFF7E0FC5FF080400021FFF7F6FCEB
:101BA0000020206000F004FB2EE0FFF7DBFE0028A1
:101BB0002AD1FEF7A9FADFF854482168401ADFF865
:101BC0005018884204D3286850F0080028601BE0B1
:101BD000042000F0A5FB2968C1F38011002903D07F
:101BE00047F61911884207D22968C1F380110029EC
:101BF0000AD1B0F5FA6F07D25FF080400021FFF7FD
:101C000011FDFEF781FA20605FF080400021FFF7B0
:101C100018FD002901D1002804D0012102200DF077
:101C2000D2F903E0002102200DF0CDF970BD10B50E
:101C30002020DFF8B4150860FEF766FADFF8C01759
:101C40008861DFF8B447206850F002002060206807
:101C500050F004002060206840084000206000F040
:101C6000A7FAFEF751FADFF858170860FEF74CFAAA
:101C7000DFF850170860FEF747FADFF880170860B2
:101C8000206830F4807020605FF080400021FFF712
:101C90007DFC4FF480400021FFF7C4FC5FF08040E2
:101CA000FFF759FC4FF40070FFF755FC00220121AB
:101CB0000F2006F046FE10BD80B54FF40070FFF710
:101CC000ADFC002802D0FEF742FA46E00020DFF823
:101CD000141508601020DFF818150860FEF714FAD4
:101CE000DFF81C178861DFF81007016851F0020166
:101CF0000160016851F004010160016851F00101C7
:101D00000160FEF701FADFF8B8160860FEF7FCF98B
:101D1000DFF8B0160860FEF7F7F9DFF8E0160860A4
:101D2000FEF7F2F9DFF8A0160860FEF7EDF9DFF82C
:101D3000DC1608604FF40070FFF70DFC5FF0804088
:101D40000021FFF723FC4FF480400021FFF71EFC29
:101D5000002200210F2006F0F4FD01BD38B500F08F
:101D600027FADFF89C46022000F0DAFA606047F2BA
:101D700031556068A8420AD3FEF7C6F9DFF8941619
:101D80000968401A652802D3FFF796FF89E060686A
:101D9000A84204D2FEF7B8F9DFF87816086009F017
:101DA000A0FD012840D14FF40070FFF71EFC002079
:101DB000DFF8341408601020DFF8281408600020D1
:101DC000DFF82C140860DFF830462068C0F34020AC
:101DD000002815D1002102200DF0F5F8FEF794F946
:101DE000DFF824562968401A40F6B831884258D3A3
:101DF000FEF78AF92860206850F40070206050E0F7
:101E0000012102200DF0DFF8FEF77EF9DFF8F8552A
:101E10002968401AC82844D3FEF776F9286020685C
:101E200030F4007020603CE02020DFF8BC13086034
:101E3000FEF76AF9DFF8D0150860DFF8BC552868AE
:101E400030F400702860022102200DF0BCF85FF031
:101E500000500021FFF7F5FB002901D1002803D035
:101E6000286850F010002860042000F059FA206023
:101E700009F031FD062803D009F02DFD052802D117
:101E800044F6206001E045F2F0502168814204D21E
:101E90005FF080400021FFF7C5FB00F003F800F081
:101EA00052F831BD38B5DFF85855012000F038FA46
:101EB000E860DFF844452068C0F34000002832D1D4
:101EC0002078C00704D41020DFF81813086002E05F
:101ED0000020C54908605FF080400021FFF7B1FB9A
:101EE000002901D1002802D02078C0072AD5E8684F
:101EF00042F6E06188420CD2FEF706F9DFF8C4141E
:101F00000968401AC9281DD3206850F0800020605D
:101F100018E0FEF7F9F8DFF8AC140860206830F03C
:101F2000800020600EE0FEF7EFF8A969401AC9288A
:101F300003D3206830F002002060FEF7E5F8DFF8F8
:101F40008414086031BD38B5DFF8AC442078C00790
:101F500003D5206830F010002060DFF8A454002082
:101F600000F0DEF92861206810F4026F5CD11020C7
:101F70009F4908602068C0F38000002834D15FF0DA
:101F800080400021FFF75DFB002901D1002802D02D
:101F90002078C00722D5286942F6E061884214D231
:101FA000FEF7B2F8DFF854140968401A40F2D17114
:101FB00088422AD30420FFF718FB206850F4006001
:101FC0002060FEF7A1F8A8611FE0FEF79DF8DFF89A
:101FD0002C1408600420FFF7BEFA16E0FEF794F810
:101FE000DFF81814086010E0FEF78EF8A969401AAF
:101FF00040F2D171884203D3206830F004002060A1
:10200000FEF782F8DFF8F41308602068C0F30010D0
:1020100000283FD0206850F020002060FEF774F8C0
:10202000DFF8D813086035E02068C0F3C02000282E
:102030001AD0FEF769F8A969401A47F2315188426F
:102040000ED3FEF761F8A861206850F0040020600C
:10205000206830F40060206010206549086019E0B5
:1020600000206349086015E05FF000700021FFF771
:10207000D9FA00205E4908602068C0F300100028EB
:1020800008D1206830F020002060FEF73DF8DFF82E
:102090006C13086031BD38B54FF480400021FFF764
:1020A000D0FA00291ED100281CD14F480068002812
:1020B00018D1FFF757FC012814D0DFF84443607DA6
:1020C00000280FD1FEF754F801280BD0DFF8285371
:1020D0002868C0F38020002804D14E2001F022FFA0
:1020E000C00718D400204549086000204249086014
:1020F0000320C3490875FEF707F80A38DFF81813FC
:102100000860002101200CF05EFFBB48016831F03F
:10211000400101604BE0286850F04000286010202A
:1021200035490860206846F6615188420DD35FF05A
:1021300080400021FFF785FA002906D1002804D14C
:10214000012101200CF03FFF03E0022101200CF0EF
:102150003AFFFDF7D9FFB04D2968401A0A2826D367
:10216000FDF7D2FF2860207D401C2075207D0428CB
:1021700001DB01202075207D012803D120201F498B
:10218000086014E0207D02280ED1042000F0EAF857
:1021900044F62161884203D320201849086006E0F4
:1021A00000201649086002E000201449086031BD93
:1021B00080B50020584908608F48016831F0080157
:1021C000016000208E494875FDF79EFF8F49086029
:1021D00001BD000000F0054000F2054010F0054090
:1021E00000300640403006408030064000C00540C8
:1021F00040C0054000400640404006408040064048
:10220000020400F000200340007102005C2D002059
:1022100000700040001006400080034038B5784C44
:10222000607D00280FD174480068C0F3C00000280A
:1022300070D0FDF769FF7949086001206075402082
:102240003549086066E0607D012859D1FDF75CFFE3
:1022500072490968401A962805D267480068C0F399
:10226000C000002856D1042000F05AF82060002059
:1022700029490860604D2868C0F3C000002834D0A8
:102280005FF080400021FFF7DCF9002906D100282B
:1022900004D1206845F6D81188420DD35FF0804004
:1022A0000021FFF7CEF9002901D100280AD02068CB
:1022B00045F6C051884205D25FF080400021FFF70B
:1022C000B1F904E05FF080400021FFF75FF920687A
:1022D00047F61911884204D3286850F480602860BA
:1022E00003E0286830F480602860FDF70DFF47495F
:1022F000086000206075286830F00800286009E058
:102300003D48016831F0080101600020607500203F
:102310000149086031BD000000410640582D0020F1
:1023200010B504002000C0B200F050F8E4B2002C58
:1023300008D0022C0DD005D3042C03D009D3052CD2
:1023400007D00DE040F2763148436421B0FBF1F054
:1023500007E04FF49E6148436421B0FBF1F000E0D8
:10236000002010BD38B5040003F014FE2C480168AD
:10237000244A1820414302EB01002100C9B250F861
:10238000215003F003FEE4B2002C08D0022C0DD043
:1023900005D3042C03D009D3052C07D00DE040F25F
:1023A000763045436420B5FBF0F007E04FF49E60C3
:1023B00045436420B5FBF0F000E0002032BD000092
:1023C0006C2D0020642D0020602D002010B4002210
:1023D00000230AE00B49182404FB03F42144040001
:1023E000E4B251F824108A185B1C062BF2D30620A5
:1023F000B2FBF0F010BC7047542D0020682D002077
:102400006C28002048240020742D0020702D00200E
:10241000E19304006C2D0020782D00207C2D0020FD
:102420005C2D002010B40122002302E0C45C1219CC
:102430005B1C4C1EA342F9D3D243084410F8010C94
:10244000D2B2824201D0002000E0012010BC7047CF
:1024500010B40122002302E0C45C12195B1C4C1E64
:10246000A342F9D3D243084400F8012C10BC7047B2
:10247000002200E0521C1300DBB28B4206D2130094
:10248000DBB2C35CFF2BF5D0002000E001207047D9
:1024900000210100C9B230390A2902D23038C0B255
:1024A00008E00100C9B24139062902D23738C0B26A
:1024B00000E00020704710F00F00DFF86815085C9E
:1024C0007047002801D120207CE0C10701D5002001
:1024D00078E0810701D5012074E0410701D5022091
:1024E00070E0010701D503206CE0C10601D504208E
:1024F00068E0810601D5052064E0410601D506208B
:1025000060E0010601D507205CE0C10501D5082087
:1025100058E0810501D5092054E0410501D50A2084
:1025200050E0010501D50B204CE0C10401D50C2081
:1025300048E0810401D50D2044E0410401D50E207E
:1025400040E0010401D50F203CE0C10301D510207B
:1025500038E0810301D5112034E0410301D5122078
:1025600030E0010301D513202CE0C10201D5142075
:1025700028E0810201D5152024E0410201D5162072
:1025800020E0010201D517201CE0C10101D518206F
:1025900018E0810101D5192014E0410101D51A206C
:1025A00010E0010101D51B200CE0C10001D51C2069
:1025B00008E0810001D51D2004E0400001D51E2067
:1025C00000E01F207047002903D1002801D14020DE
:1025D000BEE10200D20701D50020B9E10200920756
:1025E00001D50120B4E10200520701D50220AFE17C
:1025F0000200120701D50320AAE10200D20601D58C
:102600000420A5E10200920601D50520A0E1020008
:10261000520601D506209BE10200120601D50720D3
:1026200096E1C20501D5082092E1820501D5092075
:102630008EE1420501D50A208AE1020501D50B2071
:1026400086E1C20401D50C2082E1820401D50D206F
:102650007EE1420401D50E207AE1020401D50F206B
:1026600076E1C20301D5102072E1820301D5112069
:102670006EE1420301D512206AE1020301D5132065
:1026800066E1C20201D5142062E1820201D5152063
:102690005EE1420201D516205AE1020201D517205F
:1026A00056E1C20101D5182052E1820101D519205D
:1026B0004EE1420101D51A204AE1020101D51B2059
:1026C00046E1C20001D51C2042E1820001D51D2057
:1026D0003EE1420001D51E203AE1002801D51F202D
:1026E00036E110F0000211F00103002B01D1002AA5
:1026F00001D020202CE110F0000211F00203002B89
:1027000001D1002A01D0212022E110F0000211F0B5
:102710000403002B01D1002A01D0222018E110F07F
:10272000000211F00803002B01D1002A01D0232060
:102730000EE110F0000211F01003002B01D1002A6D
:1027400001D0242004E110F0000211F02003002B3E
:1027500001D1002A01D02520FAE010F0000211F08A
:102760004003002B01D1002A01D02620F0E010F018
:10277000000211F08003002B01D1002A01D0272094
:10278000E6E010F0000211F48073002B01D1002A62
:1027900001D02820DCE010F0000211F40073002BBF
:1027A00001D1002A01D02920D2E010F0000211F45A
:1027B0008063002B01D1002A01D02A20C8E010F04C
:1027C000000211F40063002B01D1002A01D02B205C
:1027D000BEE010F0000211F48053002B01D1002A5A
:1027E00001D02C20B4E010F0000211F40053002BB3
:1027F00001D1002A01D02D20AAE010F0000211F42E
:102800008043002B01D1002A01D02E20A0E010F03F
:10281000000211F40043002B01D1002A01D02F2027
:1028200096E010F0000211F48033002B01D1002A51
:1028300001D030208CE010F0000211F40033002BA6
:1028400001D1002A01D0312082E010F0000211F401
:102850008023002B01D1002A01D0322078E010F033
:10286000000211F40023002B01D1002A01D03320F3
:102870006EE010F0000211F48013002B01D1002A49
:1028800001D0342064E010F0000211F40013002B9A
:1028900001D1002A01D035205AE010F0000211F4D5
:1028A0008003002B01D1002A01D0362050E010F027
:1028B000000211F40003002B01D1002A01D03720BF
:1028C00046E010F0000211F08073002B01D1002AC5
:1028D00001D038203CE010F0000211F00073002B12
:1028E00001D1002A01D0392032E010F0000211F0AD
:1028F0008063002B01D1002A01D03A2028E010F09B
:10290000000211F00063002B01D1002A01D03B200E
:102910001EE010F0000211F08053002B01D1002ABC
:1029200001D03C2014E010F0000211F00053002B05
:1029300001D1002A01D03D200AE010F0000011F082
:102940008041002901D1002801D03E2000E03F2035
:102950007047012111FA00F07047002801D40120CE
:1029600001E05FF0FF307047002801D54042FFE7EB
:102970007047C0B230380A2801D2012000E00020A0
:10298000704730B43C22B0FBF2F23C2404FB12004E
:1029900008603C20B2FBF0F304FB13224A601820CD
:1029A000B3FBF0F2182000FB12338B60101D0723DD
:1029B000B0FBF3F403FB1400886102F2DB2240F267
:1029C000B550B2FBF0F340F2B55000FB13203C28A9
:1029D00002D35B1C0C2400E00224D01A40F26D15D7
:1029E000B0FBF5F0443048614D69443D40F26D1054
:1029F00000FB1522D21A002000E0401CA04204D2A5
:102A0000094B53F820309A42F7D2431E0B61064B14
:102A100003EB800050F8040C121A521CCA6030BC40
:102A20007047000038420200B440020078B589B017
:102A300005005FF000465FF0804469463000FFF714
:102A4000A0FF6946280000F01BF80DE0361B02E0ED
:102A50000128FBDBA619640869463000FFF791FFE7
:102A60006946280000F00CF8002801D0002CEFD1B6
:102A7000002801D1300001E05FF0FF300AB070BDE6
:102A80004A6943699A4201DA012048E042694B6988
:102A90009A4202DA5FF0FF3041E00A6903699A4224
:102AA00001DA01203BE002690B699A4202DA5FF029
:102AB000FF3034E0CA68C3689A4201DA01202EE090
:102AC000C268CB689A4202DA5FF0FF3027E08A687A
:102AD00083689A4201DA012021E082688B689A4279
:102AE00002DA5FF0FF301AE04A6843689A4201DA7E
:102AF000012014E042684B689A4202DA5FF0FF302E
:102B00000DE00A6803689A4201DA012007E00068D4
:102B10000968884202DA5FF0FF3000E00020704769
:102B200050F8082F10E0012202FA01F100F10C0226
:102B30001160CAE0012202FA01F1CBE00268012330
:102B400003FA01F1C3E00268012303FA01F122EA6A
:102B5000010101607047F0B500F1140689000F25EE
:102B60008D403468ED4302F00F0705EA040C07FAC4
:102B700001F444EA0C04346003F0030300F1200480
:102B800003FA01F126683540BF1F2943032F216056
:102B90000AD8FF0050F81C1F3023BB4002F030025F
:102BA0009943BA400A430260F0BD70B54901403113
:102BB000081892000F2191400468C94303F00F05E3
:102BC0000C4095402C430460C3F3032600F1180425
:102BD000964025680D4035432560041DC3F3031658
:102BE00000F01EF800F11C04C3F3035600F018F8BF
:102BF0000124944013F4702F00F110050BD050F80D
:102C0000146FC3F30243314003FA02F20A43026035
:102C10002868044302E0286820EA04042C6070BDA0
:102C200025680D409640354325607047012202FA21
:102C300001F140F8101F7047012202FA01F140F83B
:102C4000181F704730B5490140310B1803F10801D6
:102C500000200C331C68E50506D408283EBF0C682C
:102C600042F8044B401CF5D330BD10B50B0C0124C9
:102C700001F00F0150F8282F04FA01F141EA034155
:102C80001143016010BD002200E0521C4908FCD134
:102C900040F8302F704700EB810000F56060026063
:102CA000704700EB810000F5646042EA0342026075
:102CB000704750F8082F4FF4803346E750F8082F3C
:102CC0004FF4803303FA01F101E050F8082F11436B
:102CD0000160704740F80C1F704750F8382F920879
:102CE00041EA8201016070472DE9F041DFF8484870
:102CF0002068400840002060206830F0020020601A
:102D0000206830F004002060206830F00800206067
:102D1000DFF8285800202860DFF8246800203060A1
:102D2000DFF8207800203860206830F00200206052
:102D3000206830F004002060206830F00800206037
:102D4000206830F010002060206830F02000206003
:102D5000206830F040002060DFF8EC8720234FF43B
:102D600080722900404606F01AFD0028F4D006F0D3
:102D7000A5FD012802D106F0B7FCF8E718F12005FF
:102D800020234FF490723100280006F008FD00283F
:102D9000F4D006F093FD012802D106F0A5FCF8E777
:102DA00018F1400620234FF4A0723900300006F0DD
:102DB000F6FC0028F4D006F081FD012802D106F0CF
:102DC00093FCF8E760214046FFF752FB012804D14D
:102DD0000121002001F012F8AEE020214046FFF76B
:102DE00021FB002804D15FF40010FEF7FEFBA3E0F6
:102DF00020212800FFF716FB002804D15FF4001003
:102E0000FEF7F3FB98E020213000FFF70BFB0028D2
:102E100004D15FF40010FEF7E8FB8DE01E2001F006
:102E200081F809281BD01E2001F07CF80A2816D052
:102E30001E2001F077F8042811D01E2001F072F84E
:102E400008280CD01E2001F06DF8072807D05FF489
:102E50000010FEF7CAFB0021002000F0CFFF542035
:102E600001F060F8062803D30121542000F070FB24
:102E7000572001F057F8102803D30121572000F004
:102E800067FB582001F04EF8032803D30121582096
:102E900000F05EFB592001F045F8032803D301211F
:102EA000592000F055FB5D2001F03CF80B2804D2BE
:102EB0005D2001F037F8002803D101215D2000F0EA
:102EC00047FB5E2001F02EF8032803D301215E208A
:102ED00000F03EFB5C2001F025F80B2803D3012114
:102EE0005C2000F035FB532001F01CF80F2803D2C2
:102EF0000121532000F02CFB0021404601F002FB91
:102F0000002804D15FF40010FEF76FFB14E02021CD
:102F1000280001F0F7FA002804D15FF40010FEF752
:102F200064FB09E04021300001F0ECFA002803D1F5
:102F30005FF40010FEF759FB206850F0010020609C
:102F4000BDE8F08180B5DFF8F0050078C00742D514
:102F50001E2000F0E7FF092817D01E2000F0E2FF36
:102F60000A2812D01E2000F0DDFF04280DD01E20FC
:102F700000F0D8FF082808D01E2000F0D3FF072853
:102F800003D05FF40010FEF730FB01F09AF900283F
:102F900003D14FF40060FEF708FB01F0CEF90028E2
:102FA00003D14FF40060FEF700FB1E2000F0BAFFD3
:102FB00001F045FA002805D15FF000400021FEF73E
:102FC00031FB04E05FF000400021FEF7DFFA01F082
:102FD000F8F901F04FFA01BD10B504001E2000F011
:102FE000A1FF042801D101210CE0082801D1022110
:102FF00008E0072801D1032104E00A2801D10421B7
:1030000000E000212000C0B2002805D1DFF83C25F7
:1030100060204143505C8DE22000C0B2022807D1FD
:10302000DFF828256020414302EB0100807881E22F
:103030002000C0B2042807D1DFF8102560204143EA
:1030400002EB0100007975E22000C0B2062807D12A
:10305000DFF8F8246020414302EB0100807969E247
:103060002000C0B2082807D1DFF8E02460204143E7
:1030700002EB0100007A5DE22000C0B20A2807D10D
:10308000DFF8C8246020414302EB0100807A51E25E
:103090002000C0B20C2807D1DFF8B02460204143E3
:1030A00002EB0100007B45E22000C0B20E2807D1F0
:1030B000DFF898246020414302EB0100807B39E275
:1030C0002000C0B2102807D1DFF8802460204143DF
:1030D00002EB0100007C2DE22000C0B2122807D1D3
:1030E000DFF868246020414302EB0100807C21E28C
:1030F0002000C0B2142807D1DFF8502460204143DB
:1031000002EB0100007D15E22000C0B2162807D1B5
:10311000DFF838246020414302EB0100807D09E2A2
:103120002000C0B2182807D1DFF8202460204143D6
:1031300002EB0100007EFDE12000C0B21A2807D199
:10314000DFF808246020414302EB0100807EF1E1BA
:103150002000C0B21C2807D1DFF8F02360204143D3
:1031600002EB0100007FE5E12000C0B21E2807D17C
:10317000DFF8D8236020414302EB0100807FD9E1D2
:103180002000C0B2202808D1DFF8C02360204143CE
:1031900002EB010090F82000CCE12000C0B2222810
:1031A00008D1DFF8A8236020414302EB010090F82A
:1031B0002200BFE12000C0B2242808D1DFF88C2310
:1031C0006020414302EB010090F82400B2E12000AE
:1031D000C0B2262808D1DFF874236020414302EBF7
:1031E000010090F82600A5E12000C0B2282808D1EF
:1031F000DFF858236020414302EB010090F82800DB
:1032000098E12000C0B22A2808D1DFF840236020CE
:10321000414302EB010090F82A008BE12000C0B28C
:103220002C2808D1DFF824236020414302EB010061
:1032300090F82C007EE12000C0B22E2808D1DFF8E3
:103240000C236020414302EB010090F82E0071E155
:103250002000C0B2302807D1BC4A6020414302EBB5
:10326000010090F8300065E12000C0B2322807D19B
:10327000B64A6020414302EB010090F8320059E168
:103280002000C0B2342807D1B04A6020414302EB8D
:10329000010090F834004DE12000C0B2362807D17B
:1032A000AA4A6020414302EB010090F8360041E158
:1032B0002000C0B2382807D1A44A6020414302EB65
:1032C000010090F8380035E12000C0B2392807D15C
:1032D0009E4A6020414302EB010090F8390029E149
:1032E0002000C0B23A2807D1984A6020414302EB3F
:1032F000010090F83A001DE12000C0B23B2807D140
:10330000924A6020414302EB010090F83B0011E13A
:103310002000C0B23C2807D18C4A6020414302EB18
:10332000010090F83C0005E12000C0B23D2807D123
:10333000864A6020414302EB010090F83D00F9E02D
:103340002000C0B2402806D1804A6020414302EBF1
:103350000100006CEEE02000C0B2442806D17B4A98
:103360006020414302EB0100406CE3E02000C0B26A
:10337000482807D1754A6020414302EB010090F8CC
:103380004800D7E02000C0B2492807D16F4A60202A
:10339000414302EB010090F84900CBE02000C0B2AD
:1033A0004A2807D1694A6020414302EB010090F8A6
:1033B0004A00BFE02000C0B24B2807D1634A60201A
:1033C000414302EB010090F84B00B3E02000C0B293
:1033D0004D2807D15D4A6020414302EB010090F87F
:1033E0004D00A7E02000C0B24E2807D1574A602008
:1033F000414302EB010090F84E009BE02000C0B278
:103400004F2807D1514A6020414302EB010090F858
:103410004F008FE02000C0B2502807D14B4A6020F7
:10342000414302EB010090F8500083E02000C0B25D
:10343000512807D1454A6020414302EB010090F832
:10344000510077E02000C0B2522807D13F4A6020E7
:10345000414302EB010090F852006BE02000C0B243
:10346000532807D1394A6020414302EB010090F80C
:1034700053005FE02000C0B2542807D1334A6020D7
:10348000414302EB010090F8540053E02000C0B229
:10349000562807D12D4A6020414302EB010090F8E5
:1034A000560047E02000C0B2572807D1274A6020C5
:1034B000414302EB010090F857003BE02000C0B20E
:1034C000582807D1214A6020414302EB010090F8BF
:1034D00058002FE02000C0B2592807D11B4A6020B5
:1034E000414302EB010090F8590023E02000C0B2F4
:1034F0005C2807D1154A6020414302EB010090F897
:103500005C0017E02000C0B25D2807D10F4A6020A0
:10351000414302EB010090F85D000BE0E4B25E2C49
:1035200007D10A4A6020414302EB010090F85E0097
:1035300000E0002010BD0000702A0020742A002046
:10354000782A00207C2A00206826002064390200A6
:1035500070B505000C001E2000F0E4FC042801D129
:1035600001210CE0082801D1022108E0072801D13F
:10357000032104E00A2801D1042100E000212800F1
:10358000C0B200280DD1DFF8C40B6022DFF8C03BC9
:1035900002FB01F69E5D0670514319444978417063
:1035A000F8E32800C0B202280ED1DFF8A00B602299
:1035B000DFF89C3B02FB01F61E44B678867051434F
:1035C0001944C978C170E5E32800C0B204280ED1BF
:1035D000DFF8780B6022DFF8783B02FB01F61E442F
:1035E000367906715143194449794171D2E3280073
:1035F000C0B206280ED1DFF8540B6022DFF8503B32
:1036000002FB01F61E44B679867151431944C9790B
:10361000C171BFE32800C0B208280ED1DFF82C0B1F
:103620006022DFF82C3B02FB01F61E44367A06725C
:1036300051431944497A4172ACE32800C0B20A28C8
:103640000ED1DFF8080B6022DFF8043B02FB01F625
:103650001E44B67A867251431944C97AC17299E3FD
:103660002800C0B20C280ED1DFF8E00A6022DFF893
:10367000E03A02FB01F61E44367B067351431944BF
:10368000497B417386E32800C0B20E280ED1DFF8D3
:10369000BC0A6022DFF8B83A02FB01F61E44B67B92
:1036A000867351431944C97BC17373E32800C0B2C8
:1036B00010280ED1DFF8940A6022DFF8943A02FB5A
:1036C00001F61E44367C067451431944497C41740A
:1036D00060E32800C0B212280ED1DFF8700A602221
:1036E000DFF86C3A02FB01F61E44B67C8674514347
:1036F0001944C97CC1744DE32800C0B214280ED10E
:10370000DFF8480A6022DFF8483A02FB01F61E445F
:10371000367D067551431944497D41753AE32800C9
:10372000C0B216280ED1DFF8240A6022DFF8203A52
:1037300002FB01F61E44B67D867551431944C97DCE
:10374000C17527E32800C0B218280ED1DFF8FC09A4
:103750006022DFF8FC3902FB01F61E44367E067655
:1037600051431944497E417614E32800C0B21A2817
:103770000ED1DFF8D8096022DFF8D43902FB01F658
:103780001E44B67E867651431944C97EC17601E354
:103790002800C0B21C280ED1DFF8B0096022DFF883
:1037A000B03902FB01F61E44367F067751431944B7
:1037B000497F4177EEE22800C0B21E280AD1DFF827
:1037C00090296020414302EB0100807FDFF87C19E3
:1037D0008877DFE22800C0B2202812D1DFF86C0918
:1037E0006022DFF86C3902FB01F61E4496F8206077
:1037F00080F820605143194491F8211080F821107D
:10380000C8E22800C0B2222812D1DFF840096022A5
:10381000DFF83C3902FB01F61E4496F8226080F87E
:1038200022605143194491F8231080F82310B1E22B
:103830002800C0B2242812D1DFF810096022DFF876
:10384000103902FB01F61E4496F8246080F82460CB
:103850005143194491F8251080F825109AE2280068
:10386000C0B2262812D1DFF8E4086022DFF8E03881
:1038700002FB01F61E4496F8266080F8266051434C
:10388000194491F8271080F8271083E22800C0B26D
:10389000282812D1DFF8B4086022DFF8B43802FB20
:1038A00001F61E4496F8286080F8286051431944B8
:1038B00091F8291080F829106CE22800C0B22A285B
:1038C00012D1DFF888086022DFF8843802FB01F6A5
:1038D0001E4496F82A6080F82A605143194491F8F2
:1038E0002B1080F82B1055E22800C0B22C2812D1E2
:1038F000DFF858086022DFF8583802FB01F61E4452
:1039000096F82C6080F82C605143194491F82D10E2
:1039100080F82D103EE22800C0B22E2812D1DFF828
:103920002C086022DFF8283802FB01F61E4496F8C6
:103930002E6080F82E605143194491F82F1080F8C2
:103940002F1027E22800C0B2302812D1DFF8FC0780
:103950006022DFF8FC3702FB01F61E4496F8306067
:1039600080F830605143194491F8311080F83110DB
:1039700010E22800C0B2322812D1DFF8D00760224E
:10398000DFF8CC3702FB01F61E4496F8326080F86F
:1039900032605143194491F8331080F83310F9E143
:1039A0002800C0B2342812D1DFF8A0076022DFF867
:1039B000A03702FB01F61E4496F8346080F83460AC
:1039C0005143194491F8351080F83510E2E1280090
:1039D000C0B2362812D1DFF874076022DFF87037E2
:1039E00002FB01F61E4496F8366080F836605143BB
:1039F000194491F8371080F83710CBE12800C0B295
:103A000038280CD1DFF848276020414302EB010041
:103A100090F83800DFF8341781F83800BAE1280050
:103A2000C0B239280CD1DFF828276020414302EBCF
:103A3000010090F83900DFF8141781F83900A9E186
:103A40002800C0B23A280CD1DFF804276020414397
:103A500002EB010090F83A00DFF8F01681F83A0026
:103A600098E12800C0B23B280CD1DFF8E4266020A2
:103A7000414302EB010090F83B00DFF8D01681F8DB
:103A80003B0087E12800C0B23C280CD1DFF8C026FB
:103A90006020414302EB010090F83C00DFF8AC16D7
:103AA00081F83C0076E12800C0B23D280CD1DFF857
:103AB000A0266020414302EB010090F83D00DFF8B2
:103AC0008C1681F83D0065E12800C0B240280AD17B
:103AD000DFF87C266020414302EB0100006CDFF838
:103AE0006C16086456E12800C0B244280AD1DFF8F9
:103AF00060266020414302EB0100406CDFF84C1669
:103B0000486447E12800C0B248280CD1DFF84026BD
:103B10006020414302EB010090F84800DFF82C16CA
:103B200081F8480036E12800C0B249280CD1DFF8FE
:103B300020266020414302EB010090F84900DFF8A5
:103B40000C1681F8490025E12800C0B24A280CD1A2
:103B5000DFF8FC256020414302EB010090F84A00A9
:103B6000DFF8E81581F84A0014E12800C0B24B28BC
:103B70000CD1DFF8DC256020414302EB010090F816
:103B80004B00DFF8C81581F84B0003E12800C0B2F4
:103B90004D280CD1DFF8B8256020414302EB01002D
:103BA00090F84D00DFF8A41581F84D00F2E02800F0
:103BB000C0B24E280CD1DFF898256020414302EBBB
:103BC000010090F84E00DFF8841581F84E00E1E026
:103BD0002800C0B24F280CD1DFF874256020414383
:103BE00002EB010090F84F00DFF8601581F84F00FC
:103BF000D0E02800C0B250280CD1DFF85425602056
:103C0000414302EB010090F85000DFF8401581F8C5
:103C10005000BFE02800C0B251280CD1DFF8302599
:103C20006020414302EB010090F85100DFF81C15C1
:103C300081F85100AEE02800C0B252280CD1DFF864
:103C400010256020414302EB010090F85200DFF89C
:103C5000FC1481F852009DE02800C0B253280CD11A
:103C6000DFF8EC246020414302EB010090F85300A0
:103C7000DFF8D81481F853008CE02800C0B2542833
:103C800012D1DFF8C8046022DFF8C43402FB01F669
:103C90001E4496F8546080F854605143194491F8DA
:103CA000551080F8551075E02800C0B256280CD188
:103CB000DFF89C246020414302EB010090F856009D
:103CC000DFF8881481F8560064E02800C0B2572855
:103CD0000CD1DFF87C246020414302EB010090F816
:103CE0005700DFF8681481F8570053E02800C0B28D
:103CF00058280CD1DFF858246020414302EB010022
:103D000090F85800DFF8441481F8580042E0280089
:103D1000C0B259280CD1DFF838246020414302EBAF
:103D2000010090F85900DFF8241481F8590031E0BF
:103D30002800C0B25C280CD1DFF814246020414375
:103D400002EB010090F85C00DFF8001481F85C00E1
:103D500020E02800C0B25D280CD1DFF8F4236020F9
:103D6000414302EB010090F85D00DFF8E01381F8B9
:103D70005D000FE02800C0B25E280BD1DFF8D02331
:103D80006020414302EB010090F85E00DFF8BC13B5
:103D900081F85E002800C0B21F280EDA2021DFF86B
:103DA000AC03FEF755FBE4B2002C26D0DFF8340755
:103DB000016851F0020101601FE0EDB23F2D0EDA03
:103DC0002021DFF82407FEF743FBE4B2002C14D0D7
:103DD000DFF81007016851F0040101600DE02021B7
:103DE000DFF80807FEF734FBE4B2002C05D0DFF85B
:103DF000F406016851F00801016070BD38B50C008F
:103E0000092807D1DFF84403DFF8441360220CF0DF
:103E1000B7FC2DE0042807D1DFF83003DFF8D01617
:103E200060220CF0ADFC23E0082807D1DFF81C036A
:103E3000DFF8C01660220CF0A3FC19E0072806D1B9
:103E4000C248DFF8B41660220CF09AFC10E00A2891
:103E500006D1BE48DFF8A41660220CF091FC07E002
:103E6000BA4D2800BA4960220CF08AFC0020A877DD
:103E7000B64D20212800FEF7EBFA202115F1200095
:103E8000FEF7E6FA202115F14000FEF7E1FAE4B270
:103E9000002C0DD0DFF88C0B016851F0020101609D
:103EA000016851F004010160016851F008010160EE
:103EB00031BDA649496C0840704770B505000C003B
:103EC00002F068F8A14E706C0543756402F05EF86C
:103ED000202116F14000FEF7BBFAE4B2002C05D019
:103EE000DFF8400B016851F00801016070BD70B54A
:103EF00005000C0002F04EF8944E706C30EA050597
:103F0000756402F043F8202116F14000FEF7A0FA94
:103F1000E4B2002C05D0DFF80C0B016851F0080169
:103F2000016070BD0100C9B2442902D18748406CCC
:103F300009E00100C9B2402902D18448006C02E0C6
:103F40008249C0B2085C7047DFF8D80A007810F0E8
:103F50000E0F01D0012000E00020704710B50400D2
:103F60002820FFF7DFFF10F03F002100C9B2884290
:103F700001D1012078E02A20FFF7D4FF10F03F00A4
:103F80002100C9B2884201D101206DE02C20FFF749
:103F9000C9FF10F03F002100C9B2884201D10120C1
:103FA00062E02E20FFF7BEFF10F03F002100C9B2F3
:103FB000884201D1012057E02020FFF7B3FF10F025
:103FC0003F002100C9B2884201D101204CE02220EB
:103FD000FFF7A8FF10F03F002100C9B2884201D1CD
:103FE000012041E02420FFF79DFF10F03F00210059
:103FF000C9B2884201D1012036E02620FFF792FFA6
:1040000010F03F002100C9B2884201D101202BE00D
:104010003020FFF787FF10F03F002100C9B288422F
:1040200001D1012020E03220FFF77CFF10F03F009B
:104030002100C9B2884201D1012015E03420FFF7E8
:1040400071FF10F03F002100C9B2884201D1012068
:104050000AE03620FFF766FF10F03F00E4B2A0420E
:1040600001D1012000E0002010BD10B514000200B5
:10407000D2B2602A63DA0200D2B2382A0DDA020024
:10408000D2B21E2A09D0314A0300DBB2D154401CFF
:10409000C9430300DBB2D1541FE00200D2B2542A5C
:1040A00009D12A4A0300DBB2D154401CC9430300A2
:1040B000DBB2D15411E00200D2B2442A02D1234A29
:1040C00051640AE00200D2B2402A02D11F4A1164B0
:1040D00003E01E4A0300DBB2D1540100C9B21F291C
:1040E0000DDA20211948FEF7B3F9E4B2002C26D0EE
:1040F000DFF83009016851F0020101601FE0C0B231
:104100003F280EDA2021DFF8E003FEF7A1F9E4B240
:10411000002C14D0DFF80C09016851F00401016093
:104120000DE02021DFF8C403FEF792F9E4B2002C81
:1041300005D0DFF8F008016851F00801016010BDFA
:10414000DFF8BC230818105C7047000068260020C8
:104150006439020070B505000C002100280000F051
:10416000D1F900287AD0402C3CD1DFF8946328782C
:10417000315D884211D1687806EB040149788842A4
:104180000BD1A87806EB04018978884205D1E8783C
:1041900006EB0401C978884204D0002200210820DF
:1041A00004F0CFFB287C06EB0401097C88420BD18C
:1041B000687C06EB0401497C884205D1A87C06EBAB
:1041C0000401897C884204D000220021072004F0E9
:1041D000B8FB287D062803DB05202875FA206875C2
:1041E00000201CE0002CFBD1A87FDFF81413897F8E
:1041F0008842F5D0A87F092808D00A2806D00428CC
:1042000004D0082802D0072800D000200121FFF7A1
:10421000F5FD23E0295CBA4A0319D154401C1F283C
:10422000F8D32021B6482044FEF712F9002C06D11D
:10423000DFF8F007016851F0020101600EE0202C68
:1042400006D1DFF8E007016851F00401016005E0E4
:10425000DFF8D007016851F00801016070BD10B5AA
:10426000A74C20212000FEF7F3F8202114F12000B4
:10427000FEF7EEF8202114F14000FEF7E9F8DFF830
:10428000A407016851F002010160016851F00401C6
:104290000160016851F0080101605FF40010FDF752
:1042A0005AF910BDDFF87C07016851F08001016008
:1042B000016851F480710160016851F4007101607E
:1042C000704780B5DFF86007006800280DD1854889
:1042D0000068C0F3C010002807D120218848FEF7ED
:1042E000A1F8002801D1002026E0DFF8400700688F
:1042F00000280DD17B480068C0F30020002807D1BA
:1043000020217948FEF78EF8002801D1002013E023
:10431000DFF81C07006800280DD172480068C0F360
:104320004020002807D120217048FEF77BF80028A4
:1043300001D1002000E0012002BD80B55FF4001033
:10434000FDF76CF900283AD1DFF8DC060068002898
:104350000DD164480068C0F3C010002807D10021C7
:10436000674800F0CFF8002801D1002028E0DFF8EE
:10437000BC06006800280DD15A480068C0F3002030
:10438000002807D12021584800F0BCF8002801D1AE
:10439000002015E0DFF89806006800280DD151488C
:1043A0000068C0F34020002807D140214F4800F0AA
:1043B000A9F8002801D1002002E0012000E001203E
:1043C00002BD10B5474C2068C0F3C01000280ED0C5
:1043D00020234FF48072DFF85016494805F0DFF9CA
:1043E00001282BD1206830F08000206026E0206872
:1043F000C0F3002000280ED020234FF49072DFF885
:104400002C16394805F0CBF9012817D1206830F473
:104410008070206012E02068C0F3402000280DD09A
:1044200020234FF4A072DFF80816304805F0B7F9E2
:10443000012803D1206830F40070206010BD80B5E1
:10444000042801D101200CE0082801D1022008E055
:10445000072801D1032004E00A2801D1042000E04C
:104460000020C0B200F07DF8012801D1012000E059
:10447000002002BD10B51B4C2068C0F3400000288E
:104480000CD020224FF480711D4805F0C9F9012895
:1044900027D1206830F00200206022E02068C0F3BD
:1044A000800000280CD020224FF490710E4805F0B7
:1044B000B7F9012815D1206830F00400206010E021
:1044C0002068C0F3C00000280BD020224FF4A07158
:1044D000064805F0A5F9012803D1206830F008004E
:1044E000206010BD702A002088260020A826002009
:1044F000C4390200243A0200843A0200E43A02007D
:104500006826002010B40200012000290ED10024EA
:104510001D2C24D2115D02EB04035B7873F0FF03C2
:10452000DB43994200D00020A41CF1E720290ED1E2
:104530000024172C13D2115D02EB04035B7873F097
:10454000FF03DB43994200D00020A41CF1E7117D5A
:10455000527D72F0FF02D243914200D0002010BC85
:10456000704730B46021DFF8CC24DFF8CC341C78FD
:104570000500EDB24D43555DAC4201D000204FE245
:104580009C780500EDB24D431544AD78AC4201D0A6
:10459000002045E21C790500EDB24D4315442D790C
:1045A000AC4201D000203BE29C790500EDB24D43C6
:1045B0001544AD79AC4201D0002031E21C7A0500EF
:1045C000EDB24D4315442D7AAC4201D0002027E2D4
:1045D0009C7A0500EDB24D431544AD7AAC4201D052
:1045E00000201DE21C7B0500EDB24D4315442D7BE0
:1045F000AC4201D0002013E29C7B0500EDB24D439C
:104600001544AD7BAC4201D0002009E21C7C0500C2
:10461000EDB24D4315442D7CAC4201D00020FFE1AA
:104620009C7C0500EDB24D431544AD7CAC4201D0FD
:104630000020F5E11C7D0500EDB24D4315442D7DB4
:10464000AC4201D00020EBE19C7D0500EDB24D4372
:104650001544AD7DAC4201D00020E1E11C7E050097
:10466000EDB24D4315442D7EAC4201D00020D7E180
:104670009C7E0500EDB24D431544AD7EAC4201D0A9
:104680000020CDE11C7F0500EDB24D4315442D7F88
:10469000AC4201D00020C3E193F820400500EDB208
:1046A0004D43154495F82050AC4201D00020B7E1AD
:1046B00093F822400500EDB24D43154495F8225081
:1046C000AC4201D00020ABE193F824400500EDB2EC
:1046D0004D43154495F82450AC4201D000209FE191
:1046E00093F826400500EDB24D43154495F8265049
:1046F000AC4201D0002093E193F828400500EDB2D0
:104700004D43154495F82850AC4201D0002087E174
:1047100093F82A400500EDB24D43154495F82A5010
:10472000AC4201D000207BE193F82C400500EDB2B3
:104730004D43154495F82C50AC4201D000206FE158
:1047400093F82E400500EDB24D43154495F82E50D8
:10475000AC4201D0002063E193F830400500EDB297
:104760004D43154495F83050AC4201D0002057E13C
:1047700093F832400500EDB24D43154495F83250A0
:10478000AC4201D000204BE193F834400500EDB27B
:104790004D43154495F83450AC4201D000203FE120
:1047A00093F836400500EDB24D43154495F8365068
:1047B000AC4201D0002033E193F838400500EDB25F
:1047C0004D43154495F83850AC4201D0002027E104
:1047D00093F839400500EDB24D43154495F8395032
:1047E000AC4201D000201BE193F83A400500EDB245
:1047F0004D43154495F83A50AC4201D000200FE1EA
:1048000093F83B400500EDB24D43154495F83B50FD
:10481000AC4201D0002003E193F83C400500EDB22A
:104820004D43154495F83C50AC4201D00020F7E0D0
:1048300093F83D400500EDB24D43154495F83D50C9
:10484000AC4201D00020EBE01C6C0500EDB24D4302
:1048500015442D6CAC4201D00020E1E05C6C0500F9
:10486000EDB24D4315446D6CAC4201D00020D7E051
:1048700093F848400500EDB24D43154495F8485073
:10488000AC4201D00020CBE093F849400500EDB2E6
:104890004D43154495F84950AC4201D00020BFE08B
:1048A00093F84A400500EDB24D43154495F84A503F
:1048B000AC4201D00020B3E093F84B400500EDB2CC
:1048C0004D43154495F84B50AC4201D00020A7E071
:1048D00093F84D400500EDB24D43154495F84D5009
:1048E000AC4201D000209BE093F84E400500EDB2B1
:1048F0004D43154495F84E50AC4201D000208FE056
:1049000093F84F400500EDB24D43154495F84F50D4
:10491000AC4201D0002083E093F850400500EDB296
:104920004D43154495F85050AC4201D0002077E03B
:1049300093F851400500EDB24D43154495F85150A0
:10494000AC4201D000206BE093F852400500EDB27C
:104950004D43154495F85250AC4201D000205FE021
:1049600093F854400500EDB24D43154495F854506A
:10497000AC4201D0002053E093F856400500EDB260
:104980004D43154495F85650AC4201D0002047E005
:1049900093F857400500EDB24D43154495F8575034
:1049A000AC4201D000203BE093F858400500EDB246
:1049B0004D43154495F85850AC4201D000202FE0EB
:1049C00093F859400500EDB24D43154495F8595000
:1049D000AC4201D0002023E093F85C400500EDB22A
:1049E0004D43154495F85C50AC4201D0002017E0CF
:1049F00093F85D400500EDB24D43154495F85D50C8
:104A0000AC4201D000200BE093F85E30C0B24843C6
:104A1000104490F85E00834201D0002000E00120A5
:104A200030BC7047702A0020742A0020782A0020A9
:104A30007C2A0020643902006826002070B5784C7A
:104A4000784E204601F0F8F8204601F00FF9764C38
:104A500010212046FBF794FA20212046FBF790FA1C
:104A600008212046FBF78CFA40212046FBF788FA04
:104A70006E48FBF7E1FA40212046FBF7C5FA10210A
:104A80002046FBF7B7FA20212046FBF7B3FA684926
:104A90004FF4722008600D464FF0FF320021284687
:104AA0000BF09FFE28460BF097FE6248FBF7C4FA16
:104AB0006148FBF7C1FA304601F0BEF8304601F01C
:104AC000D5F85E4E304601F0B7F8304601F0CEF82A
:104AD0005B4E5C493046FCF74AF940F20442FF2144
:104AE0003046FCF777F94FF0FF32FF213046FCF7F4
:104AF00087F9554A4FF47F413046FCF781F904218C
:104B00003046FCF799F94FF480713046FCF794F980
:104B10002021762001F045FA4021772001F041FA6A
:104B2000762001F04FFA772001F04CFA4FF6FF7132
:104B30003046FCF70DF9012208212046FBF756F913
:104B4000424C0120606001F025FA002128460BF05C
:104B500053FE01F01BFA0120206070BD30B581B01A
:104B600001F018FA39484168012905D101F00EFA1F
:104B70004FF0FF3001B030BD8468C568344801682B
:104B80000C1B01F003FAA54238BF2546314AA5FBAC
:104B90000220800901B030BD2C49086800281CBFE4
:104BA00023480BF026BE704710B5044601F0F2F919
:104BB00021461F480BF020FEBDE8104001F0E6B989
:104BC00070B52549214E254D042008604C6A706857
:104BD00030B92A68100712D5B268A21AF26004E050
:104BE0004FF0FF30F0600022726000230B634FF43F
:104BF00080711348FCF725F9B4600820A86070BDE7
:104C000000B581B04FF480710D48FCF71AF90F48D8
:104C100001214160082212490A6001B000BD000074
:104C2000004400F0000400F000F005400718070001
:104C300000C002400510070005140700045C00F0E6
:104C400000E004401732000400D430006429002042
:104C500050E00440CDCCCCCC24E0044014F405401A
:104C60001CF4054070B5DFF8804A20684008400019
:104C70002060206830F004002060DFF8705A2021A6
:104C80002800FBF787F910212800FBF783F9402162
:104C90002800FBF77FF980212800FBF77BF9002033
:104CA000DFF84C1A08600020DFF8301B0860002095
:104CB000DFF82C1B08600020DFF8281B0860DFF8F5
:104CC000286B04213000FBF765F9082366220421D4
:104CD0003000FBF7B1F80020DFF8101B086002215C
:104CE0003000FBF757F90823662202213000FBF75A
:104CF000A3F80220DFF82C1B086001213000FBF72D
:104D00003FF9DFF8246B04213000FBF743F9082357
:104D1000662204213000FBF78FF80020DFF80C1B1F
:104D2000086002213000FBF735F9082366220221D2
:104D30003000FBF781F80220DFF8F41A0860012147
:104D40003000FBF71DF9DFF8EC6A02213000FBF7B9
:104D500017F90A23012202213000FBF76DF8042124
:104D60003000FBF70DF90A23012204213000FBF784
:104D700063F808213000FBF703F90A230122082118
:104D80003000FBF759F8DFF8B06A04213000FBF778
:104D9000F7F80A23012204213000FBF74DF8DFF871
:104DA0009C6A01213000FBF7EBF802213000FBF791
:104DB000E7F82021DFF8880AFBF7E2F8DFF8846AD9
:104DC00002213000FBF7DCF80A2301220221300027
:104DD000FBF732F801213000FBF7D2F80A23012259
:104DE00001213000FBF728F801212800FBF7C8F863
:104DF0000A23012201212800FBF71EF8DFF8485A98
:104E000001212800FBF7BCF80A2301220121280018
:104E1000FBF712F8DFF8345A80212800FBF7B0F8CE
:104E20000A23012280212800FBF706F840212800F0
:104E3000FBF7A6F80A23012240212800FAF7FCFF1D
:104E4000FBF762F90A38DFF8381B0860FBF75CF9FA
:104E5000DFF8301B08605FF07060DFF82C1B086023
:104E6000206850F00100206070BD70B5DFF8780850
:104E70000078C00727D5DFF8E84B2568FBF744F931
:104E8000DFF8FC6A3168401A0A2806D300F041F8BE
:104E9000FBF73AF9306000F0C0F8DFF8F01A20684C
:104EA000684008600A68206802400A60DFF8B41BA6
:104EB000206845400D600A68206882430A6000F05F
:104EC000CDF800F08DFB70BDDFF81C08016851F0D3
:104ED000040101607047DFF8881B096808407047CB
:104EE000DFF8A81A096808407047DFF87C1B0968DA
:104EF00008407047DFF8741B096808407047DFF806
:104F0000701B096808407047DFF8681B0968084093
:104F1000704710B5DFF8604B00F0F7FA207000F032
:104F200015FB60700024FCF760FD01285CD10120B6
:104F300000F0E0FB012801D154F00104082000F04A
:104F4000D9FB012801D154F008044FF4807000F01F
:104F5000D1FB012801D154F480744FF4007000F0AB
:104F6000C9FB012801D154F40074102000F0C2FBE9
:104F7000012801D154F01004202000F0BBFB0128CF
:104F800001D154F02004402000F0B4FB012801D1ED
:104F900054F04004802000F0ADFB012801D154F012
:104FA00080043B20FEF7BEFF002806D0DFF8CC0AC5
:104FB0000068002801D154F480643B20FEF7B2FF62
:104FC000022806D1DFF8B80A0068002801D154F49D
:104FD0000064DFF8B00A0068002801D054F480446F
:104FE000DFF8A40A046002E0DFF89C0A04684D20A0
:104FF000FEF798FF002806D0DFF8900A0068002826
:1050000001D054F4004400F0F3FB0443200000F00E
:10501000BDFADFF84C1A086010BD80B5DFF8581AE9
:10502000087810F03F00497871F03F01C943884289
:105030000ED0FBF769F8DFF8581A0968401A40F2F9
:105040002D11884209D35FF40000FCF7AEFA04E0AA
:10505000FBF75AF8DFF8381A086001BD2DE9F04176
:10506000DFF8044A2568DFF880160868C0F380007E
:10507000002808D00020DFF8F4291060086830F01C
:105080000400086005E0DFF8E409016811F0604100
:105090000160052000F0DCFB012805D1DFF8CC0918
:1050A000016851F001010160182000F0D1FB0128D6
:1050B00005D1DFF8B809016851F40061016007F01B
:1050C00061F9022807D1DFF89809006810F0E04084
:1050D000B0F1005F04D0FBF717F8DFF8B8190860EB
:1050E000042000F0B5FB012808D0FBF70DF8DFF82D
:1050F000A4190968401AB0F5FA7F05D3DFF86C09E6
:10510000016851F002010160072000F0A1FB0128B5
:1051100005D1DFF85809016851F004010160092048
:1051200000F096FB012809D01E2000F091FB012819
:1051300004D01F2000F08CFB012805D1DFF82C09DA
:10514000016851F008010160022000F081FB012894
:1051500009D0202000F07CFB012804D0212000F0A1
:1051600077FB012805D1DFF80409016851F010012F
:105170000160062000F06CFB012805D1DFF8EC0887
:10518000016851F02001016006F051FD002810D1A6
:10519000082000F05DFB012805D0DFF8C408006896
:1051A00010F4406F05D0DFF8C408016851F4807135
:1051B000016006F03CFD00280AD10E2000F048FBFB
:1051C000012805D1DFF8A408016851F400710160DD
:1051D00006F02DFD002812D11A2000F039FB01281D
:1051E0000DD1DFF88808016851F400710160016891
:1051F00051F480710160016851F4000101600B20DD
:1052000000F026FB012804D0DFF8540800684004B1
:1052100005D5DFF85808016851F0400101600A2007
:1052200000F016FB012805D1DFF84008016851F0B5
:1052300000410160152000F00BFB012805D1DFF8CB
:105240002C08016851F480010160142000F000FB7B
:10525000012805D1DFF81408016851F00051016000
:10526000132000F0F5FA012805D1DFF800080168E5
:1052700051F080010160122000F0EAFA012805D106
:10528000DFF8E807016851F080410160192000F063
:10529000DFFA01282AD1FAF737FFDFF8EC160860A9
:1052A0005320FEF73FFEC0F303164FF47A704643D7
:1052B000FAF72AFFDFF8CC160968401A86420AD3AB
:1052C000DFF8A807016851F4800101600120DFF8D0
:1052D000C817086030E0DFF89407016851F48011C6
:1052E00001600020DFF8B017086025E0FAF70CFF36
:1052F000DFF8901608605320FEF714FE060016F043
:105300000F064FF47A704643FAF7FEFEDFF8781680
:105310000968401A86420BD3DFF87C070068002832
:105320000AD1DFF84807016851F48011016003E0F9
:105330000020DFF8641708600C2000F089FA0128CB
:1053400005D1DFF82807016851F480610160112060
:1053500000F07EFA012805D1DFF81007016851F44A
:1053600080210160102000F073FA012805D1DFF8D8
:10537000FC06016851F400310160012000F068FA78
:10538000012805D1DFF8E406016851F4803101609D
:105390000D2000F05DFA012805D1DFF8D006016884
:1053A00051F400510160032000F052FA012805D1A8
:1053B000DFF8B806016851F4004101600F2000F0E9
:1053C00047FA012805D1DFF8A406016851F48041AD
:1053D0000160162000F03CFA012805D1DFF88C06A8
:1053E000016851F4805101601B2000F031FA01285E
:1053F00005D1DFF87806016851F4001101604FF41F
:105400000070FCF70BF9002808D04FF48040002111
:10541000FCF717F900290CD100280AD1172000F059
:1054200017FA012805D1DFF84406016851F400217C
:105430000160DFF86876DFF83486D8F8000038427B
:1054400004D008200021FCF7EDF803E0082000213B
:10545000FCF79CF8D8F8000000F09AFA06004FF428
:1054600080400021FCF7EDF8002901D100280DD083
:105470005FF080400021FCF7E4F8002901D100280A
:1054800004D0D8F800000740C8F80070D8F8000031
:105490003043C8F800004FF40070FCF7BFF8002854
:1054A0000BD04FF480400021FCF7CBF8002901D14C
:1054B000002802D00020C8F80000D8F800000AF048
:1054C000F9FC206020680AF056FA2060DFF8A01589
:1054D0002068684008600A68206802400A60DFF8B7
:1054E0009425206845401560136820688343136045
:1054F0000868000301D5FAF72AFE206830EA06069C
:10550000300000F0A4F8BDE8F08138B50024DFF8E1
:10551000145300202860072000F0CAFB02202860F6
:1055200000210FE0B14A00201060640064086400AC
:10553000DFF86C050068002801D054F00104042055
:105540001060491C0829EDD3200032BD38B5002475
:10555000B74D00202860072000F0AAFB0220286039
:1055600000210FE0B14A002010606400640864006C
:10557000DFF830050068002801D054F00104042051
:105580001060491C0829EDD3200032BD30B4020060
:105590001000002305E0DFF8101551F82310084330
:1055A0005B1C032BF7D3DFF80055E96808401300B4
:1055B000002403E055F824100B40641C032CF9D39D
:1055C0001843E860022106E005EB810353F8043C30
:1055D00045F82130491E0029F6D12A6030BC7047B9
:1055E00010B5DFF87C040068002811D5FAF78CFDAF
:1055F000DFF8B8140968401A41F28831884201D3B3
:10560000FBF7B2F93848016851F0080101601DE06C
:10561000354C2068C0F3C000002812D0FAF774FDA2
:10562000DFF888140968401A40F2D171884203D229
:1056300003F0B7FBFAF78BFD206830F0080020601C
:1056400004E0FAF761FDDFF86414086010BD10B5DE
:1056500004004FF480400021FBF7F3FF002901D143
:10566000002812D04FF40070FBF7D8FF00280CD0B0
:1056700000205B4908600020584908600020594913
:10568000086000201A4908602BE0A00503D510200F
:105690005349086002E0002051490860E00503D545
:1056A00020204E49086002E000204C490860082094
:1056B0000021FBF7C6FF002901D1002803D04020BC
:1056C0004849086002E0002046490860DFF8E0032E
:1056D000044203D080200649086002E0002004490B
:1056E000086010BD00000000482B002000D00340DF
:1056F00000D2034038B5012806D12025DFF8780311
:10570000047814F001044EE0022806D12225DFF8C7
:105710006803047814F0020445E0042806D1242527
:10572000DFF85403047814F004043CE0082806D1A0
:105730002625DFF84403047814F0080433E0B0F5BC
:10574000807F06D13025DFF83003047814F0400460
:1057500029E0B0F5007F07D13225DFF81C0344783B
:10576000E44314F040041EE0102804D12825DFF89B
:105770004403046817E0202804D12A25DFF8380301
:10578000046810E0402804D12C25DFF830030468B9
:1057900009E02E25DFF828130C68802803D05FF479
:1057A0000000FBF712FF2800C0B2FEF7BBFB10F0B1
:1057B0003F0F11D02800C0B2FEF7B4FB000605D49D
:1057C000002C01D0012008E0002006E0002C01D1CF
:1057D000012002E0002000E0002032BD80D0034024
:1057E00040D0034000D103400060024010600240FE
:1057F0000020B4490968002901D150F00050B24995
:105800000968002901D150F08040B0490968002999
:1058100001D150F00040AE490968002901D150F093
:10582000805070470860024000300640103006404B
:1058300008300640001006400040064000F00540D9
:1058400000C00540002006400050004000500240CB
:1058500038B50400824D2878C00609D52820FEF707
:1058600061FB10F03F002100C9B2884200F0838044
:105870002878800608D52A20FEF754FB10F03F0058
:105880002100C9B2884276D02878400608D52C205D
:10589000FEF748FB10F03F002100C9B288426AD0F1
:1058A0002878000608D52E20FEF73CFB10F03F00BC
:1058B0002100C9B288425ED02878C00708D52020D0
:1058C000FEF730FB10F03F002100C9B2884252D0F1
:1058D0002878800708D52220FEF724FB10F03F002F
:1058E0002100C9B2884246D02878400708D5242034
:1058F000FEF718FB10F03F002100C9B288423AD0F1
:105900002878000708D52620FEF70CFB10F03F0092
:105910002100C9B288422ED02868C00408D534209E
:10592000FEF700FB10F03F002100C9B2884222D0F0
:105930002868800408D53620FEF7F4FA10F03F00FE
:105940002100C9B2884216D02868C00508D5302089
:10595000FEF7E8FA10F03F002100C9B288420AD0F1
:105960002868800509D53220FEF7DCFA10F03F00E8
:10597000E4B2A04201D1012000E0002032BD0000CD
:105980006C2B0020702B0020742B0020502B00204B
:1059900010B504004FF480400021FBF752FE0029AF
:1059A00001D1002804D04E20FEF7BCFAC00706D46F
:1059B00000245FF000500021FBF7E8FD4DE0374880
:1059C000044208D05FF080400021FBF73AFE002936
:1059D00001D1002804D01A2000F063FC012801D175
:1059E00000243AE0142000F05CFC012804D14E2091
:1059F000FEF798FA400712D4142000F052FC002859
:105A000004D14E20FEF78EFA800708D45FF0804064
:105A10000021FBF716FE002901D100281CD05FF001
:105A200000500021FBF7FEFD142000F03AFC012895
:105A300004D14E20FEF776FA400609D4142000F077
:105A400030FC002806D14E20FEF76CFA000601D586
:105A5000802402E0402400E00024200010BD00006B
:105A60004C2B0020542B0020582B00205C2B0020B6
:105A7000602B0020642B0020D42D002004F0054072
:105A800008F0054000520240782B002000510240EF
:105A9000682B00207C2B0020802B0020C00050E0D1
:105AA000046002400430064074290020842B00204A
:105AB0003F080080081006401010064020100640E5
:105AC00010400640082006400420064004500040D4
:105AD00004D0034010B401000022002000230EE097
:105AE000401E0BE0400014000A00920F12EB8402EB
:105AF0008900401C8242F3D3121A401C5B1C102BFD
:105B0000F0D3400810BC7047401801686FF3520191
:105B10001143016000F124012030920704D5B02226
:105B200002604FF4306003E08C22026040F60C000B
:105B300008607047401800F11001006883074CBFEF
:105B40005208521E0A607047081801681AE010B522
:105B50008B0900EB831003689C0700F1100348BF1A
:105B600052081B689A1AC9074CBF1C3018300260D3
:105B700010BD401800F12C010A6000F130010B60EB
:105B800050F8281F41F001010160704740F8041FE0
:105B900070470830012A02680CBF114322EA010154
:105BA000016070470C30012A02680CBF114322EAE1
:105BB0000101016070472430012A02680CBF1143C3
:105BC00022EA0101016070471030012A02680CBF0F
:105BD000114322EA010101607047081850F8041FC0
:105BE0000A4302607047081850F8041F21EA0202B5
:105BF0000260704718B58100DFF8C422C0F30723A4
:105C000001F47F71D31841EA431343F08443012424
:105C10001C600023009302E0009C641C0094009B25
:105C2000102BF9D3C0F30720121841EA421141F0BA
:105C300084410020086011BDC0F30722DFF8841200
:105C400080008A1800F47F7040EA421040F08440DF
:105C500001210160704780008A1800F47F7040EADB
:105C6000421040F08440002101607047C0F30722D9
:105C7000DFF85412EFE7C0F30722DFF85012DFE736
:105C8000C0F30722DFF84412E5E7DFF8441208B159
:105C90008868704708687047DFF838020068704706
:105CA000DFF830120A6822EA00000860704700003E
:105CB0000138FDD170477047DFF81C12086070474B
:105CC00070B5DFF80C221369146A014623F48003CF
:105CD00001F0010543F4006303F0010085F00105C4
:105CE00044F400641361284214620ED061F0010094
:105CF00003404FF48070906013614FF400201568EA
:105D0000EE054AD4401EFAD170BD080960F30A13AB
:105D1000DFF8D40113610440DFF8D00108400443E8
:105D2000C80000F0400004431462480B60F34D3398
:105D300060F34D3440209060002C47BF1462136123
:105D400013611462DFF8A8010340DFF8A8010840DE
:105D50000343C80D60F3DC54480008D5DFF8980110
:105D600024F48004084043F48003044301E024F059
:105D7000804408050BD44FF4004060490D68EE07DD
:105D800001D4401EFAD123F4006324F400641361AB
:105D900014621020BDE870408AE70028B5D170BDBC
:105DA000F0B557490A6D0B6E002B4CBF03F0700025
:105DB00002F0300040B1102847D0202847D03028CA
:105DC00047D0702848D04AE00FF25410C2F3841430
:105DD00050F824504B4C04EA0306B6F1004F4FF044
:105DE000FF3003D0002B41D416053FD43C4E37681A
:105DF00076680968C6F3042C06F01F060CF1010C46
:105E0000761C16FB0CF67600B5FBF6F5C7F3090613
:105E1000C7F389276F4301F47041BF0AB1F5005FF2
:105E200006FB057542F480020DD0B1F5405F18D035
:105E3000B1F5804F17D0B1F5E04F16D0B1F5104F46
:105E400008BF314812E0314810E0244DC2E7304D20
:105E5000C0E747F23055BDE74FF40045BAE70020F0
:105E6000F0BD2C4802E02C4800E01E48510217D536
:105E7000002B10D559000BD51C40B4F1004F03D0B6
:105E8000002B05D4110503D46D00C3F3865104E043
:105E9000C3F3C55101E0C2F3C351491CB5FBF1F591
:105EA000A84288BF2846F0BD1C4901230A6800F0BB
:105EB0000F0003FA00F000E00A6810430860704722
:105EC00000E50F4000E60F4000E70F4000E80F40FC
:105ED00050E00F405CE00F407CE00F400024F400F5
:105EE00060E10F4040787D018FFFFF7F3000008030
:105EF000FEFF3FF80100C0070000404068E10F408E
:105F000010E00F4000080080002D310100B4C404EF
:105F100000093D0080F0FA02005A62026CE00F4076
:105F200040420F0000201C0080841E0000802500DD
:105F3000999E36000040380000093D0000803E0078
:105F400000004B00404B4C0000204E00808D5B0059
:105F500000C05D000080700000127A0000007D002B
:105F600080969800001BB7000080BB00C0E8CE0000
:105F7000647ADA000024F4000000FA0080A812011C
:105F8000002D310100366E0140787D0180B50AF0A8
:105F90003BFC02E080B50AF033FC00B10120C0B246
:105FA00002BD10B50FF2D402830852F82320136803
:105FB000C00000F01800FF248440A343814019432F
:105FC000116010BD04282B4903D1086840F48030CB
:105FD0000BE0052804D10A6842F400320A607047D9
:105FE000062804D1086840F48020086070470F2814
:105FF00005D12148016841F00201016070470CD9C8
:106000000FF21413A0F110011038400953F82000CA
:10601000012201F01F018A400260704704281549DF
:1060200003D1086820F480300BE0052804D10A6809
:1060300022F400320A607047062804D1086820F470
:106040008020086070470F2805D10B48016821F0B7
:106050000201016070470CD90FF2D003A0F11001CA
:106060001038400953F82000012201F01F018A4036
:106070000260704724ED00E010E000E00000000046
:1060800018ED00E01CED00E020ED00E000E400E091
:1060900004E400E008E400E00CE400E010E400E0C8
:1060A00014E400E018E400E01CE400E020E400E078
:1060B00024E400E028E400E02CE400E030E400E028
:1060C00034E400E038E400E03CE400E040E400E0D8
:1060D00044E400E048E400E04CE400E050E400E088
:1060E00054E400E058E400E05CE400E060E400E038
:1060F00064E400E068E400E06CE400E070E400E0E8
:1061000074E400E078E400E07CE400E080E400E097
:1061100084E400E088E400E000E100E004E100E065
:1061200008E100E00CE100E010E100E080E100E0C7
:1061300084E100E088E100E08CE100E090E100E033
:106140007CB5DFF8F44600202060FAF717F8002845
:106150000DD15FF08070FBF728FA0020DFF8DC1625
:1061600008605FF0FF30DFF8D816086026E000F026
:10617000A2FC10F0210FFAD1DFF8C056002000F089
:10618000ABFA2860DFF8B866012000F0A5FA3060AD
:1061900028683168C943884210D0002028605FF029
:1061A000FF3030603068297801F0FF0151EA0021AA
:1061B000009104220421684600F018FC5FF0FF30D3
:1061C000DFF880160860DFF8801608600120206084
:1061D00073BD70B5DFF860060068012855D1DFF89F
:1061E0006066DFF8584620683168C943884206D0A7
:1061F00000F0B8F95FF08070FBF7D7F945E0206850
:1062000000F0E9F905001E20FDF78CFE062802D1FA
:1062100035F050050BE01E20FDF784FE072804D062
:106220001E20FDF77FFE0A2801D135F00405206805
:1062300085420DD02560ED433560206800F00AFBF3
:106240000100DFF808060278C9B2032002F079FBEA
:10625000F9F794FF002804D15FF08070FBF7A5F9EF
:1062600013E000F028FC10F0210F0ED1002000F008
:1062700033FA2168884208D03168207800F0FF00A6
:1062800050EA0120042100F0FDFB70BDDFF8B005ED
:106290000168DFF8A805007800F0FF0050EA01204F
:1062A0007047C0B2002800F00581022800F02C8160
:1062B000C0F01F81042800F03D81C0F03081062825
:1062C00000F00181C0F04181082800F0DD80C0F0BD
:1062D00005810A2820D0C0F0E2800C285CD02FD3A2
:1062E0000E2838D042D310284BD060D3122869D062
:1062F00073D3142800F0878017D3162800F09980F4
:10630000C0F08C80182800F0A980C0F09D801A2869
:106310006ED0C0F0AE8023E1DFF820050078800762
:1063200001D5012000E000201BE1DFF81005007816
:1063300010F04300402801D1012000E0002010E1CE
:10634000DFF8F804007810F05F00402801D1012048
:1063500000E0002005E1DFF8E404007810F05F00C1
:10636000442801D1012000E00020FAE0DFF8CC044D
:10637000007810F05F00502801D1012000E00020DB
:10638000EFE0DFF8B804007810F05F00542801D186
:10639000012000E00020E4E0DFF8A004007810F025
:1063A0005F00482801D1012000E00020D9E0DFF89B
:1063B0008C04007810F05F004C2801D1012000E02F
:1063C0000020CEE0DFF87404007810F05F001C2895
:1063D00001D1012000E00020C3E0DFF86004007874
:1063E00010F05F00182801D1012000E00020B8E083
:1063F000DFF84804007810F05B00182801D1012074
:1064000000E00020ADE0DFF83404007810F0030075
:10641000012801D1012000E00020A2E0DFF81C04E7
:10642000007810F06300202801D1012000E0002056
:1064300097E0DFF80804007810F00600042801D186
:10644000012000E000208CE0DFF8F003007810F07D
:106450003B0F01D1012000E0002082E0DFF8DC03E7
:10646000007810F03B00082801D1012000E0002056
:1064700077E0DFF8C803007810F03B00102801D166
:10648000012000E000206CE0DFF8B003007810F09D
:106490000700012801D1012000E0002061E0DFF8C1
:1064A0009C03007810F00700052801D1012000E0CE
:1064B000002056E0DFF884030068002801D10120A5
:1064C00000E000204DE0DFF87403007810F07F005A
:1064D000202801D1012000E0002042E0DFF85C0329
:1064E000007810F07F00242801D1012000E0002076
:1064F00037E0DFF84803007810F07F00042801D16E
:10650000012000E000202CE0DFF83003007810F0DC
:106510007F00082801D1012000E0002021E0DFF801
:106520001C03007810F07F000C2801D1012000E04E
:10653000002016E0DFF80403007810F07F00102838
:1065400001D1012000E000200BE0DFF8F00200782C
:1065500010F07F00142801D1012000E0002000E0AD
:106560000020704738B5DFF8D44200202060DFF803
:10657000D0522068C043286000F09DFA10F0210F2F
:106580000CD1F9F7FBFD012808D12968207800F02B
:10659000FF0050EA0120042100F074FA31BD10F030
:1065A0007F00A84908600868A4490968884203D0A8
:1065B0005FF0FF30A4490860704710F07F00A249E7
:1065C000086008689D490968884203D05FF0FF3081
:1065D0009C490860704738B5040000F0A0F8050039
:1065E00003F030FC01281BD115F1010F01D0A807E1
:1065F00016D49448016811F1010F02D00078800789
:106600000ED49148016811F1010F02D00078800783
:1066100006D403F036FC040005208C49087053E0D2
:1066200002F03EFD012820D102F066FD10F1010FBD
:106630001BD015F1010F01D0A80716D481480168BD
:1066400011F1010F02D0007880070ED47E48016856
:1066500011F1010F02D00078800706D402F04CFD42
:1066600004000320794908702EE015F1010F18D0BD
:106670007448016811F1010F02D00078800710D42E
:106680007148016811F1010F02D00078800708D429
:10669000A54202D06E4804602C0001206B490870AE
:1066A00012E06848016811F1010F04D0046802206B
:1066B0006649087008E06448016811F1010F03D0D1
:1066C00004680420614908705FF0FF305E4908608B
:1066D0005C490860200032BD1CB5040000F0EBF9F5
:1066E00010F0210F11D104220421684600F069F94D
:1066F000002C04D1009800F0FF0000900DE00098FD
:10670000000A70F0FF00009007E0002C02D100208A
:10671000009002E05FF0FF300090009816BD10B5C9
:106720005FF0FF345FF48020FEF7DFFB002801D02C
:1067300002247EE05FF48020FEF7E6FB002802D012
:106740004348046875E05FF40030FEF7CEFB002894
:1067500001D001246DE05FF40030FEF7D5FB002886
:1067600002D03B48046864E04FF48050FEF7BDFB64
:10677000002801D040245CE04FF48050FEF7C4FBB9
:10678000002802D03248046853E05FF48030FEF7FE
:10679000ACFB002801D020244BE05FF48030FEF7F2
:1067A000B3FB002802D02A48046842E04FF40040BE
:1067B000FEF79BFB002801D008243AE04FF400408C
:1067C000FEF7A2FB002802D02148046831E04FF414
:1067D0008040FEF78AFB002801D0102429E04FF406
:1067E0008040FEF791FB002802D01948046820E0A1
:1067F0004FF40050FEF779FB002801D0042418E084
:106800004FF40050FEF780FB002802D010480468C7
:106810000FE05FF40010FEF768FB002801D0182499
:1068200007E05FF40010FEF76FFB002801D0084876
:106830000468200010BD0000102C0020042C002053
:10684000082C0020182C0020142C0020E52D0020FE
:106850000C2C0020810701D50A2046E0C10705D590
:10686000400701D5092040E008203EE0410615D54B
:10687000010705D5400701D50F2036E00C2034E094
:10688000C10605D5400701D510202EE00D202CE0D3
:10689000400701D50E2028E00B2026E0810605D513
:1068A000400701D5072020E006201EE010F0180167
:1068B000182905D1400701D5122016E0112014E057
:1068C000010705D5400701D503200EE002200CE0AA
:1068D000C10605D5400701D5052006E0052004E0E6
:1068E000400701D5012000E00020C0B2704730B45D
:1068F000002513E050F8042BD30744BFA9F101038E
:106900009A18091F042942F8045BFAD213468C072F
:1069100044BF15809B1CC90748BF1D7050F8041B5D
:106920000029E7D130BC704738B5044600F029F89B
:10693000624D0321296000F024F80120E40900FAE7
:1069400004F45F48E443046000F01BF80020286072
:106950000A20BDE83240FFF7ABB910B500F011F8DE
:10696000564C0321216000F00CF8554900200860C6
:1069700000F007F8002020600A20BDE81040FFF773
:1069800097B90A20FFF794B910B50220FFF790F9E4
:106990004C4C2168C807FCD4606810F00C0F0CD177
:1069A0004948FFF727F90220FFF782F92068C1075D
:1069B000FCD4606810F00C0F01D0022010BD002044
:1069C00010BD10B5414B8C091C60C1F383019208C6
:1069D00059600AD004E0596811B91C68641C1C6035
:1069E000521E196940F8041BF5D110BD2DE9F84F6E
:1069F00081468A46354D6869C007FCD4DFF8D080EF
:106A0000344F354E4FEA9A1028609408CAF3830039
:106A1000686005D12AE0686810B92968491C2960B6
:106A200030683840404505D13068010404BF504605
:106A3000FFF77AFFD9F800002861FFF7A2FFD5F829
:106A400014B05FEACB70FAD45FEACB600AD5306845
:106A50000740474504D13068010408BFFFF77DFFB8
:106A600058460DE0641E09F10409D4D1306807408E
:106A7000474504D13068010408BFFFF76EFF68691D
:106A8000BDE8F28F38B50D461349114B0A6804462C
:106A9000104802409A4205D10968080404BF2846FC
:106AA000FFF742FF0948A9090160C5F3830141606E
:106AB0000461406932BD034800687047FCD00F4054
:106AC000C0E20A4018F00A40005800F004F00A4002
:106AD000000005100000FF7000E00F40054801684D
:106AE00041F47001016070470348016841F0404182
:106AF0000160704788ED00E034EF00E00448016871
:106B000041F00501016070470249401E086070476E
:106B100010E000E014E000E04C49FFE701200860CD
:106B20007047012100F01F0001FA00F04849086099
:106B30007047012100F01F0001FA00F0454908608C
:106B4000704745490860704700F01F00012202FAB3
:106B500000F0424ACB0748BF10608B0748BF9061E6
:106B60004B0748BF1062090748BF906070473A4A18
:106B7000126800F03F0002EB0012394893680340AE
:106B8000194391607047F0B5334C2568354C00F0DF
:106B90003F0005EB0016B7682740840604D504299A
:106BA00014BF062941F00101DDF814C0ACF1010E5B
:106BB00041EA0E14274307F04064B4F1406F04D05B
:106BC000A40E0CFA04F4A218521E326007F04042E0
:106BD000B2F1404F0FD0042918BF062906D140F06A
:106BE000200005EB001000F10C0304E0920F0CFAFA
:106BF00002F003445B1E7360B760F0BD164909687C
:106C000000F03F0001EB0010806800F00700410831
:106C1000490004291EBF42085200062A04BF40084A
:106C20004000704700F0FF0110B5CB080E4A02EBA0
:106C30008302890001F01C0113680F248C40000CB2
:106C4000A34388401843106010BD000004F00F40BB
:106C500028F00F402CF00F4008F00F401CF00F40C0
:106C6000F73FFC0008C0FFFF10F50F401AE050F896
:106C7000081F41F002010160704700F540600121EA
:106C80000160704700F540600149016070470000F5
:106C900051E5CC1A00F540600068012818BF0020BB
:106CA000704700BF50F8081F41F0010101607047B4
:106CB00000F58360016841F4807101607047000055
:106CC0007CB500200090DFF8804C20684008400030
:106CD0002060DFF8785C0423E0226946280002F097
:106CE0005EFD0028F5D000980128FCD0DFF8606C2C
:106CF0000423E4226946300002F051FD0028F5D05B
:106D000000980128FCD02878FBF733FE00280ED02D
:106D10006878FBF72EFE002809D0A878FBF729FE3B
:106D2000002804D0E878FBF724FE002806D10220D2
:106D300001F0D7F9206850F0020020603078FBF7AE
:106D400018FE00280ED07078FBF713FE002809D03B
:106D5000B078FBF70EFE002804D0F078FBF709FEB0
:106D6000002806D1012001F0BCF9206850F0040091
:106D70002060206850F00100206073BD10B5DFF87E
:106D8000C84B2078C00722D52068C0F340000028F7
:106D90000CD00422E021DFF8B40B02F041FD012801
:106DA00015D1206830F00200206010E02068C0F3A8
:106DB000800000280BD00422E421DFF8940B02F0BD
:106DC0002FFD012803D1206830F00400206010BDA1
:106DD00080B5022001F085F9012001F082F9DFF889
:106DE000680B016851F004010160016851F0020173
:106DF000016001BDDFF8500B007810F0060F01D0E4
:106E0000012000E00020704770B50D001400DFF88D
:106E1000C06B1A00802101FB04F1314400F0FAF844
:106E2000012840F0E380802000FB04F030444078EB
:106E3000002819D0230000220021FF2001F0CDF806
:106E4000002C00F0C980012C05D100220021002077
:106E500009F070FDC0E0022C40F0BE80002200214D
:106E6000002009F0B7FEB7E0DFF8680B802101FBD6
:106E700004F13144897801600021DFF85C2B802324
:106E800003FB04F31A4451700068012835D002282E
:106E900038D003283BD006286DD007286FD00828AB
:106EA0003AD00B287BD00C287DD00D2840D00E285E
:106EB00000F081800F286AD0102831D02F2852D0BE
:106EC000522816D081283FD0822842D0832845D02E
:106ED000852860D087284AD0882831D08A2866D073
:106EE0008F2850D090281FD09D2825D0A22866D06A
:106EF0006CE0200000F041F96EE00021200000F07D
:106F0000BCF969E00121200000F0B7F964E002213A
:106F1000200000F0B2F95FE0200001F0C9FB5BE067
:106F2000200000F0AAFA57E0200000F0F4FA53E045
:106F3000200000F0D1FA4FE0200000F059FB4BE0B8
:106F4000200000F007FD47E00021200000F01AFAC1
:106F500042E00121200000F015FA3DE0022120006E
:106F600000F010FA38E0200000F02AFE34E02000A3
:106F700000F034FD30E0200000F055FE2CE0200051
:106F800000F07EFE28E0200000F0F2FE24E0200069
:106F900000F057FF20E0200000F0A5FF1CE02000DB
:106FA00000F084FB18E0200000F05FFC14E02000FB
:106FB00000F034FC10E0200000F07AFE0CE023002A
:106FC0000022A221F02001F008F805E023000022B1
:106FD0000021FF2001F001F82900DFF8FC298020C2
:106FE000444302EB040000F08FF812E002280FD1B6
:106FF000230000220021FF2000F0EFFF2900DFF82E
:10700000D8298020444302EB040000F07DF800E022
:10701000002070BD2DE9F84305000E00002400207B
:1070200000E0401C904205D2295C0329F9D10021DF
:1070300029540400904201D2002C01D1002061E0CB
:10704000671E00E07F1E002F5BD4E85D0228F9D1A7
:107050000020E855E41B641C092C01D2022051E0F9
:10706000083CE00701D502204CE06408002C01D068
:107070007D2C01D3022045E0D81EA04201D3032B72
:1070800001D203203EE0781C411C695C285C00F0C2
:10709000C9FF30703078844201D0022032E05FF0C6
:1070A0000108F81C411C695C285C00F0BBFF707093
:1070B000707818EB00085FF0000913E017EB490047
:1070C000401D411C695C285C00F0ACFF06EB090127
:1070D0008870A14504D206EB0900807858FA80F840
:1070E00019F101094C45E9D27FEA080808F0FF08C8
:1070F00006EB04008078804501D0022002E00120E8
:1071000000E00020BDE8F283F8B505000E0001277D
:1071100002203070002413E0285D0009FBF7CBF952
:1071200006EB44014870285D10F00F00FBF7C3F92F
:1071300006EB44018870002C01D0285D3F18641CC8
:107140002878801C8442E7D3FF4307F0FF0738000C
:107150000009FBF7B0F906EB4401487017F00F0780
:107160003800FBF7A8F906EB44018870032006EB12
:107170004401C8706000001DF2BD38B50400DFF89E
:107180005058802000FB04F02844C0788DF800009F
:107190006846802101FB04F129440979417080216E
:1071A00001FB04F1294449798170802101FB04F13C
:1071B00029448979C170684600F043FF00280BD14B
:1071C000684600F05AFF002806D123000022522111
:1071D000F82000F002FF4FE0802000FB04F028447C
:1071E000007AC04300F0FF00802101FB04F1294434
:1071F000C979884206D0230000225221FF2000F0E6
:10720000ECFE39E0012C1CD1002009F0C6FB00285F
:1072100006D1230000225221F92000F0DEFE2BE0EF
:107220005FF480000021FAF70CFA00291ED1002833
:107230001CD1802000FB04F02844C079FFF7AFF98F
:1072400014E0022C12D1002009F0D6FC002806D14F
:10725000230000225221F92000F0BFFE0CE0802024
:1072600000FB04F02844C079FFF7A7F923000022AF
:107270005221F02000F0B1FE31BD2DE9F0410500B2
:107280000C00002C01D1012604E0012C01D10226C2
:1072900000E00326012D0BD1002009F07EFB002821
:1072A00020D12B0000223100F92000F096FE67E08B
:1072B000022D0BD1002009F09FFC002812D12B00D9
:1072C00000223100F92000F088FE59E00020F9F793
:1072D0007BFF002806D12B0000223100F92000F0AE
:1072E0007CFE4DE0DFF8F0662120802101FB05F1F6
:1072F0007054002C06D18120802101FB05F131441E
:1073000088700EE0012C06D18220802101FB05F15E
:107310003144887005E08320802101FB05F1314470
:10732000887000271BE0802000FB05F0304400EB54
:10733000070840213800FCF703FF88F803000DE040
:10734000012CF0D1802000FB05F0304400EB070851
:1073500020213800FCF7F4FE88F803007F1C202F62
:107360000ED2002CECD1802000FB05F0304400EB65
:10737000070800213800FCF7E3FE88F80300EDE77A
:10738000BDE8F081F0B589B005000C00DFF840667B
:10739000802000FB05F03044C0788DF8000068467E
:1073A000802101FB05F1314409794170802101FB05
:1073B00005F1314449798DF80210802101FB05F176
:1073C00031448979C170002C01D1812704E0012C5E
:1073D00001D1822700E08327684600F04EFE002896
:1073E00006D12B0000223900F82000F0F6FD42E023
:1073F000012D3AD1002009F0D0FA002806D12B0047
:1074000000223900F92000F0E8FD34E05FF480004C
:107410000021FAF716F9002920D100281ED10020FA
:1074200008E0802101FB05F131440144C97901AA3A
:107430001154401C2028F4D3002C04D1002101A8B1
:10744000FCF788FE0AE0012C04D1202101A8FCF7FA
:1074500081FE03E0402101A8FCF77CFE2B00002206
:107460003900F02000F0B9FD05E02B0000223900C2
:10747000F92000F0B2FD09B0F0BD2DE9F0410400A3
:10748000DFF84C05802101FB04F10844C579DFF8E1
:1074900048652220802101FB04F170549020802156
:1074A00001FB04F131448870802000FB04F030447B
:1074B000C57000270CE0802000FB04F0304400EB96
:1074C00007083900280001F07BFE88F804007F1CC3
:1074D000202FF0D3BDE8F081F8B50400DFF8F854B0
:1074E0002120802101FB04F168549D20802101FBB3
:1074F00004F12944887000260AE0802000FB04F093
:10750000284400EB0607300001F066FEF870761C98
:10751000202EF2D3F1BDF8B50400DFF8B45480207A
:1075200000FB04F02844C0788DF8000068468021F4
:1075300001FB04F1294409794170802101FB04F128
:10754000294449798DF80210802101FB04F1294476
:107550008979C170684600F090FD002806D12300AB
:1075600000229021F82000F038FD40E0012C38D1B5
:10757000002009F012FA002806D1230000229021F1
:10758000F92000F02AFD32E0802000FB04F02844BE
:10759000C679082E06D3230000229021FF2000F098
:1075A0001CFD24E05FF480000021FAF74AF800296E
:1075B00010D100280ED100270AE0802000FB04F043
:1075C00028443844027A3900300001F00DFE7F1C57
:1075D000202FF2D3230032009021F02000F0FDFC98
:1075E00005E0230000229021FF2000F0F6FCF1BD11
:1075F0007CB50400DFF8D853802000FB04F0284459
:10760000C0788DF800006846802101FB04F1294410
:1076100009794170802101FB04F1294449798DF8F1
:107620000210802101FB04F129448979C170684668
:1076300000F023FD002806D1230000229D21F82020
:1076400000F0CBFC31E0012C29D1002009F0A5F994
:10765000002806D1230000229D21F92000F0BDFC66
:1076600023E05FF480000021F9F7EBFF00290FD140
:1076700000280DD1002609E0802000FB04F02844FA
:107680003044C179300001F0D1FD761C202EF3D3B7
:10769000230000229D21F02000F09FFC05E0230044
:1076A00000229D21F92000F098FC73BD70B5040004
:1076B000C748802101FB04F10844C578C64E172055
:1076C000802101FB04F170548B20802101FB04F127
:1076D00031448870802000FB04F03044C5702800DD
:1076E00002F007FC802101FB04F1314408712800FD
:1076F00002F0DAFB802101FB04F131444871010002
:10770000090A802202FB04F2324491710100090C43
:10771000802202FB04F23244D171000E802101FB71
:1077200004F131440872280002F0D0FB802202FBF1
:1077300004F232445072020092B2120A802303FB18
:1077400004F333449A720200120C802303FB04F307
:107750003344DA720200120E802303FB04F3334435
:107760001A73802202FB04F23244517402000B00AF
:107770001A0A0023802303FB04F333449A740200A3
:107780000B001A0C0023802303FB04F33344DA7448
:10779000880D0021802101FB04F131440875280087
:1077A00002F0EBFB802101FB04F13144487301003E
:1077B000090A802202FB04F2324491730100090C91
:1077C000802202FB04F23244D173000E802101FBBF
:1077D00004F131440874280002F09CFB802101FB75
:1077E00004F131444875280002F0B7FB802101FB09
:1077F00004F1314488750021280002F09CFB8021AF
:1078000001FB04F13144C8750121280002F093FB0B
:1078100080214C4306EB0401087670BD70B504006E
:107820006B4D802000FB04F02844C678802000FBCC
:1078300004F028440179300002F0CDFB802000FBE9
:1078400004F0284441793000C046C046802000FB47
:1078500004F028448179300002F0DEFB230032007E
:107860008A21F02000F0B9FB70BDF8B5040058483B
:10787000802101FB04F10844C678574D1620802171
:1078800001FB04F168548C20802101FB04F12944A0
:107890008870802000FB04F02844C67002F090FB42
:1078A000802101FB04F129440871000A802101FBB9
:1078B00004F12944487102F078FB802101FB04F1B6
:1078C00029448871000A802101FB04F12944C87110
:1078D00002F0E0FB802101FB04F129440872000A58
:1078E000802101FB04F129444872012E0ED10026AB
:1078F0000E2E28D2802000FB04F0284400EB06075F
:10790000B01C02F0F6FAB872761CF1E7022E0ED126
:1079100000260E2E17D2802000FB04F0284400EB36
:107920000607B01C02F0F6FAB872761CF1E70020E8
:1079300007E0802101FB04F12944014400228A72FE
:10794000401C0E28F5D3F1BD402B0020382B002021
:107950003C2B002010B504001D49802000FB04F0E2
:107960000844807D802202FB04F20A44D27D72F03A
:10797000FF02D243904206D0230000228821FF203C
:1079800000F02BFB23E0012C0ED1802202FB04F23D
:107990000A4492F82320802303FB04F3194491F84E
:1079A000221008F0C7FF0FE0022C0DD1802202FB4D
:1079B00004F20A4492F82320802303FB04F31944C1
:1079C00091F8221009F006F9200000F071FE10BDB8
:1079D0009C120020442B00201C14002038B5040009
:1079E000DFF8C85C802000FB04F02844C0788DF8E4
:1079F00000006846802101FB04F1294409794170A7
:107A0000802101FB04F1294449798170802101FB27
:107A100004F129448979C170012C40F0CA8000200A
:107A200008F0BBFF002800F0C480684600F025FB8A
:107A3000012874D1802000FB04F02844C07901287B
:107A40002FD15FF480000021F9F7FBFD002921D13F
:107A500000281FD1DFF8180E802101FB04F1294412
:107A6000097A0170802101FB04F12944497A4170AF
:107A7000802101FB04F12944897A8170802101FB76
:107A800004F12944C97AC170DFF8E80D016851F0AA
:107A900004010160230000228721F02000F09DFAFC
:107AA0008DE0802000FB04F02844C07902282FD10B
:107AB0005FF480000021F9F7C4FD002921D10028DE
:107AC0001FD1DFF8B40D802101FB04F12944097AAC
:107AD0000170802101FB04F12944497A4170802121
:107AE00001FB04F12944897A8170802101FB04F1B2
:107AF0002944C97AC170DFF87C0D016851F0020198
:107B00000160230000228721F02000F066FA56E091
:107B1000230000228721F82000F05FFA4FE068463A
:107B200000F08FFA01283DD1802000FB04F02844AA
:107B3000C07902282FD15FF480000021F9F781FD80
:107B4000002921D100281FD1DFF82C0D802101FB55
:107B500004F12944097A0170802101FB04F12944D0
:107B6000497A4170802101FB04F12944897A8170AE
:107B7000802101FB04F12944C97AC170DFF8F40CBB
:107B8000016851F002010160230000228721F020EA
:107B900000F023FA13E0230000228721F82000F0F0
:107BA0001CFA0CE0230000228721F82000F015FACF
:107BB00005E0230000228721F92000F00EFA31BDF4
:107BC00010B5012828D1DFF8B41C0922802303FB5B
:107BD00000F3CA54A122802303FB00F30B449A70E4
:107BE000002209E0802303FB00F30B441344DFF879
:107BF000804CA45CDC70521C042AF3D30022042ABB
:107C000010D2802303FB00F30B441344DFF8684CCD
:107C1000A45CDC71521CF2E7030000222F21F92042
:107C200000F0DBF910BD10B50400012C0FD10020CD
:107C300008F0B3FE002803D0200000F076FA1EE022
:107C4000230000220621F92000F0C7F917E0022CDA
:107C50000FD1002008F0D0FF002803D0200000F052
:107C600064FA0CE0230000220621F92000F0B5F9A7
:107C700005E0230000220621F82000F0AEF910BD37
:107C800010B50400012C0FD1002008F086FE8428D6
:107C900003D1200000F0ECFB09E0230000220721C3
:107CA000F92000F09AF902E0200000F0E1FB10BD9D
:107CB00038B50400012C54D1002008F06EFE0028D5
:107CC0004FD0DFF8B85B0A20802101FB04F1685433
:107CD0009120802101FB04F1294488700020F9F7EC
:107CE00073FA802101FB04F12944C8705FF0FF3072
:107CF000F9F76EFA802101FB04F1294408710100B3
:107D0000090A802202FB04F22A4451710100090C85
:107D1000802202FB04F22A449171000E802101FBB3
:107D200004F12944C8715FF0FF300020C046802173
:107D300001FB04F1294408720100090A802202FBB8
:107D400004F22A4451720100090C802202FB04F261
:107D50002A449172000E80214C4305EB0401C87245
:107D600005E0230000220E21F92000F036F931BD94
:107D700038B50400DFF83459802000FB04F02844B3
:107D8000C0788DF800006846802101FB04F1294489
:107D900009794170802101FB04F1294449798170FE
:107DA000802101FB04F129448979C170684600F003
:107DB00048F9012804D0684600F05FF9012839D15C
:107DC0005FF480000021F9F73CFC002929D100284C
:107DD00027D1802000FB04F02844C179012009F05C
:107DE00023F8802000FB04F02844017A022009F0E7
:107DF0001BF8802000FB04F02844417A032009F09E
:107E000013F8802000FB04F02844C17A042009F014
:107E10000BF8802000FB04F02844017B052009F0CA
:107E200003F823000022DFF8580A0168F02000F070
:107E3000D4F805E0230000228F21F82000F0CDF8CF
:107E400031BD38B50400DFF8345A0A20802101FB27
:107E500004F168547820802101FB04F129448870E2
:107E60000020F9F7B1F9802101FB04F12944C87021
:107E70000120F9F7A9F9802101FB04F129440871D7
:107E80000220F9F7A1F9802101FB04F1294448718E
:107E9000002008F082FD802101FB04F12944887153
:107EA000012008F07AFD802101FB04F12944C8710A
:107EB000022008F072FD802101FB04F129440872C0
:107EC0000020802101FB04F1294448720020802118
:107ED00001FB04F12944887200218020444305EB12
:107EE0000400C17231BD38B50400DFF8C0578020EE
:107EF00000FB04F02844C0788DF80000684680211B
:107F000001FB04F1294409794170802101FB04F14E
:107F1000294449798170802101FB04F12944897940
:107F2000C170684600F0A9F8002806D1230000229D
:107F30008521F82000F051F84EE0802000FB04F08D
:107F40002844C0790006802101FB04F12944097A04
:107F500010EB0140802101FB04F12944497A10EB28
:107F60000120802101FB04F12944897A50FA81F033
:107F7000C10704D5F8F7EBF802F06FF826E08107A7
:107F800002D5F8F7F1FC21E0810102D500F0F2FE04
:107F90001CE0410706D51E20FBF7C4FF0121FBF7BB
:107FA0002DFF13E0002805D501214FF40050FBF709
:107FB00084FF0BE0410005D501214FF40050FBF791
:107FC00096FF03E0400601D501F0E8FF2300002200
:107FD0008521F02000F001F831BD70B4DFF89C4835
:107FE0000425802606FB03F6A5550025802606FB02
:107FF00003F626447570802505FB03F52544A8701B
:10800000802000FB03F02044C170802000FB03F0BF
:1080100020440271120A8020434304EB03004271A2
:1080200070BC704738B50C00C0B2FAF731FA0500E1
:108030002D012000C0B2FAF72BFA45192800C0B272
:1080400032BDDFF8341802780B789A4201D0002054
:1080500012E042784B789A4201D000200CE08278FE
:108060008B789A4201D0002006E0C078C978884217
:1080700001D0002000E001207047DFF8F4170278FB
:108080000B789A4201D0002112E042784B789A4254
:1080900001D000210CE082788B789A4201D0002137
:1080A00006E0C278C9788A4201D0002100E00121AF
:1080B000002914D10178332901D000210FE0417843
:1080C000312901D000210AE08178302901D0002136
:1080D00005E0C078312801D0002100E0012108002E
:1080E0007047022810D1DFF890073021017030214D
:1080F0004170302181703021C170DFF8780701684C
:1081000051F0020101600FE0DFF8640730210170D7
:1081100030214170302181703021C170DFF8540767
:10812000016851F004010160704770B50400DFF888
:108130004C572720802101FB04F1685486208021C0
:1081400001FB04F1294488705FF0FF30F9F766FA0B
:108150000100090E802202FB04F22A44D1700100C2
:10816000090C802202FB04F22A4411710100090A61
:10817000802202FB04F22A445171802101FB04F1A8
:10818000294488710026002006F032FF012801D121
:1081900056F00106012006F02BFF012801D156F010
:1081A0000206802000FB04F02844C6715FF0FF3017
:1081B000F9F734FA002807D0F9F749FA802101FBD2
:1081C00004F12944087205E00020802101FB04F13C
:1081D000294408725FF0FF3040F2FF11F9F731FADD
:1081E0000100090E802202FB04F22A4451720100B0
:1081F000090C802202FB04F22A4491720100090A50
:10820000802202FB04F22A44D172802101FB04F196
:1082100029440873002C16D14FF48040F9F7FEF979
:10822000002802D1F4F748F900E000200100090A13
:10823000802202FB04F22A445173802101FB04F1E5
:108240002944887313E05FF0FF3040F2FF11F9F723
:10825000F8F902000B001A0A0023802303FB04F341
:108260002B445A73802000FB04F0284481735FF094
:10827000FF30FCF73AFE0100090E802202FB04F2F7
:108280002A44D1730100090C802202FB04F22A4423
:1082900011740100090A802202FB04F22A4451747D
:1082A000802101FB04F1294488747FF07040FCF7C1
:1082B00012FE0100090E802202FB04F22A44D1744E
:1082C0000100090C802202FB04F22A44117501000E
:1082D000090A802202FB04F22A445175802101FB25
:1082E00004F12944887500F010FD0100090E802278
:1082F00002FB04F22A44D1750100090C802202FB22
:1083000004F22A4411760100090A802202FB04F2D9
:108310002A445176802101FB04F129448876FDF737
:10832000B5FF802101FB04F12944C876000A8021B1
:1083300001FB04F12944087704F030F8802101FBA7
:1083400004F129444877002C10D14FF40040F9F78C
:108350003CF90020802101FB04F1294488770020AA
:10836000802101FB04F12944C8770DE01E20FBF7B2
:10837000D9FD802101FB04F1294488770020802168
:1083800001FB04F12944C8771020F9F747F90028C8
:1083900008D0F9F735F9802101FB04F1294481F86F
:1083A000200014E00820F9F739F9002808D0F9F77F
:1083B0002EF9802101FB04F1294481F8200006E018
:1083C0000020802101FB04F1294481F820004FF4B2
:1083D0008040F9F723F9002803D1F4F76DF8C04382
:1083E00001E05FF0FF300100090A802202FB04F285
:1083F0002A4482F82110802101FB04F1294481F8EC
:108400002200012008F0EAFC802101FB04F129444C
:1084100081F82300022008F0E1FC802101FB04F137
:10842000294481F82400032008F0D8FC802101FBB6
:1084300004F1294481F82500062008F0CFFC8021B2
:1084400001FB04F1294481F82600042008F0C6FC51
:10845000802101FB04F1294481F82700052008F060
:10846000BDFC80214C4305EB040181F8280070BD60
:1084700070B50400DFF804542720802101FB04F1CB
:1084800068547720802101FB04F12944887003207F
:10849000F9F730FA802101FB04F12944C870000A81
:1084A000802101FB04F1294408710420F9F722FA24
:1084B000802101FB04F129444871000A802101FB5D
:1084C00004F1294488710120F9F714FA802101FB95
:1084D00004F12944C871000A802101FB04F12944F8
:1084E00008720020F9F706FA802101FB04F1294403
:1084F0004872000A802101FB04F12944887200209F
:10850000802101FB04F12944C8720020802101FB75
:1085100004F1294408730220F9F7ECF9802101FBEA
:1085200004F129444873000A802101FB04F1294425
:108530008873F3F7A4FF0600002E02D47604760CAD
:1085400003E07604760C56F40046802000FB04F02D
:108550002844C6733000000A802101FB04F129443D
:108560000874F3F7A9FF64214E43B6FBF0F08021B5
:1085700001FB04F1294448740020802101FB04F12F
:10858000294488740020802101FB04F12944C87427
:108590000020802101FB04F129440875002080217E
:1085A00001FB04F1294448750020802101FB04F1FE
:1085B00029448875F3F757FF802101FB04F1294412
:1085C000C875000A802101FB04F1294408760020C7
:1085D000802101FB04F1294448760020802101FB21
:1085E00004F12944887600F093FB0100090E8022F3
:1085F00002FB04F22A44D1760100090C802202FB1E
:1086000004F22A4411770100090A802202FB04F2D5
:108610002A445177802101FB04F129448877002006
:10862000802101FB04F12944C8770020802101FB4F
:1086300004F1294481F820000020802101FB04F18D
:10864000294481F821000020802101FB04F1294404
:1086500081F822000020802101FB04F1294481F8E7
:1086600023000020802101FB04F1294481F824002B
:108670000020802101FB04F1294481F8250000201D
:10868000802101FB04F1294481F82600002080218B
:1086900001FB04F1294481F8270000218020444394
:1086A00005EB040080F8281070BD00009C1200202B
:1086B00070B50400714D2920802101FB04F168543C
:1086C0008820802101FB04F1294488704520802105
:1086D00001FB04F12944C8703120802101FB04F121
:1086E000294408715320802101FB04F12944487179
:1086F0004C20802101FB04F1294488710020802155
:1087000001FB04F12944C8710020802101FB04F120
:10871000294408720020802101FB04F12944487299
:108720000020802101FB04F129448872002080216F
:1087300001FB04F12944C8720020802101FB04F1EF
:10874000294408730020802101FB04F12944487367
:108750000020802101FB04F129448873002080213E
:1087600001FB04F12944C8730020802101FB04F1BE
:10877000294408740020F7F7CBFC802101FB04F1A9
:10878000294448740120F7F7C3FC802101FB04F160
:1087900029448874FF26802000FB04F02844C67416
:1087A000802000FB04F028440675802000FB04F0C4
:1087B000284446750420C046802101FB04F1294469
:1087C0008875802000FB04F02844807DC043802110
:1087D00001FB04F12944C875002006E0802101FB5B
:1087E00004F1294401440E76401C0A28F6D33320B4
:1087F000802101FB04F1294481F8220035208021E9
:1088000001FB04F1294481F823000020802101FBB1
:1088100004F1294481F824000020802101FB04F1A7
:10882000294481F825000020802101FB04F129441E
:1088300081F826000020802101FB04F1294481F801
:1088400027000020802101FB04F1294481F8280041
:108850000020802101FB04F1294481F82900002136
:108860008020444305EB040080F82A1070BD00000E
:108870003C2B0020402B0020382B00201C14002013
:10888000442B00207CB5DFF83C43206840084000C2
:108890002060002500E06D1CB5F5007F34D2DFF8C4
:1088A00028630823EA0012F58052694606EBC500EA
:1088B00000F075FF0028F2D001F000F8012802D185
:1088C00000F012FFF8E7082106EBC500F9F7D0FD2C
:1088D0000128E0D1002004E0002106EBC50211547C
:1088E000401C0828F8D30822E90011F5805106EB56
:1088F000C50000F095FF0028F5D000F0DFFF01284B
:10890000C9D100F0F1FEF8E700F013F9AF4D00F027
:1089100017F928602868AE490860206850F0010007
:108920002060FDF7B9F9C00605D5352233210220B4
:1089300000F007F804E035223321012000F001F8AF
:1089400073BD2DE9F04106000D0014009D4F3878ED
:10895000C00701D400204EE001200021F8F771FE8D
:10896000002947D1002845D1387810F00E0F41D1A9
:108970005FF00040F8F752FE00283BD1934F386873
:10898000401C38603868B0F5007F01D300203860A3
:10899000052008F023FADFF83082396808F8310042
:1089A000042008F01BFA396808EBC1014870032065
:1089B00008F014FA396808EBC1018870022008F049
:1089C0000DFA396808EBC101C870012008F006FAF9
:1089D000396808EBC1010871386808EBC0004671BE
:1089E000386808EBC0008571386808EBC000C471B6
:1089F000012000E00020BDE8F08138B5714C2078FE
:108A0000C0077DD52068C0F34000002819D0714D03
:108A100008222868C10011F580516B482B6800EBD3
:108A2000C30000F0FDFE01286AD12868401C2860C0
:108A30002868B0F5007F63D3206830F00200206022
:108A40005EE02068C0F3C000002825D0002108E0C7
:108A500000225D4B03EBC1031A54401C0828F7D3D6
:108A6000491CB1F5007F01D20020F7E700F061F862
:108A700008224FF48051544800F0D2FE01283FD123
:108A8000206830F008002060206850F0020020606C
:108A900001205049086033E02068C0F380000028BE
:108AA00016D0002108E00022474B03EBC1031A5403
:108AB000401C0828F7D3491CB1F5007F01D20020E3
:108AC000F7E700F036F8206830F00400206017E087
:108AD0003F4D3E4800682968884211D02C68641CCC
:108AE000B4F5007F00D300240822E10011F5805185
:108AF000354800EBC40000F093FE012800D12C6043
:108B000031BD3048007810F00A0F01D0012000E09C
:108B100000207047C0B2012805D12A48016851F0F1
:108B20000801016004E02748016851F00401016078
:108B300070470020254908600020254908607047DB
:108B400038B592B00024012536E01F4810F83410E3
:108B500064310E9100EBC4014978491E0D9100EB80
:108B6000C40189780C9100EBC401C9780B9100EB2A
:108B7000C40109790A910021099110F83510643176
:108B8000059100EBC5014978491E049100EBC50130
:108B90008978039100EBC501C978029100EBC5000B
:108BA000007901900020009009A96846F9F768FF54
:108BB000002800D42C006D1CB5F5007FC5D3200023
:108BC00013B030BDF42B00201C000020EC2B002043
:108BD000F02B0020F82B002038B5774C00202060C7
:108BE000764D2900764808F033FA28687549086000
:108BF0000120206031BDF8B56F480068012879D1A7
:108C00006E4C2068152801D2012000E014206D4D23
:108C100021682A688018814206D321686848006864
:108C200008F0A6FA2068286021686548006808F006
:108C3000D7FA5FF400300021F8F7A8FC01200021EA
:108C4000F8F7FFFC002946D1002844D15020FBF75B
:108C500069F900283FD05120FBF764F900283AD089
:108C60005220FBF75FF9002835D0032008F0B6F852
:108C70000500042008F0B2F80600052008F0AEF860
:108C800007005220FBF74EF9B84205D25FF40030DE
:108C90000021F8F7C7FC1EE05220FBF743F987429A
:108CA00019D15120FBF73EF9B04205D25FF40030F4
:108CB0000021F8F7B7FC0EE05120FBF733F98642AC
:108CC00009D15020FBF72EF9854204D35FF4003020
:108CD0000021F8F7A7FC4020FBF724F93A49884225
:108CE00000D308002168814204D35FF400300021E2
:108CF000F8F798FC0820FBF7DCF8002804D15FF4B3
:108D000000300021F8F742FCF1BD2C4800687047A4
:108D10002B480068704780B52848016811F1010FA1
:108D200002D00168491C0160254A116811F1010F48
:108D300002D01168491C11600168106808F06DFAD2
:108D400001BD38B51E4C002020601C4D002028605D
:108D500028681C4908605FF400300021F8F716FC11
:108D60005FF480100021F8F711FC2968206808F0F2
:108D7000FFF931BD10B5114C002020602068114969
:108D800008605FF400300021F8F700FC5FF4801009
:108D90000021F8F7FBFB21680948006808F0E8F9B2
:108DA00010BD80B505480168064A11600168044895
:108DB000006808F0DDF901BD8C2A0020842A00201B
:108DC000802A0020882A002040420F0080B508F049
:108DD0002BFA02BD38B5002400E0641C082C4BD2ED
:108DE000DFF8A0582023620112F5D07269466001B5
:108DF000284400F0D4FC0028F2D000F05FFD0128E8
:108E000002D100F071FCF8E7202160012844F9F755
:108E10002FFB012819D1002004E0002162012A441F
:108E20001154401C2028F8D32022610111F5D07183
:108E30006001284400F0F4FC0028F5D000F03EFD6D
:108E40000128CAD100F050FCF8E76001284400F086
:108E5000D2FA0028C1D12022610111F5D071600140
:108E6000284400F0DDFC0028F5D000F027FD0128A3
:108E7000B3D100F039FCF8E7DFF80C481C234FF4BD
:108E800038726946200000F08AFC0028F4D000F017
:108E900015FD012802D100F027FCF8E71C21200075
:108EA000F9F7E6FA012815D1002002E0002121544B
:108EB000401C1C28FAD31C224FF43871200000F00B
:108EC000AFFC0128F7D000F0F9FC012802D100F036
:108ED0000BFCF8E7DFF8B407416851F0010141608D
:108EE00031BD2DE9F041DFF8A4472079C00740F1FA
:108EF000D5806068C0F3800000281FD0606830F023
:108F000004006060002009E00022DFF878374501A6
:108F10002B441A54491C2029F6D3401C082801D29E
:108F20000021F8E7002504E00021280000F07EF988
:108F30006D1C1C2DF8D3DFF858072060206800282E
:108F400026D02068F9F7BDFA0500082D13D220229B
:108F5000690111F5D071DFF82C076B01184400F09E
:108F60005FFC012814D12800F9F7F3FC216831EAED
:108F7000000020600CE01C224FF43871DFF8080775
:108F800000F04EFC012803D1206830F080502060B2
:108F90005FF080500021F8F7F9FA10200021F8F76F
:108FA000F5FA00F07DF8002812D10020DFF8E41671
:108FB00008706068C0F3C000002804D000220021BF
:108FC0000E20FFF7BEFC606830F00800606065E0CE
:108FD0006068C0F3C000002804D1002201210E20E7
:108FE000FFF7AFFC606850F008006060DFF8A4563F
:108FF000002028705FF080500021F8F713FB01205B
:109000000021F8F71EFB002901D1002800D045E01F
:10901000062007F0E3FE060000270CE0380000F011
:1090200009FB012806D1380000F07CF9012801D1A4
:1090300007260A277F1C062FF0D310200021F8F7FF
:10904000A5FA002700E07F1C062F1CD2DFF83406AB
:109050003100C9B249010844052101FB07F110F8AC
:1090600001804046C0B20028EDD039003000C0B2C7
:1090700000F0F7F80128E6D1606850F01000606059
:1090800085F800800AE06068C0F30010002805D071
:1090900001202870606830F010006060BDE8F08149
:1090A00010B50C20FAF75AFF012815D14FF4806053
:1090B000FBF71BFF002807D0DFF8CC05016851F053
:1090C0000101016001240FE0DFF8BC0501684908D7
:1090D00049000160002407E0DFF8AC050078C00714
:1090E00001D5012400E000240A20FDF7DAF8012868
:1090F00000D10024200010BD5FF0FF30DFF8941590
:109100000A78022A01D108203FE00A78012A01D119
:1091100000203AE00A78032A01D1042035E00A78D9
:10912000042A01D10C2030E00A78052A01D1202040
:109130002BE00A78062A01D1242026E00A78072AA3
:1091400001D1102021E00A78082A01D114201CE066
:109150000A78092A01D1012017E00A780A2A01D1E8
:10916000052012E00A780B2A01D140200DE00A7890
:109170000C2A01D1482008E00A780D2A01D150209C
:1091800003E009780E2900D118207047DFF8FC149D
:109190004868C0F34000002807D10868002804D1BF
:1091A0004868C0F38000002801D0012000E00020C2
:1091B0007047DFF8D804416851F0040141607047FE
:1091C000082807D2202905D2DFF8B824400110442E
:1091D000405C00E0002070471C2803D2DFF8A81490
:1091E000085C00E00020704738B50400082C1CD251
:1091F00020291AD2DFF8A0546A541F2915D128005B
:1092000000F0F9F8002006E0295CDFF8782463011B
:109210001A441154401C2028F6D3DFF8700401686A
:10922000012212FA04F40C43046031BD10B51C286D
:1092300016D2DFF8684421541B2811D1200000F019
:10924000A8F9002004E0215CDFF83C241154401C04
:109250001C28F8D3DFF83404016851F08051016014
:1092600010BD2DE9F04782460C00012007F0B6FD45
:109270000500022007F0B2FD0600DFF808045FEAEF
:109280004A110144052202FB04F211444F785FEABF
:109290004A110144052202FB04F2114491F80280B4
:1092A0005FEA4A110144052202FB04F2114491F8DD
:1092B00003905FEA4A1101440520444301EB040096
:1092C00004794F4503D1A04501D1002028E0434651
:1092D0003A002900300000F054F9012801D10120A2
:1092E0001EE043463A002900300000F03CF9002817
:1092F00001D1002014E023004A462900300000F08C
:1093000040F9012801D100200AE023004A46290043
:10931000300000F028F9012801D1002000E00120F0
:10932000BDE8F08738B50400062C01D3002061E0C9
:10933000032007F053FD0500042007F04FFD010056
:10934000DFF8442302EB84004079002804D002EBCC
:1093500084000079002801D100204BE002EB84005A
:10936000C079002804D002EB84008079002801D164
:1093700000203FE002EB84004079814201D20020CE
:1093800038E002EB8400C079884201D2002031E04D
:1093900002EB8400407981421DD102EB8400007908
:1093A000854201D2002025E002EB8400007985424D
:1093B00001D101201EE002EB8400C079814201D27C
:1093C000012017E002EB84008079A84201D301203C
:1093D00010E000200EE002EB8400C079814208D149
:1093E00002EB84008079A84201D2002002E0012033
:1093F00000E0012032BD70B5040001250026ADE07B
:10940000052000FB06F020444078182814DA0520D7
:1094100000FB06F02044C07818280DDA052000FB78
:1094200006F0204480783C2806DA052000FB06F090
:10943000204400793C281DDB0020052101FB06F1BA
:10944000214448700020052101FB06F12144887069
:109450000020052101FB06F12144C87000200521F0
:1094600001FB06F1214408710020052101FB06F1F2
:10947000605400250E20052101FB06F1615C884245
:109480001DD20020052101FB06F121444870002077
:10949000052101FB06F1214488700020052101FB14
:1094A00006F12144C8700020052101FB06F121448A
:1094B00008710020052101FB06F1605400250520FC
:1094C00000FB06F020448378052000FB06F02044D2
:1094D0004278052000FB06F020440179052000FBBE
:1094E00006F02044C07800F03EF8002835D1052071
:1094F00000FB06F020448378052000FB06F02044A2
:109500004278052000FB06F020440179052000FB8D
:1095100006F02044C07800F034F800281DD1002067
:10952000052101FB06F1214448700020052101FBC3
:1095300006F1214488700020052101FB06F1214439
:10954000C8700020052101FB06F1214408710020AC
:10955000052101FB06F160540025761C062EFFF460
:109560004FAF280070BD824201D2012008E0904236
:1095700005D18B4201D2012002E0002000E0002052
:109580007047904203D1994201D1012000E00020B0
:10959000704738B50400002549E004EB85000079E8
:1095A00000282ED004EB85004079002829D004EB58
:1095B00085008079002824D004EB8500C07900283C
:1095C0001FD004EB8500037904EB8500427904EB9E
:1095D0008500817904EB8500C079FFF7C4FF01287D
:1095E00024D004EB8500037904EB8500427904EB79
:1095F0008500817904EB8500C079FFF7C2FF01285F
:1096000014D0002004EB85010871002004EB8501D3
:109610004871002004EB85018871002004EB85016E
:10962000C87120780221A940884320706D1C062D46
:10963000B3D331BD002803D11349097889071DD45C
:10964000012803D110490978490717D4022803D10A
:109650000D490978090711D4032803D10A4909786B
:10966000C9060BD4042803D107490978890605D413
:10967000052805D104480078400601D5012000E006
:1096800000207047801E002004290020202A00208E
:10969000FF000010F02D0020AC2800202029002021
:1096A00080B50020DFF8141608600020DFF81016DF
:1096B00008600020DFF80C16086000F018FA002897
:1096C00008D10120DFF8001608605FF40020F7F7EA
:1096D0006CFF03E00020DFF8F0150860F6F714FDDA
:1096E000DFF8E815086001BD80B5DFF8D405006833
:1096F000002844D1DFF8D8050168012923D1DFF81B
:10970000D4150A68521C0A60002202600868032807
:1097100002D200F09EFA32E0DFF8BC0500780028A3
:1097200004D10020DFF8B415096808600120DFF8D3
:10973000941508600120DFF8901508605FF40020A0
:10974000F7F733FF1BE0DFF890050078012816D10A
:10975000DFF88C050068012811D1F6F7D5FCDFF899
:1097600084150968401A0A2809D3DFF87C050168C6
:10977000DFF87805006800F02FFA00F005FADFF84E
:1097800044050068012809D1F6F7BEFCDFF83C1556
:109790000968401A652801D300F03AFA01BD38B5CE
:1097A000DFF820452568012D04D0DFF81C552D6811
:1097B000012D01D1002032E0012525600024DFF8D1
:1097C00014552C600024DFF810552C700124DFF8AC
:1097D00020552C60DFF814452260DFF80C2513605B
:1097E000DFF810351860DFF8F4040160012008602C
:1097F0001168206800F0F0F9002004E00021DFF893
:10980000F8241154401C2028F8D300F070F90028E7
:1098100002D100F0FDF901E000F0B6F9012032BDFF
:1098200070B5DFF8A0341C68012C04D0DFF8984430
:109830002468012C01D100203FE001241C6000239A
:10984000DFF890442360DFF8B4440B001B0A237058
:109850006170931CDFF8A8542B600123DFF8A45437
:109860002B60002304E0C55C04EB0306B5705B1CB1
:109870009342F8D30023DFF8904423600123DFF8FC
:10988000584423700123DFF8684423600023DFF885
:1098900050442360DFF854341960DFF84C140A6038
:1098A000DFF85014086000F022F9002802D100F01F
:1098B000AFF901E000F068F9012070BDDFF80404A1
:1098C0000068704710B5DFF84444200007F0EDFC55
:1098D000200007F0F8FC00281AD0DFF82C040068FC
:1098E000012809D0DFF818040068002804D00421FA
:1098F000200007F0E5FC08E0DFF814040068002809
:1099000003D00421200007F0DBFC00F081F9EDE03A
:10991000DFF8F413086801284DD0DFF8E42310685D
:1099200000281DD10868022868D1012008600122A2
:109930005021200007F0C0FCDFF8D40301680129A2
:1099400006D1002101600721200007F0B9FC06E0E4
:109950000168491E01600B21200007F0B1FCC5E041
:109960001068012814D10868002811D10020106067
:10997000DFF8900301684A1C0260DFF88003415C55
:10998000200007F0ACFC0521200007F099FC11E055
:109990001068401E1060DFF86C0301684A1C02600A
:1099A000DFF85803415C200007F099FC01212000FA
:1099B00007F086FC9AE0200008300068DFF85413B6
:1099C000DFF854230B68D0540868401C0860DFF8A7
:1099D00040130868002811D00868012806D100202B
:1099E00008600521200007F06BFC7FE00868401E3E
:1099F00008600921200007F063FC77E0BC4801689B
:109A000001292AD100210160B348017801290AD136
:109A1000F6F77AFBB34908600120B14908600020DD
:109A2000A749086062E00078002813D1002004E014
:109A3000B949095CB04A1154401CB64909688842CA
:109A4000F6D3A9480168A948006800F0C5F800F0FD
:109A50009BF84BE000F0DCF848E0200007F021FC28
:109A60009D480078002826D10021002000E0401CFD
:109A7000A84A1368984206D29F4B1B5CA64C245CF4
:109A8000A342F4D00121012902D100F0C1F82AE05B
:109A9000002005E09849095C964B1B681954401C4E
:109AA00011688842F6D300208C49096808600020BC
:109AB0008449086017E00021002000E0401C954A1E
:109AC0001268904207D28D4A02449278924B1B5CF6
:109AD0009A42F3D00121012902D100F099F802E065
:109AE00000207849086000207549086010BDF8B56D
:109AF000724C2068002845D1884D04212800F6F7D3
:109B000049FA08212800F6F73BFA002600E0761C07
:109B10000A2E0ED2824F00203860FA20FCF7C8F8D7
:109B200004203860FA20FCF7C3F87E48006800285B
:109B3000EDD07C480068002801D1002023E07A485D
:109B4000FCF77AF87948F6F777FA7948F6F774FA75
:109B500004212800F6F736FA08212800F6F728FA3B
:109B6000E0211820FCF71DFAFCF71AF90100012288
:109B7000664807F067FB1820FCF724FA01202060F4
:109B8000012000E00120F2BD10B5F6F7BDFA4F4903
:109B900008600020524908600120494908605B4C78
:109BA000200007F082FB200007F079FB0022502103
:109BB000200007F081FB01205249086050480168ED
:109BC000491E01604D480178200007F088FB032101
:109BD000200007F075FB10BD0022414B1A600222E5
:109BE000474B1A60454A03001B0A1370507002204D
:109BF000454A1060002003E00022474B1A54401CE5
:109C00002028F9D34248016000204249086070478B
:109C100010B501202E4908603C4C200007F041FBA4
:109C20000021200007F05BFB0721200007F048FB24
:109C300041F21850FCF73CF8002029490860200048
:109C400007F027FB00201E49086000201B49086020
:109C500010BD80B500201E490860FFF748FF0028AE
:109C600001D1012000E00020012802D1FFF7D0FF40
:109C700022E001201E4908600020194908601648AA
:109C8000007800280ED1002003E000211A4A115468
:109C9000401C2028F9D31448016814480068FFF7D5
:109CA0009BFF07E010480068801C154908600120F0
:109CB00014490860FFF768FF01BD0000C82A0020B2
:109CC000D02A0020D42A0020CC2A0020F82A002004
:109CD000E02A0020102B0020DB2D00200C2B002080
:109CE000DC2A0020FC2A0020042B0020002B00206E
:109CF000D82A0020082B00204C280020C027002054
:109D0000EC2A0020E42A0020F42A0020000002406F
:109D1000F02A0020E82A00202C28002000500040D3
:109D20001050004020500040002000F003080100C7
:109D3000030C010080B500F0B8F900F0FCF9DFF881
:109D40001809016851F00101016001BD1CB5DFF87F
:109D500008492078C00774D55720FAF7E3F8DFF8F0
:109D6000FC180A6882421CD0DFF8F4180868002842
:109D70000AD0002008605FF0FF30DFF8E8180860C4
:109D8000206850F0080020605920FAF7CBF800282E
:109D900004D0012200215920FAF767F900F0CBF92D
:109DA0002DE00868002815D00868012802D100F0CD
:109DB000ECF901E000F035FADFF8A4080068DFF8FC
:109DC000A4180968C943884219D05FF48000F7F7E6
:109DD000ECFB14E0206830F02000206020200021FF
:109DE000F7F7D4FB5FF080700021F7F7CFFB00207E
:109DF0000821F7F7CBFB00202021F7F7C7FB2068ED
:109E0000C0F3C00000281CD0DFF8540801688DF8AA
:109E100000100068000A8DF80100DFF848080168AA
:109E20008DF802100068000A8DF80300042220213A
:109E30006846FFF7F5FC012803D1206830F00800E0
:109E4000206013BD80B5DFF814080068022810D325
:109E5000DFF804080068C0F34010002809D1002092
:109E60000821F7F7EEFB002903D1002801D10120DA
:109E700000E0002002BDDFF8E0070068C0F34010FA
:109E8000704780B500202021F7F7DBFB002901D1C6
:109E9000002805D0DFF8E40B016851F002010160F1
:109EA000DFF8D80B006802BD00280DD010280BD2B7
:109EB000DFF8A8170968012906D1DFF8C41B01EBF8
:109EC000800050F8080C00E00020704700280DD0FA
:109ED00010280BD2DFF884170968012906D1DFF8B2
:109EE000A41B01EBC00050E9040101E000200021A7
:109EF000704700280CD010280AD2DFF860170968D4
:109F0000012905D1DFF8681C084410F8020C00E0B4
:109F10000020704700280CD010280AD2DFF83C1728
:109F20000968012905D1DFF8601B084410F8020C0C
:109F300000E000207047821E0E2A0CD2DFF81C279A
:109F40001268012A07D1DFF82C2C02EB40000844EC
:109F500010F8040C00E000207047811E0E290AD280
:109F6000DFF8F8160968012905D1DFF80C1C084450
:109F700010F8020C00E000207047811E0E290BD261
:109F8000DFF8D8160968012906D1DFF85C1C01EB5F
:109F9000800050F8080C00E000207047DFF8B80699
:109FA000016851F0100101607047DFF8B0060068E9
:109FB000012803D1DFF8340C006800E0002070476E
:109FC000DFF898060068012803D1DFF8880C0068E4
:109FD00000E000207047F8B504000D00A01E0E2818
:109FE00019D2DFF8A46A06EB040010F8020C8542CF
:109FF00011D0DFF8887B386800280CD12000F8F7F2
:10A00000A8FCDFF8541C0968014204D006EB0400E8
:10A0100000F8025C3C60F1BDF8B504000D00A01E24
:10A020000E2819D2DFF8506B06EB040010F8020C72
:10A03000854211D0DFF8487B386800280CD1200019
:10A04000F8F787FCDFF8101C0968014204D006EB22
:10A05000040000F8025C3C60F1BDDFF80006006817
:10A06000012809D1DFF8F005016851F00401016011
:10A070000020DFF8E81B08607047DFF8E0050068A3
:10A08000012801D0002004E0DFF8CC050068C0F30F
:10A0900080007047DFF8C4050068012803D1DFF8AD
:10A0A000C00B006800E0002070473EB5042320226A
:10A0B00001A96846FFF773FB0028F7D0FFF7FEFB06
:10A0C000012802D1FFF710FBF8E7DFF894459DF86F
:10A0D0000000206020689DF8011050EA01202060F7
:10A0E000206880B22060DFF87C559DF8020028606F
:10A0F00028689DF8031050EA01202860286840F085
:10A100007F4050F47F00286004216846F8F7B0F9DA
:10A11000012804D020682968C94388420AD0002059
:10A1200020602068C0432860DFF82C05016851F0EA
:10A130000801016037BD10B5DFF820455720F9F759
:10A14000F1FE20602068002807D0206806F000FAA1
:10A150002068012801D100F037FADFF8FC0401681B
:10A1600031F0200101600020DFF8F81A0860F5F7EF
:10A17000CBFF0A38DFF8F01A086041F20500DFF87B
:10A18000EC1A088000F036FD10BD10B500F032FD6D
:10A1900020200021F7F7FAF9DFF8D44A20780128C7
:10A1A00004D0022805D100F05FFA08E000F070FC4E
:10A1B00005E0022020705FF48000F7F706FADFF870
:10A1C00098140868C0F30010002829D020780128CE
:10A1D00026D0012020700020DFF8802A1060086857
:10A1E00030F0020008600020DFF8742410605FF097
:10A1F000FF30DFF870241060086830F0100008604D
:10A200000020DFF8601A0860002007E0FF21DFF877
:10A2100078281154DFF860291154401C0E28F5D31A
:10A2200010BD3EB55FF080700021F7F7AFF9202038
:10A230000021F7F7F7F9684606F0B3F9DFF81C4498
:10A24000216888424BD1F5F75FFFDFF8281A0860D4
:10A25000DFF80404016831F0200101609DF802106C
:10A2600009029DF801000143B1F5805F05D1216825
:10A270004FF4805000F0C8F840E0B1F5905F3DD158
:10A280009DF804009DF8071071F0FF01C943884252
:10A2900002D1DFF8E81708609DF80650FF2D0ED0B8
:10A2A0005920F9F73FFE854209D0012229005920A3
:10A2B000F9F7DBFE41F20500DFF8B01908809DF8E0
:10A2C0000500FF2801D1F5F742FF00F093FC21685B
:10A2D000DFF89809B0F9000000F096F80EE0F5F705
:10A2E00013FFDFF890190968401AB0F57A7F05D39B
:10A2F000DFF86403016851F02001016037BD401CA4
:10A30000002803D0012801D0102807D3102804D337
:10A31000D148016831F004010160022070473EB568
:10A320000C0040218DF8001001008DF80110010093
:10A3300009B2090A8DF802106D460021E97001008A
:10A3400009B2B1F5905F2BD1FBF7A0FF2871000A8D
:10A35000E871C1480068C0F38000002802D0FF20E7
:10A3600068710BE0DFF8100900EB840151F8081C5C
:10A370006971002100EB840040F8081C032C01D116
:10A3800033206871DFF80007204410F8020CA87130
:10A39000DFF8E80701688C422FD1002101602CE032
:10A3A00042F2010100B288421CD1DFF8CC07204400
:10A3B00010F8020C2871A8480068C0F3800000283B
:10A3C00002D0FF20687101E0002068710020A871B0
:10A3D0000020E871DFF8A80701688C420DD1002148
:10A3E00001600AE04FF4A05080B233212971352179
:10A3F00069710100090AA971E8712200D2B26946A7
:10A40000002006F0EAF837BD7CB505000C004020BE
:10A410008DF800006E467570280000B2000A8DF8B5
:10A42000020000208DF80300280041F2010100B273
:10A4300088420ED15FF0FF30F7F7F0F80100090E07
:10A4400031710100090C71710100090AB171F071DB
:10A4500072E0280041F2030100B2884211D15FF09E
:10A46000FF3040F2FF11F7F7ECF80200120E3271E4
:10A470000200120C7271020092B2120AB271F071F3
:10A480005AE0280041F2050100B2884216D15FF07F
:10A49000FF3040F2FF11F7F7D4F802000B001A0E5C
:10A4A0000023327102000B001A0C002372710200AB
:10A4B0000B001A0A0023B271F1713DE0280041F24D
:10A4C000040100B288420CD1FEF71FFC0100090E06
:10A4D00031710100090C71710100090AB171F0714B
:10A4E0002AE01E20F9F71EFD092802D14FF4805002
:10A4F00019E01E20F9F716FD042802D14FF4A050F0
:10A5000011E01E20F9F70EFD0A2802D14FF4A850E1
:10A5100009E01E20F9F706FD072802D141F20240AA
:10A5200001E041F2034080B2332131713521717174
:10A530000100090AB171F0712200D2B2694601200E
:10A5400006F04BF8280000B200F01CFBDFF81C17E7
:10A55000088073BD81790902C0790143B1F5A05F1C
:10A5600001D104202FE041F20140814201D10620B7
:10A5700029E041F20240814201D1072023E041F26B
:10A580000340814201D108201DE0B1F5805F01D177
:10A59000092018E040F65110814207D040F65A10C9
:10A5A000814203D040F65B10814201D105200AE0D0
:10A5B000B1F5804F01D1102005E0B1F5A85F01D1C0
:10A5C0000A2000E0002070470020DFF890160860A5
:10A5D0002148016831F0020101600220DFF8901685
:10A5E000087000202BE00021DFF8842511540021A1
:10A5F000DFF88C2442F8201000220023DFF88414B6
:10A6000001EBC001C1E900230021DFF8DC2542F89D
:10A610002010FF21DFF870241154DFF85C2511545D
:10A620000021DFF8542642F82010DFF848150022F8
:10A6300001F81020002201EB40014A70401C0E2856
:10A64000D1D30020DFF8A41508600020DFF8101631
:10A650000860704700000000882B00208C2B002031
:10A66000A02B0020A42B00202DE9FE435FF080707A
:10A670000021F6F78BFFDFF814442068C0F3400098
:10A68000002800F09881684605F08BFF002800F054
:10A690006881DFF8C8753968884240F059813868A8
:10A6A000F8F757F9DFF8B0150A68104308603D68FD
:10A6B000AD1E6E46B17809027078014342F2010086
:10A6C00081420BD13868DFF8B8140968884200F07D
:10A6D0003F813079DFF8A014485539E141F2030099
:10A6E000814254D1DFF89C0300EBC501D1E900237E
:10A6F00032F0FF3233F0000300EBC501C1E9002363
:10A7000000EBC501D1E90089327900231B0643EA39
:10A710001223120658EA020259EA030300EBC501AC
:10A72000C1E9002300EBC501D1E90089727900235A
:10A730001B0443EA1243120458EA020259EA0303D3
:10A7400000EBC501C1E9002300EBC501D1E9008997
:10A75000B27900231B0243EA1263120258EA020292
:10A7600059EA030300EBC501C1E9002300EBC50171
:10A77000D1E9002396F807805FF0000952EA080249
:10A7800053EA090300EBC500C0E90023E0E041F211
:10A79000050081427AD1BB4800EBC501D1E9002315
:10A7A00032F0000233F0FF3300EBC501C1E90023B2
:10A7B00000EBC501D1E9008932790023130600229C
:10A7C00058EA020259EA030300EBC501C1E900237C
:10A7D00000EBC501D1E9008972790023130400223E
:10A7E00058EA020259EA030300EBC501C1E900235C
:10A7F00000EBC501D1E90089B279002313020022E0
:10A8000058EA020259EA030300EBC501C1E900233B
:10A8100000EBC501D1E9002396F807805FF000093D
:10A82000C1465FF0000852EA080253EA090300EB50
:10A83000C501C1E90023DFF8441309683A68914271
:10A8400000F0868000EBC501D1E9002312F0000280
:10A8500013F02003002B01D1002A03D001208A49E4
:10A86000485575E000EBC500D0E9000110F000008C
:10A8700011F00801002901D1002803D002208249EB
:10A88000485565E000208049485561E041F20100EB
:10A8900081422FD17A493079000641F8250051F8DC
:10A8A0002500727950EA024041F8250051F8250050
:10A8B000B27950EA022041F8250051F82520F079BC
:10A8C000024341F8252051F82500002808D03868B7
:10A8D000F8F73FF8DFF888130A681043086037E09C
:10A8E0003868F8F736F8DFF878130A6832EA0000BB
:10A8F00008602DE041F20400814219D1BA49307953
:10A90000000641F8250051F82500727950EA02400E
:10A9100041F8250051F82500B27950EA022041F8AB
:10A92000250051F82520F079024341F825200FE059
:10A93000B1F5805F0CD16846FFF70CFE8C49485595
:10A940008C48317900F81510717900EB45004170A1
:10A950003868FFF7D4FC3860206830F002002060CF
:10A960007AE0F5F7D1FBC3490968401AC82873D3C8
:10A97000BA4D2868F7F7EDFFB7490A6832EA0000D8
:10A98000086000207A492A68114401F8020CFF206F
:10A9900079492A68114401F8020C3B492A6811449C
:10A9A00001F8020C2868FFF7AAFC2860206830F044
:10A9B0000200206050E0A74D28684FF6FC71084265
:10A9C0004AD0F5F7A1FBA84E3168401A0A2843D3B4
:10A9D000F5F79AFB3060002704E03068FFF78FFC42
:10A9E00030607F1C0F2F37D29C4E3068F7F7B1FFD5
:10A9F00029680842F1D02068C0F38000002805D003
:10AA000031684FF49050FFF78AFC1DE058493068D8
:10AA1000084410F8020C002805D131684FF480502A
:10AA2000FFF77DFC10E03068084410F8020C102895
:10AA300005D1316842F20100FFF771FC04E0316892
:10AA40004FF49050FFF76BFC206850F0020020603C
:10AA5000F5F75AFB874908607E4800687E49096817
:10AA6000884204D0206850F02000206003E0206875
:10AA700030F020002060BDE8F7830000902B00201C
:10AA800018270020D824002094290020882B00209B
:10AA90003EB5574C206830F0200020605FF0807099
:10AAA0000021F6F7BFFD2068C0F34000002843D026
:10AAB000684605F076FD00282FD069468A78120294
:10AAC00049780A43B2F5805F17D1644D29688842FE
:10AAD00013D16846FFF73EFD00280AD02868F7F733
:10AAE00038FF5C490A68104308600868C04363493E
:10AAF000086000205B4908600AE05A480168491C68
:10AB000001600068032803DA54480168491E0160A7
:10AB1000206830F00200206029E0F5F7F5FA554989
:10AB20000968401AC82822D3206830F0020020604B
:10AB300000204C4908601AE0484801680F2910D2EB
:10AB40000168491C016001684FF48050FFF7E7FB82
:10AB5000206850F002002060F5F7D6FA45490860F9
:10AB600005E0206850F008002060FFF72DFD37BD9C
:10AB700084290020E8280020A4290020B82B0020E8
:10AB8000B42B00200100080000B2B0F5805F05D1B1
:10AB900041F205001421334A116023E041F205001F
:10ABA0000A00030012B29A4202D141F2030019E0F6
:10ABB0000A0041F2030312B29A4202D141F20100AB
:10ABC00010E041F20402130009B299420AD025496B
:10ABD0000B68142B03DB00200860100002E00A68F9
:10ABE000521C0A6000B2704750270020A82B00209A
:10ABF000882B002080B55920F9F794F9204909687D
:10AC000002291ED3012808D100202021F6F70AFDD1
:10AC100000200821F6F7BAFC1BE0022808D100202A
:10AC20000821F6F7FFFC00202021F6F7AFFC10E02A
:10AC300000200821F6F7AAFC00202021F6F7A6FC48
:10AC400007E000200821F6F7A1FC00202021F6F7FC
:10AC50009DFC01BDA02B0020A82B0020B02B0020C4
:10AC6000AC2B0020982B00209C2B0020D62D002000
:10AC7000DF2D0020942B002088270020A42B00200B
:10AC80008C2B002038B5DFF8A04920684008400030
:10AC90002060206830F0020020600020DFF88C196E
:10ACA0000860206830F0040020608021DFF880090F
:10ACB000F5F770F90020DFF87C190860206850F083
:10ACC00008002060DFF8705980212800F5F762F94C
:10ACD0000020DFF86819086040212800F5F75AF9CC
:10ACE0000020DFF85C190860DFF85809FAF7A4FFC4
:10ACF00041F60500F5F7A0F941F60540F5F79CF996
:10AD000080215FF04020F5F767F940215FF0402097
:10AD1000F5F762F9DFF83059002280212800FAF7B0
:10AD2000F3FE4FF47A6280212800FAF703FF8021B6
:10AD30002800FAF709FF01220C212800FAF732FF58
:10AD40004FF4007280212800FAF747FF00F0D0FB93
:10AD50001021DFF8F808F5F7F5F8DFF8F4580321CB
:10AD60002800F7F7DDFE03212800F7F7ECFE0123AA
:10AD7000002203212800F7F7EEFE6C2300220321B6
:10AD80002800F7F712FF03212800F7F7D7FE40212C
:10AD90002120FBF706F903212800F7F7CBFE03215A
:10ADA0002800F7F7C0FE2120FBF70CF9032128004B
:10ADB000F7F75BFFDFF89C582800FAF73DFF280003
:10ADC000FAF754FFDFF8905832212800F5F7CFFF4B
:10ADD0000122FF212800F6F707F8DFF88028FF217D
:10ADE0002800F6F70DF8A0215620FBF7DAF801212C
:10ADF0002800F6F721F801212800F6F722F856205E
:10AE0000FBF7E0F8FF212800F5F7A2FF0020DFF8AC
:10AE1000501808700020DFF84C180870F5F774F926
:10AE2000DFF844180860F5F76FF9DFF8401808609C
:10AE3000206850F00100206031BD10B5DFF8E84710
:10AE40002078C0075AD5DFF818080078002812D0FB
:10AE5000022807D003D304280AD006D30EE000F05E
:10AE600073F911E000F0F7F80EE000F0D5F90BE00F
:10AE700000F010FA08E000F0D0F805E04FF40050C0
:10AE8000F6F7A3FB00F034FB4D20F9F74BF810F078
:10AE90000F0F0ED15FF40000F6F75DFB4FF480500A
:10AEA0000021F6F773FB4FF400600021F6F76EFB0C
:10AEB00024E0DFF878070068012804D02068C0F398
:10AEC0004000002805D04FF400600021F6F7AAFBEF
:10AED00004E04FF400600021F6F758FB2068C0F34F
:10AEE0008000002805D04FF480500021F6F79AFB2F
:10AEF00004E04FF480500021F6F748FB10BDDFF866
:10AF0000641708707047DFF85C070078704780B5F9
:10AF1000DFF850070178012922D1DFF844070178D2
:10AF200001290ED1DFF80007007810F0060F04D1D8
:10AF3000DFF8F8060068012801D1012043E0002075
:10AF400041E00078002809D14D20F8F7EBFF10F020
:10AF50000F0F01D1002036E0022034E0022032E061
:10AF60000178022922D1DFF8F806017802290ED1F2
:10AF7000DFF8B406007810F0060F04D1DFF8AC0655
:10AF80000068012801D101201DE000201BE00078AD
:10AF9000002809D14D20F8F7C5FF10F00F0F01D19F
:10AFA000002010E002200EE002200CE000780328D0
:10AFB00001D1022007E0DFF8A8060078002801D1BF
:10AFC000002000E00220C0B202BD1CB5DFF88046C0
:10AFD0006A4603212000F7F735FEDFF89406009952
:10AFE0000160006840F6A171884205D30120DFF8B6
:10AFF0003C16086000F07CFA03212000F7F79AFD68
:10B0000013BD80B50321DFF84806F7F72EFE0121B6
:10B01000DFF84406F5F715FF01BD80B500F068FACA
:10B020004D20F8F77FFF10F00F0F13D0DFF8340634
:10B030000178012902D00178032904D10220DFF828
:10B040002016087006E00078022803D10120DFF8FE
:10B050001016087001BD10B500F07BFA012872D1FE
:10B06000DFF800060178012902D0017803291AD1FE
:10B0700001210170DFF8B005016831F002010160C3
:10B08000016831F00401016000F032FA4D20F8F758
:10B0900049FF10F0C00F01D100F0C6F90320DFF81E
:10B0A000C01508704FE00078002806D100F020FAA3
:10B0B0000020DFF8AC15087045E000F03DF94D20A8
:10B0C000F8F730FF10F0C00080283AD14D20F8F793
:10B0D00029FF10F00F0F34D04FF480400021F6F715
:10B0E000B0FA002901D1002808D05FF0804000218B
:10B0F000F6F7A7FA002924D1002822D1DFF8284545
:10B100002068C0F3400000281BD1DFF86405006808
:10B1100040F26D21884206D300F0EAF9206850F031
:10B12000020020600FE0DFF84C050068002802D123
:10B1300000F0ACF907E0F4F7E7FFDFF8301508603E
:10B1400001E000F0D5F910BD80B500F002FA012849
:10B1500061D14D20F8F7E6FE10F00F0F03D100206B
:10B16000DFF800150870DFF8FC040178022930D1FF
:10B17000DFF8B404016831F002010160016831F0C8
:10B180000401016000F0B4F94FF480400021F6F7AB
:10B1900058FA002901D1002814D05FF08040002126
:10B1A000F6F74FFA002901D100280BD04D20F8F70F
:10B1B000B9FE10F0C000802804D00220DFF8A014EF
:10B1C000087028E00420DFF89814087000F05EF999
:10B1D00021E00178032910D10121017000F088F9E4
:10B1E0004D20F8F79FFE10F0C00F14D100F01CF9AD
:10B1F0000320DFF86C1408700DE00078002806D1F9
:10B200000020DFF85C14087000F072F903E000F031
:10B21000CFF800F06DF901BD10B5DFF80C442068DF
:10B22000C0F3C000002808D04FF480400021F6F79A
:10B2300008FA002901D100280DD02068C0F3C00011
:10B2400000281DD14FF480400021F6F7FAF90029BB
:10B2500001D1002814D000F04BF9F4F755FFDFF8C6
:10B26000081408604D20F8F75DFE10F00F0F03D1B1
:10B27000012000F0D0F90CE0022000F0CCF908E049
:10B2800000F042F8012804D100F032F9012000F06A
:10B29000C2F910BD10B5DFF890432068C0F3C000BC
:10B2A000002808D04FF480400021F6F7CAF90029A1
:10B2B00001D100280DD02068C0F3C000002813D1B0
:10B2C0004FF480400021F6F7BCF9002901D1002895
:10B2D0000AD000F00DF9F4F717FFDFF88C130860BF
:10B2E000012000F098F90EE000F00EF801280AD1D4
:10B2F0004D20F8F717FE10F0C00F01D100F0F8F85C
:10B30000022000F088F910BD10B54D20F8F70AFEB4
:10B3100010F0C00F02D04FF47A7401E04FF41674AD
:10B32000F4F7F2FEDFF844130968401AA04201D393
:10B33000012000E0002010BD80B52020F8F7B9FD05
:10B3400000280FD04D20F8F7EDFD10F00F0F09D0B9
:10B35000F6F74BFB002805D04FF48040F9F7BBFD12
:10B36000002801D0012008E04FF40040F9F7B3FDB8
:10B37000002801D1012000E00020012809D1F4F7C4
:10B38000C3FEBD490860A848016831F004010160AE
:10B390000DE0F4F7B9FEB8490968401A40F2E93106
:10B3A000884204D3A048016851F00401016001BD46
:10B3B00080B52020F8F77DFD00280FD04D20F8F74C
:10B3C000B1FD10F00F0F09D0F6F70FFB002805D0E4
:10B3D0004FF48040F9F77FFD002801D0012008E0FC
:10B3E0004FF40040F9F777FD002801D1002000E07C
:10B3F0000120012809D1F4F787FE9F4908608A4897
:10B40000016831F0040101600DE0F4F77DFE9A4916
:10B410000968401A40F2E931884204D38248016841
:10B4200051F00401016001BD38B5854C0020206059
:10B43000002082490860844D002208212800FAF784
:10B44000A8FB4FF480400021F6F7FBF8002901D15A
:10B45000002806D04FF47A6282212800FAF777FBA1
:10B4600005E04FF4486282212800FAF770FB0122C0
:10B4700004212800FAF78DFB40202060F4F744FEF9
:10B480007A49086001207B49086031BD38B5002049
:10B490006B490860694C002020606B4D002204213C
:10B4A0002800FAF776FB4FF480400021F6F7C9F840
:10B4B000002901D1002806D04FF47A6283212800A8
:10B4C000FAF745FB05E04FF4486283212800FAF7BC
:10B4D0003EFB012208212800FAF75BFB8020206058
:10B4E000F4F712FE6149086001206249086031BD2D
:10B4F00010B50020524908600020504908604B48B0
:10B500000068012805D04D20F8F70CFD10F00F0F52
:10B5100005D100220C214C48FAF73BFB11E04A4CC4
:10B520004FF47A6282212000FAF711FB4FF47A621D
:10B5300083212000FAF70BFB01220C212000FAF7EF
:10B5400028FB00204B490860F4F7DEFD47490860FE
:10B5500010BD10B5344C2068C0F3C000002808D0DE
:10B560004FF480400021F6F76CF8002901D1002843
:10B570000DD02068C0F3C000002846D14FF48040B1
:10B580000021F6F75EF8002901D100283DD02748B8
:10B590000068012801D101203CE0364800680028FD
:10B5A00010D14FF480400021F6F74BF8002901D16B
:10B5B000002803D000201F49086007E080201D49B3
:10B5C000086003E0F4F7A0FD27490860FFF790FF4B
:10B5D000F4F79AFD24490968401A192813D34FF447
:10B5E00080400021F6F72DF8002901D1002804D071
:10B5F000206850F00800206003E0206830F0080068
:10B600002060012006E0002004E0F4F77DFD1649EB
:10B610000860012010BD80B511490870F4F774FD71
:10B620001549086001BD0000D02B0020D42B00205C
:10B63000004006400042064000C0054000C20540F0
:10B6400000C10540014000F0009002400070004041
:10B6500000800340040400F000400340400D03005C
:10B66000E32D0020E42D0020E82B0020DC2B00201F
:10B67000E42B0020D82B0020E02B002010B5B34C89
:10B68000002020600120A060F4F73EFDB049086072
:10B690004FF48040F5F7C2FF002805D00A2020753E
:10B6A000802000F077FE04E000202075072000F0E5
:10B6B00071FE4FF480600021F5F768FF4FF40070D1
:10B6C0000021F5F763FF0020206300206063012064
:10B6D000206010BD10B59D4C2068002800F0FA8055
:10B6E00000F038F96075607D032802D1A07D032841
:10B6F0000BD1607D042802D1A07D042805D1607D96
:10B7000002280CD1A07D022809D05FF0FF30F5F7A8
:10B7100022FF00206063002020630020E062607D43
:10B72000032802D0F4F7F0FCA061607D022811D15B
:10B7300080200021F5F776FF40200021F5F726FF55
:10B7400004200021F5F722FF4FF480700021F5F767
:10B750001DFF3AE0607D032811D180200021F5F71C
:10B7600015FF40200021F5F75DFF04200021F5F7CB
:10B770000DFF4FF480700021F5F708FF25E08020D1
:10B780000021F5F703FF40200021F5F7FFFE13200D
:10B79000FAF787FD002804D104200021F5F7F6FE12
:10B7A00003E004200021F5F73DFF1620FAF779FDAC
:10B7B000002805D14FF480700021F5F7E7FE04E082
:10B7C0004FF480700021F5F72DFFF0F750FE0028B0
:10B7D00005D15FF480300021F5F724FF04E05FF429
:10B7E00080300021F5F7D2FEF0F745FE002805D1A4
:10B7F0004FF400400021F5F715FF04E04FF400403E
:10B800000021F5F7C3FEA06801280FD10023002214
:10B8100000210020F0F7ECFDF4F776FC4C490968B4
:10B82000401AC82856D30020A06053E0207D0A2883
:10B830004EDAF4F79DFC012806D1207D012803D0C3
:10B84000200005F0D3FF43E0F5F79AF8012803D173
:10B85000200005F0F1FF3BE05FF400000021F5F768
:10B8600095FE207D032803D1200006F093F82FE0F9
:10B87000207D022803D1200006F0C2FA28E0207DB6
:10B88000082803D1200006F09DFD21E0207D072837
:10B8900003D1200007F052F81AE0207D002803D1E0
:10B8A000200007F0CBFA13E0207D012803D120000F
:10B8B00005F020FD0CE0207D092803D1200007F0D1
:10B8C00029FB05E00220F5F770FE200005F08EFF51
:10B8D000607DA07510BD1D48007D70471B48407DF0
:10B8E000704710B5194C207D022808D0207D032810
:10B8F00005D0207D012802D0207D00280AD14FF4F8
:10B9000080400021F5F79DFE002901D1002801D0DB
:10B91000606800E0002010BD80B5FFF7DFFF02285F
:10B9200003D10A4807F0DBFA0DE05FF0FF30F5F7CE
:10B9300075FE002803D0054805F058FF03E0642198
:10B94000024806F00FFD01BD00000000C8260020DF
:10B95000FC2B002010B50A20FAF7A3FC012801D126
:10B9600002241CE01320FAF79CFC012801D10024DA
:10B9700015E01420FAF795FC012801D103240EE00C
:10B980001520FAF78EFC012801D1042407E01A20C3
:10B99000FAF787FC012801D1012400E00024572098
:10B9A000F8F7C0FA012805D15920F8F7BBFA0028AA
:10B9B00000D002242000C0B210BD000080B50020DD
:10B9C000DFF8881608700821DFF88406F4F7E2FA39
:10B9D0000820DFF8801608600120DFF87C16086078
:10B9E0000020DFF8781608700020DFF87416087061
:10B9F00001BD80B5DFF860060068012840F01681BF
:10BA0000DFF848160878002802D100F06AF915E03E
:10BA10000878012802D100F07DF90FE008780228AB
:10BA200002D100F022FA09E0002008700820DFF8B7
:10BA3000241608604FF48050F5F7C7FD2020F8F772
:10BA400071FA30F08000482807D04E2805D05A28D7
:10BA500003D04FF48060F5F77EFD2620F8F762FAF8
:10BA600030F08000482807D04E2805D05A2803D04F
:10BA70004FF40060F5F76FFD2820F8F753FA30F027
:10BA80008000482800F09A802820F8F74BFA30F020
:10BA900080004E2800F092802820F8F743FA30F01A
:10BAA00080005A2800F08A802A20F8F73BFA30F00C
:10BAB0008000482800F082802A20F8F733FA30F01E
:10BAC00080004E287AD02A20F8F72CFA30F0800037
:10BAD0005A2873D02C20F8F725FA30F08000482837
:10BAE0006CD02C20F8F71EFA30F080004E2865D07C
:10BAF0002C20F8F717FA30F080005A285ED02E205C
:10BB0000F8F710FA30F08000482857D02E20F8F7C8
:10BB100009FA30F080004E2850D02E20F8F702FAB3
:10BB200030F080005A2849D03420F8F7FBF930F083
:10BB30008000482842D03420F8F7F4F930F0800033
:10BB40004E283BD03620F8F7EDF930F08000482839
:10BB500034D03620F8F7E6F930F080004E282DD0AA
:10BB60003020F8F7DFF930F08000482826D0302068
:10BB7000F8F7D8F930F080004E281FD03020F8F7C1
:10BB8000D1F930F080005A2818D03220F8F7CAF9DD
:10BB900030F08000482811D03220F8F7C3F930F097
:10BBA00080004E280AD03220F8F7BCF930F080002F
:10BBB0005A2803D05FF40020F5F7CDFC8020F8F779
:10BBC00078F900282DD04FF48060F5F727FD002884
:10BBD00008D04FF48060F5F7BEFC5FF08060002174
:10BBE000F5F720FD4FF40060F5F718FD002808D0A8
:10BBF0004FF40060F5F7AFFC5FF080600021F5F7CF
:10BC000011FD5FF40020F5F709FD00280ED05FF468
:10BC10000020F5F7A0FC5FF080600021F5F702FD41
:10BC200004E05FF080600021F5F7B0FC01BDDFF8B3
:10BC300028040068002801D100200CE0DFF80C0483
:10BC40000078002806D1DFF814040078002801D11C
:10BC5000002000E001207047DFF8FC0300680028A6
:10BC600001D1002007E0DFF8E4030078012801D1CA
:10BC7000012000E000207047DFF8E01308707047F3
:10BC8000DFF8DC030178022909D14E20DFF8D41354
:10BC900008605FF0FF30DFF8D013086020E0017823
:10BCA000012909D14820DFF8C01308605FF0FF3098
:10BCB000DFF8B013086013E00078032808D14E20A5
:10BCC000DFF8A01308604820DFF89C13086007E045
:10BCD0005FF0FF30DFF88C130860DFF88C1308602A
:10BCE000704710B50820DFF86C130860DFF86C436C
:10BCF000207800280DD05FF000700021F5F7A1FC3E
:10BD0000002904D1002802D100F081F901E00020CF
:10BD1000207010BD10B50020DFF838130860002433
:10BD2000FFF7AEFF2021012000F01DF9012801D10D
:10BD300054F001042221022000F015F9012801D15C
:10BD400054F002042421042000F00DF9012801D14F
:10BD500054F004042621082000F005F9012801D13F
:10BD600054F008042821102000F0FDF8012801D12A
:10BD700054F010042A21202000F0F5F8012801D108
:10BD800054F020042C21402000F0EDF8012801D1CE
:10BD900054F040042E21802000F0E5F8012801D164
:10BDA00054F0800430214FF4807000F0DCF801285A
:10BDB00001D154F4807432214FF4007000F0D3F8B4
:10BDC000012801D154F4007434214FF4805000F064
:10BDD000CAF8012801D154F4806436214FF4005090
:10BDE00000F0C1F8012801D154F4006440F6FF705E
:10BDF000844203D099490878002802D100F019F94B
:10BE000032E0974800780978884202D000F0FFF8C5
:10BE10002AE0F4F779F995490968401A40F6A171CA
:10BE2000884221D300F005F98020F8F742F8002875
:10BE300005D05FF080600021F5F7F4FB14E0E00727
:10BE400003D44FF48060F5F7D0FB200703D44FF400
:10BE50000060F5F7CAFB14F47F64B4F57F6F03D07C
:10BE60005FF40020F5F7C1FB10BD10B5082079493B
:10BE7000086000242021012000F09FF8012801D152
:10BE800054F001042221022000F097F8012801D18A
:10BE900054F002042421042000F08FF8012801D17D
:10BEA00054F004042621082000F087F8012801D16D
:10BEB00054F008042821102000F07FF8012801D157
:10BEC00054F010042A21202000F077F8012801D135
:10BED00054F020042C21402000F06FF8012801D1FB
:10BEE00054F040042E21802000F067F8012801D191
:10BEF00054F0800430214FF4807000F05EF8012887
:10BF000001D154F4807432214FF4007000F055F8E0
:10BF1000012801D154F4007434214FF4805000F012
:10BF20004CF8012801D154F4806436214FF40050BC
:10BF300000F043F8012801D154F400644748007828
:10BF4000002801D000F063F8F4F7DEF847490968EB
:10BF5000401AC92803D240F6FF70844202D1002063
:10BF60003A49087010BD38B504000D002800C0B271
:10BF7000F7F7D8FF30F080003A490968884211D0BD
:10BF80002800C0B2F7F7CEFF30F080005A2809D061
:10BF90002800C0B2F7F7C6FF30F0800032490968C8
:10BFA000884208D12000F8F796FF002801D0012030
:10BFB00002E0002000E0012032BD38B504000D0091
:10BFC0002800C0B2F7F7AEFF30F0800025490968BD
:10BFD000884211D02800C0B2F7F7A4FF30F08000EB
:10BFE0005A2809D02800C0B2F7F79CFF30F0800033
:10BFF0001D490968884208D12000F8F76CFF002825
:10C0000001D0002002E0012000E0012032BD80B517
:10C0100001200E4908701148007811490870F4F7A2
:10C0200073F8124908605FF080600021F5F7AEFAFE
:10C0300001BD80B50220054908700020074908703D
:10C04000F4F762F80949086001BD0000DE2D002008
:10C050000030064020300640282B0020DC2D002038
:10C06000DD2D0020302B0020342B00202C2B002035
:10C0700010B5DFF89C4BF4F747F8A061F4F744F8EB
:10C08000DFF8901B0860F4F73FF8DFF88C1B0860BE
:10C090000020206000202071DFF8800B016851F043
:10C0A0000101016010BD10B5DFF8700B0078C0070A
:10C0B00040F16781DFF8D44B5FF0E040F8F70BFF09
:10C0C00020605FF0E040F8F70BFFDFF8C41B08606A
:10C0D0000121032002F077FF206810F0E04F04D028
:10C0E000F4F712F8DFF8301B0860F4F70DF8DFF80A
:10C0F000281B0968401ADFF89C1B884203D3642080
:10C10000DFF80C1B0860DFF8081B0868642802D100
:10C1100000F07DF935E10868012802D100F0C6F988
:10C120002FE10868652802D100F0DEFA29E10868ED
:10C13000662802D100F07CFB23E10868672802D161
:10C1400000F000FA1DE10868682802D100F044FA06
:10C1500017E10868692802D100F083FA11E1086844
:10C160006B2802D100F0C7FB0BE108686C2802D1F4
:10C1700000F0F6FB05E108686D2802D100F02BFC09
:10C18000FFE008686E2802D100F0A8FCF9E008681A
:10C190006F2802D100F0D5FCF3E00868702802D1C6
:10C1A00000F002FDEDE00868712802D100F038FDD2
:10C1B000E7E00868722802D100F013FEE1E00868A9
:10C1C000CF2803D1092000F03FFFDAE00868D0282B
:10C1D00003D1092001F01EF9D3E00868D12803D16A
:10C1E0000A2000F031FFCCE00868D22803D10A20F1
:10C1F00001F010F9C5E00868C92803D1052000F056
:10C2000023FFBEE00868CA2803D1052001F002F927
:10C21000B7E00868CB2803D1082000F015FFB0E094
:10C220000868CC2803D1082001F0F4F8A9E00868D8
:10C23000CD2802D100F029FEA3E00868CE2802D163
:10C2400000F0C2FE9DE008686A2802D101F085F97D
:10C2500097E008687D2802D101F07AFA91E0086839
:10C26000D42802D101F030FB8BE00868D52802D138
:10C2700001F07AFB85E00868D62802D101F0F5FBD1
:10C280007FE00868D82802D101F03EFC79E0086818
:10C29000D92803D1012001F0B7FC72E00868DA2840
:10C2A00003D1022001F0B0FC6BE00868732802D1D2
:10C2B00000F0F2FC65E00868742802D100F03FFD50
:10C2C0005FE00868752803D1012000F0BDFE58E04A
:10C2D0000868772803D1022000F0B6FE51E0086814
:10C2E000792803D1032000F0AFFE4AE008687B28DC
:10C2F00003D1042000F0A8FE43E00868762803D1AB
:10C30000012001F087F83CE00868782803D102207A
:10C3100001F080F835E008687A2803D1032001F0A5
:10C3200079F82EE008687C2803D1042001F072F827
:10C3300027E00868D32802D101F074FA21E00868E8
:10C34000D72802D100F0E2FD1BE00868DB2802D10B
:10C3500001F065F915E00868B0F5967F02D101F0AB
:10C36000F8FC0EE00868002802D100F01BF808E095
:10C370000868B0F5C87F02D101F030FD01E064200B
:10C38000086010BDDFF8880800797047DFF8800882
:10C3900040697047DFF82C1C08707047DFF8240CE8
:10C3A0000078704738B5DFF8684800202071DFF862
:10C3B000DC58286810F0E040B0F1E04F07D0F3F708
:10C3C000A3FEA169401A41F28831884219D2286837
:10C3D00010F0E040B0F1E04F0DD1F3F795FEDFF83B
:10C3E00034180968401A41F2883188420BD34FF45F
:10C3F000C87020600AE0F3F787FEDFF818180860BD
:10C4000001E06420206002F0B5FB606131BD10B531
:10C41000DFF8FC4702202071DFF874080068C000D4
:10C4200008D54020F7F745FD00283ED101F0FEFC7D
:10C4300020603AE0DFF85408006810F0C040B0F126
:10C44000C04F0DD101202060F3F75EFEB0F51670ED
:10C45000A061DFF8C807016851F00201016024E023
:10C460004FF40070F5F7DAF800281BD04FF4804045
:10C470000021F5F7E6F8002901D1002812D0F3F7E2
:10C4800043FEA169401AB0F5FA7F0ED3F3F73CFEE4
:10C49000A0616069802802D10020606105E08020F1
:10C4A000606102E002F0E9FA606110BD10B5DFF8EA
:10C4B000604702202071F3F727FEA169401AB0F50A
:10C4C000167F34D3F3F720FEA061DFF85017086819
:10C4D000C0F34000002819D1086850F0020008603D
:10C4E0005FF0FF30F5F79AF8002808D15FF0FF30D1
:10C4F00040F2FF11F5F7A5F802F007FB01E002F0AA
:10C50000E8FA012101F0B1FD606110E0086830F047
:10C51000020008605FF0FF30F5F780F8002803D0D4
:10C5200047F65010606102E047F238706061DFF852
:10C530005C07006810F0C040B0F1C04F01D064202B
:10C54000206010BD38B51E20F7F7ECFC072805D099
:10C5500001F06CFCDFF8B81608603CE0DFF83057FB
:10C560002868C00005D501F061FCDFF8A41608605A
:10C5700031E0DFF818070068C00008D5DFF8904602
:10C5800043F65400606101F073FC206023E0DFF8A3
:10C590008046052020710220F7F78BFCE0602868B8
:10C5A00010F0C04F07D0E068002802D00020E06003
:10C5B00001E00120E060E068002806D0062060610C
:10C5C00000210220F7F779FC05E05B206061002183
:10C5D0000220F7F78CFC31BD1CB51E20F7F7A2FC3A
:10C5E000072805D001F022FCDFF82416086037E0A8
:10C5F000DFF89C060068C00005D501F017FCDFF8E5
:10C60000101608602CE0DFF884060068C00008D52A
:10C61000DFF8FC4543F67800606101F029FC2060FA
:10C620001EE0DFF8EC45062020715E20F7F77AFC6B
:10C63000401CE060012001900020009001230322B3
:10C640000121E06801F03DFCE0600121E06801F0BB
:10C650000CFD60610022E168491E5E20F7F705FDD0
:10C6600013BD38B5DFF828562868C00005D501F09D
:10C67000DDFBDFF89C15086035E0DFF81006006888
:10C68000C00008D5DFF8884545F23700606101F049
:10C69000EFFB206027E0DFF87845072020715FF08E
:10C6A0000040F7F706FCE060286810F0C04F07D0A4
:10C6B000E068002802D00020E06001E00120E06096
:10C6C000E068002808D044F20600606100215FF0B5
:10C6D0000040F7F7F2FB06E00620606100215FF002
:10C6E0000040F7F704FC31BD1CB5DFF8A405016874
:10C6F000C9002FD5DFF81845E068216988421CD0B1
:10C70000E068012801D1092014E0E068022801D185
:10C7100004200FE0E068032801D108200AE0E06867
:10C72000042801D1072005E0E068052801D10A208E
:10C7300000E000200021F7F761FBE068642805D1E4
:10C740004FF4967020600020E06070E001F06EFB16
:10C7500020606CE0DFF834150A68D20005D4DFF8F9
:10C76000B0442268A3689A423AD0DFF8A44443F662
:10C77000711060611E20F7F7D5FB092802D1012056
:10C78000E06021E01E20F7F7CDFB042802D1022053
:10C79000E06019E01E20F7F7C5FB082802D103204E
:10C7A000E06011E01E20F7F7BDFB072802D104204E
:10C7B000E06009E01E20F7F7B5FB0A2802D105204A
:10C7C000E06001E06420E060E0682061E0686428E7
:10C7D00003D001F04DFB206029E02068A06026E036
:10C7E00004222271E268642A11D145F25C4262613E
:10C7F0000268920002D50A68520005D509688900CE
:10C8000015D40068400012D50120E0600FE001203F
:10C81000019000200090012305220121E06801F031
:10C8200050FBE0600121E06801F01FFC606113BD76
:10C8300070B5DFF85C442068C0000ED5DFF8D04347
:10C84000E068012805D11E20F7F76CFB0021F7F7FF
:10C85000D5FA01F0EBFA20604CE0DFF8305428689C
:10C86000C00005D4DFF8A8633068B168884216D0EC
:10C87000DFF89C4345F6716060615FF00040002185
:10C88000F4F7DFFE002901D1002802D00020E0608B
:10C8900001E00120E06001F0EBFA20602AE00320D3
:10C8A00030715FF000400021F4F7CBFE002904D185
:10C8B000002802D10120F06013E02068800002D53A
:10C8C0002868400005D5286880000AD42068400008
:10C8D00007D5F068002802D10120F06001E00020B7
:10C8E000F060F068002803D145F25C40706101E01F
:10C8F0006E20706170BD1CB5DFF894030068C00045
:10C9000004D501F093FAC249086028E0DFF87C03FF
:10C910000068C00007D5BE4C47F27730606101F077
:10C92000A7FA20601BE0BA4C092020713820F7F7E5
:10C93000F9FAE060002001900120009001231E22FE
:10C940000021E06801F0BDFAE0600121E06801F03B
:10C950008CFB60610022E1683820F7F786FB13BD8D
:10C9600038B5CB4D2868C00004D501F05FFAA8495E
:10C9700008602FE0C5480068C00007D5A44C47F602
:10C980006D10606101F074FA206023E0A04C0A2071
:10C9900020711020F7F78DFAE060286810F0C04F82
:10C9A00007D0E068002802D00020E06001E001200C
:10C9B000E060E068002806D06E2060610021102051
:10C9C000F7F77BFA06E045F25C4060610021102039
:10C9D000F7F78DFA31BD7CB5AD4C2068C00004D5A9
:10C9E00001F024FA8A49086077E0A8480068C0008E
:10C9F00007D5874C47F25430606101F039FA206066
:10CA00006BE0834D0B2028713920F7F78BFAE86033
:10CA1000E8683C2823D2287BC00713D4002001906B
:10CA20000120009002233C220021E86801F049FA2D
:10CA3000E860E8683C2833D20121E86801F015FB82
:10CA4000686145E0206810F0C04F04D03920F6F747
:10CA5000C3FAE860EDE747F6731068613DE0E86807
:10CA60000A21B0FBF1F201FB120000280BD10020DB
:10CA70000190012000900A23F0223221E86801F0A1
:10CA800020FAE860D5E7206810F0C04F04D03920C4
:10CA9000F6F7A2FAE860CCE747F6731068611CE08D
:10CAA000E8683C21B0FBF1F0E9683C22B1FBF2F30D
:10CAB00002FB13110A22B1FBF2F401F0AFFA0600F7
:10CAC000200001F0ABFA50EA062050F080006861C7
:10CAD0000022E9683920F7F7C8FA73BD1CB56C4825
:10CAE0000068C00004D501F0A1F94949086027E0B9
:10CAF00066480068C00007D5454C45F66D0060618A
:10CB000001F0B6F920601BE0414C0C202071182088
:10CB1000F7F708FAE060012001900020009001235F
:10CB20000A220121E06801F0CCF9E0600121E0680F
:10CB300001F09BFA60610022E1681820F7F795FA8E
:10CB400013BD1CB552480068C00004D501F06EF951
:10CB50002F49086027E04D480068C00007D52C4CDD
:10CB600045F66D40606101F083F920601BE0284CC0
:10CB70000D2020711620F7F7D5F9E0600120019013
:10CB80000020009001230A220121E06801F099F9B8
:10CB9000E0600121E06801F068FA60610022E1686C
:10CBA0001620F7F762FA13BD1CB539480068C000BB
:10CBB00004D501F03BF91649086027E033480068C6
:10CBC000C00007D5124C45F67100606101F050F9C4
:10CBD00020601BE00E4C0E2020710C20F7F7A2F90C
:10CBE000E060012001900020009001230A22012131
:10CBF000E06801F066F9E0600121E06801F035FAD3
:10CC000060610022E1680C20F7F72FFA13BD0000E5
:10CC1000CC280020A02A0020A42A00209C2A002042
:10CC20001CB51B480068C00005D501F0FFF8DFF80F
:10CC3000EC1B086029E015480068C00008D5DFF843
:10CC4000DC4B45F67140606101F012F920601CE098
:10CC5000DFF8C84B0F2020710E20F7F763F9E06072
:10CC6000012001900020009001230A220121E068A8
:10CC700001F027F9E0600121E06801F0F6F9606158
:10CC80000022E1680E20F7F7F0F913BDA82A002072
:10CC9000AC2A0020C02709003EB5DFF8844B20688D
:10CCA000C00005D501F0C2F8DFF8701B086045E050
:10CCB000DFF890030068C00008D5DFF8604B45F648
:10CCC0005060606101F0D4F8206037E0DFF84C5B21
:10CCD000102028710620F7F725F9E8600A20F7F7F9
:10CCE00021F9E96881420FD047F673106861206826
:10CCF00010F0C04F22D000210A20F6F729FC0021B5
:10CD00000620F6F725FC19E0012001900020009094
:10CD100001230A220121E86801F0D3F8E86001212B
:10CD2000E86801F0A2F968610022E9680620F7F7D7
:10CD30009CF90022E9680A20F7F797F937BD3EB55C
:10CD4000DFF8DC4A2068C00005D501F06FF8DFF895
:10CD5000CC1A086044E0BB480068C00008D5DFF882
:10CD6000BC4A47F25070606101F082F8206037E001
:10CD7000DFF8A85A112028710820F7F7D3F8E860E7
:10CD80000420F7F7CFF8E96881420FD047F6731017
:10CD90006861206810F0C04F22D000210820F6F70B
:10CDA000D7FB00210420F6F7D3FB19E00120019006
:10CDB0000020009001230A220121E86801F081F897
:10CDC000E8600121E86801F050F968610022E96833
:10CDD0000420F7F74AF90022E9680820F7F745F937
:10CDE00037BD3EB5DFF8384A2068C00005D501F0F0
:10CDF0001DF8DFF8281A086046E092480068C00075
:10CE000008D5DFF8184A47F67100606101F030F884
:10CE1000206039E0DFF8045A122028711A20F7F751
:10CE200081F8E8601C20F7F77DF8E96881421CD1A1
:10CE3000002001900120009001231E220121E868BA
:10CE400001F03FF8E8600021E86801F00EF950F0C9
:10CE5000800068610022E9681A20F7F706F90022CD
:10CE6000E9681C20F7F701F90EE047F673106861D6
:10CE7000206810F0C04F07D000211A20F6F768FB99
:10CE800000211C20F6F764FB37BD38B5DFF8905958
:10CE90002868C00005D500F0C9FFDFF880190860D8
:10CEA00033E068480068C00008D5DFF8704943F6F1
:10CEB0007870606100F0DCFF206026E0DFF85C49FC
:10CEC000132020714FF48060F6F7F3FFE0602868CC
:10CED00010F0C04F07D0E068002802D00020E060CA
:10CEE00001E00120E060E068002807D05B2060617D
:10CEF00000214FF48060F6F7E0FF06E00620606155
:10CF000000214FF48060F6F7F2FF31BD38B51E20E6
:10CF1000F7F708F8092804D01E20F7F703F80A28C5
:10CF200005D100F083FFDFF8F418086048E0DFF86F
:10CF3000F0582868C00005D500F078FFDFF8DC184D
:10CF400008603DE03F480068C00008D5DFF8CC48E5
:10CF500045F63760606100F08BFF206030E0DFF85D
:10CF6000BC48142020714FF40070F6F7A2FFE06077
:10CF7000FEF7B1FC296811F0C04F0ED00100C9B214
:10CF800007290AD0C0B2082807D0E068002802D0DC
:10CF90000020E06001E00120E060E068002807D0A8
:10CFA0006E20606100214FF40070F6F786FF07E005
:10CFB00045F25C40606100214FF40070F6F797FF86
:10CFC00031BD0000DA2D00201CB5DFF854080068E0
:10CFD000C00005D500F02AFFDFF84018086030E0F7
:10CFE00018480068C00008D5DFF8304847F673409D
:10CFF000606100F03DFF206023E0DFF8204815204D
:10D0000020713B20F6F78EFFE060012001900020A8
:10D010000090012302220021E06800F052FFE0604E
:10D02000E068002803D145F25C40606104E0012122
:10D03000E06801F01AF860610022E1683B20F7F730
:10D0400014F813BDA82A00203EB50400DFF8D0076D
:10D050000168C9000ED5DFF8C457E868296988421D
:10D0600004D02100C9B2E86801F07EF900F0DEFECC
:10D070002860CEE1DFF88C1B0968C90005D4DFF811
:10D080009C572968AA6891426ED0DFF8905720001B
:10D09000C0B201F012F8E860E86828612000C0B270
:10D0A000012803D143F60610686159E02000C0B2A0
:10D0B000022803D143F65B10686151E02000C0B242
:10D0C000032803D143F64F10686149E02000C0B245
:10D0D000042803D143F66610686141E02000C0B225
:10D0E000052803D147F20630686139E02000C0B25C
:10D0F000062803D147F25B30686131E02000C0B2FE
:10D10000072803D147F24F30686129E02000C0B200
:10D11000082803D147F25B30686121E02000C0B2EB
:10D120000B2803D140F25E60686119E02000C0B2B4
:10D130000C2803D147F65E10686111E02000C0B2F0
:10D14000092803D147F60610686109E0E4B20A2C09
:10D1500003D147F65B10686102E047F65010686142
:10D1600000F086FE286054E116212971E9686429DF
:10D1700080F03F81012001900020009001231F22B8
:10D180000021E86800F09DFEE8601E20F6F7CAFE68
:10D19000072804D01E20F6F7C5FE0A281ED1E8682D
:10D1A00009280FD0E8681B280CD0E868052809D0AA
:10D1B000E868062806D0E868022803D0E868032853
:10D1C00040F01281012001900020009001231F22D5
:10D1D0000021E86800F075FEE860E0E71E20F6F741
:10D1E000A1FE062840F0F4802000C0B20B2827D111
:10D1F000E868132818D0E868142815D0E8681128C2
:10D2000012D0E86812280FD0E86818280CD0E86817
:10D21000152809D0E8680E2806D0E8681D2803D034
:10D22000E8681C2840F0E080012001900020009078
:10D2300001231F220021E86800F043FEE860D7E7E1
:10D240002000C0B20C2833D1E8680F2824D0E86849
:10D25000102821D0E86819281ED0E8681A281BD0A9
:10D26000E8681D2818D0E868152815D0E8680E2849
:10D2700012D0E86813280FD0E86814280CD0E868AA
:10D28000112809D0E868122806D0E868182803D0C9
:10D29000E8681C2840F0A880012001900020009040
:10D2A00001231F220021E86800F00BFEE860CBE7B5
:10D2B0002000C0B202280ED02000C0B204280AD03C
:10D2C0002000C0B2062806D02000C0B2082802D034
:10D2D000E4B20A2C3ED1E8680F282FD0E868102865
:10D2E0002CD0E868192829D0E8681A2826D0E868E0
:10D2F0001D2823D0E868052820D0E86806281DD01E
:10D30000E86802281AD0E868032817D0E8681328CC
:10D3100014D0E868142811D0E86811280ED0E86805
:10D3200012280BD0E868152808D0E8680E2805D028
:10D33000E868182802D0E8681C2855D1012001901F
:10D340000020009001231F220021E86800F0B9FDB1
:10D35000E860C0E7E868132823D0E868142820D0E4
:10D36000E86811281DD0E86812281AD0E868182843
:10D3700017D0E8681C2814D0E8681D2811D0E86888
:10D3800015280ED0E8680E280BD0E868052808D0CC
:10D39000E868062805D0E868022802D0E868032873
:10D3A00022D1012001900020009001231F220021A2
:10D3B000E86800F086FDE860CCE7012001900020DD
:10D3C000009001231F220021E86800F07AFDE86048
:10D3D000E8680528F1D0E8680628EED0E868022859
:10D3E000EBD0E8680328E8D0E86801F0D6F9686176
:10D3F0000FE047F673116961006810F0C04F08D064
:10D400002000C0B201F0E1F92000C0B200F055FEEA
:10D41000E86037BD38B50400DFF804040168C900CE
:10D420000AD5DFF8F8532100C9B2E86801F0F4F832
:10D4300000F0FCFC28608FE0DFF8C8170968C9001D
:10D4400005D4DFF8D8130A688B689A426DD02000A3
:10D45000C0B200F032FE0D2809D00C2807D00E28EB
:10D4600005D000F0E3FCDFF8B413086006E020000C
:10D47000C0B201F073F8DFF8A413C8602000C0B296
:10D48000012807D02000C0B2052803D02000C0B278
:10D49000092805D140F27160DFF8801348613FE050
:10D4A0002000C0B20B2805D140F27160DFF86C1388
:10D4B000486135E02000C0B20C2805D147F6711054
:10D4C000DFF8581348612BE02000C0B2022807D0D3
:10D4D0002000C0B2062803D02000C0B20A2805D11F
:10D4E00045F67130DFF83413486119E02000C0B20E
:10D4F000032803D02000C0B2072805D144F671707C
:10D50000DFF8181348610BE0E4B2082C04D145F6AB
:10D510007130C249486103E046F27160BF49486119
:10D5200000F0A6FCBD49086016E017220A710068E9
:10D5300010F0C04F07D0C868002802D14020C86052
:10D5400001E00020C860C868002803D145F25C40B3
:10D55000486101E06E20486131BD1CB51E20F6F720
:10D56000E1FC072804D01E20F6F7DCFC0A2804D1D1
:10D5700000F05CFCA949086050E0A9490868C000B7
:10D5800009D5A64C0022E1681420F6F76EFD00F0E4
:10D590004DFC206042E0DFF86C060068C00004D457
:10D5A0009E4C2068A26890420BD09C4C47F23F30C2
:10D5B00060611420F6F7B6FCE06000F059FC2060D2
:10D5C0002CE008202071E0680522B0FBF2F302FB9A
:10D5D0001300002817D1002001900120009005239E
:10D5E00064221421E06800F06CFCE060E0686428CC
:10D5F00003D145F25C40606110E00121E06800F079
:10D6000034FD60610AE047F673106061086810F04D
:10D61000C04F03D01420F5F7DFFCE06013BD10B558
:10D620007F480068C00004D500F000FC7B4908601A
:10D630008DE0DFF8D0050068C00007D5774C40F2D8
:10D640005460606100F014FC206080E0734C18208E
:10D650002071002060610120F7F73DFC002803D015
:10D66000606950F4005060610820F7F734FC00282E
:10D6700003D0606950F4805060611020F7F72BFCF4
:10D68000002803D0606950F0200060612020F7F787
:10D6900022FC002803D0606950F010006061402037
:10D6A000F7F719FC002803D0606950F004006061AE
:10D6B0008020F7F710FC002803D0606950F00200CA
:10D6C00060614FF48070F7F706FC002803D06069B2
:10D6D00050F4804060614FF40070F7F7FCFB0028C5
:10D6E00003D0606950F0400060614FF48040F7F76C
:10D6F000F2FB002803D0606950F4006060614FF4D1
:10D700008060F7F7E8FB002805D14FF40060F7F7D9
:10D71000E2FB002803D0606950F0080060614FF41C
:10D720008050F7F7D8FB002803D0606950F4807070
:10D7300060614FF40050F7F7CEFB002803D060691A
:10D7400050F001006061606950F08000606110BDC0
:10D750001CB51E20F6F7E6FB072804D01E20F6F7BE
:10D76000E1FB0A2804D100F061FB2C49086053E07A
:10D770000620F6F7F3FB002804D100F057FB2749F9
:10D78000086049E026490868C00009D5234C0022FA
:10D79000E1683D20F6F769FC00F048FB20603BE0C3
:10D7A000DFF860040068C00004D41C4C2068A26844
:10D7B00090420BD0194C47F2713060613D20F6F772
:10D7C000B1FBE06000F054FB206025E019202071DF
:10D7D000E0680522B0FBF2F302FB1300002810D131
:10D7E000002001900120009005235F220521E068C0
:10D7F00000F067FBE0600121E06800F036FC60614A
:10D800000AE047F673106061086810F0C04F03D05B
:10D810003D20F5F7E1FBE06013BD0000CC280020BF
:10D82000AC2A00201CB5DFF8380B0168C90008D508
:10D83000DFF8304BE06801F054F800F0F7FA2060B0
:10D8400041E0DFF8C0130968C90005D4DFF8144BC4
:10D850002168A26891420BD0DFF8084B47F6774069
:10D86000606101F01EF8E06000F002FB20602AE039
:10D870001A212171E168642917D20120019000204A
:10D880000090012304220021E06800F01AFBE06010
:10D89000E068002803D145F25C40606113E001219B
:10D8A000E06800F0E2FB60610DE047F67311616132
:10D8B000006810F0C04F06D000214E20F5F748FE5A
:10D8C00000F0EFFFE06013BD1CB54E20F6F72AFB19
:10D8D000C00705D400F0AAFADFF8881A086042E011
:10D8E000DFF87C0A0168C90008D5DFF8784AE068EB
:10D8F00001F03CF800F09AFA206034E0C149096870
:10D90000C90005D4DFF85C4A2168A26891420BD0B7
:10D91000DFF8504A47F65440606101F001F8E060DA
:10D9200000F0A6FA20601EE01B212171E168642945
:10D9300010D2012001900020009001230422012137
:10D94000E06800F0BEFAE0600121E06800F08DFBC5
:10D95000606108E047F673116161006810F0C04F24
:10D9600001D00420E06013BD1CB5DFF8F4090168A4
:10D97000C90021D5DFF8EC492069E168884217D059
:10D980002069062807D2E068062804D30021202059
:10D99000F6F793FA09E02069052806D3E068052820
:10D9A00003D200212020F6F7A2FAE06801F034F853
:10D9B00000F03CFA206057E092490968C90005D49C
:10D9C000DFF8A0492168A26891420DD0DFF89449A0
:10D9D00047F63810606100F0EBFFE060E06820611E
:10D9E00000F046FA20603FE01C212171E1686429C3
:10D9F00028D21E20F6F796FA09280BD101200190B3
:10DA000000200090012305220021E06800F059FA6F
:10DA1000E0600AE0012001900020009001230A222A
:10DA20000021E06800F04DFAE060E068002803D1D2
:10DA300045F25C40606117E00121E06800F015FBF1
:10DA4000606111E047F673116161006810F0C04F2A
:10DA50000AD000214D20F5F77BFD00212020F6F7AC
:10DA600046FA00F0A5FFE06013BD38B54D20F6F78B
:10DA700059FA10F00F0F03D010F0C000402805D164
:10DA800000F0D4F9DFF8DC1808603CE0DFF8D0588B
:10DA90002868C00005D500F0C9F9DFF8C81808608B
:10DAA00031E058480068C00008D5DFF8B84846F6AD
:10DAB0003E50606100F0DCF9206024E0DFF8A4480B
:10DAC0001D2020712020F6F7F4F9E060286810F09E
:10DAD000C04F07D0E068002802D00020E06001E0DD
:10DAE0000120E060E068002806D06E20606100211F
:10DAF0002020F6F7E2F906E045F25C406061002183
:10DB00002020F6F7F4F931BD7CB5DFF854582868C9
:10DB1000C00005D500F08AF9DFF84818086070E009
:10DB200038480068C00008D5DFF8384845F25E4044
:10DB3000606100F09DF9206063E0DFF828481E2056
:10DB400020713A20F6F7EEF9E060E0683C2814D244
:10DB5000002001900120009001233C220021E06878
:10DB600000F0AFF9E060E0683C282DD2E0680028C2
:10DB700024D145F25C4060613EE0E0680A21B0FBE0
:10DB8000F1F201FB120000280BD1002001900120CE
:10DB900000900A23F0220021E06800F092F9E06092
:10DBA000E1E7286810F0C04F04D03920F5F714FAE7
:10DBB000E060D8E747F67310606122E00121E06879
:10DBC00000F053FA606117E0E0683C21B0FBF1F02F
:10DBD000E1683C22B1FBF2F302FB13110A22B1FB14
:10DBE000F2F500F01BFA0600280000F017FA50EAE0
:10DBF000062050F0800060610022E1683A20F6F7CC
:10DC000034FA73BDA82A00203EB50400DFF850079F
